:020000041000EA
:10000000784B0020D9060110E1060110E30601102B
:1000100000000000000000000000000000000000E0
:10002000000000000000000000000000E5060110D4
:100030000000000000000000E7060110E9060110C2
:1000400000000000EB060110173A0110EB0601104A
:10005000EB060110EB060110B302001013050010AF
:10006000BB3201106B3301105F340110EB0601103D
:10007000B50A0010EB060110EB060110EB060110AB
:10008000B1140010EB060110EB060110EB06011095
:10009000EB060110EB060110EB060110EB06011058
:1000A0000000000000000000000000000000000050
:1000B0000000000000000000000000000000000040
:1000C0000348854614F09EFC0048004745F00010A8
:1000D000784B002010B5FE480068C07B8009800185
:1000E000C01CFB490968C873F9480068007C800996
:1000F0008001001DF64909680874F5480068203041
:10010000807820218843F249096820318870F048BE
:1001100000682030807840218843ED49096820310B
:100120008870EC480068807840084000E949096818
:100130008870E84800680078000900010830E54947
:1001400009680870E3480068007880218843E14925
:1001500009680870DF480068007840218843403013
:10016000DC4909680870DB480068C07810218843C2
:100170001030D8490968C870D648006880780421D2
:100180008843001DD34909688870D2480068807888
:1001900020218843CF4909688870CE48006880785C
:1001A00010218843CB4909688870CA480068807864
:1001B00080218843C74909688870C64800688078EC
:1001C00040218843C34909688870C24800680078A4
:1001D00010218843BF4909680870BE48006800784C
:1001E00020218843BB4909680870BA4800688078B4
:1001F00002218843801CB74909688870B5480068A7
:10020000C078202188432030B2490968C870062090
:1002100000F0A2F9AF4800688078082188430830D0
:10022000AC490968887010BDAA490968487000BFC8
:10023000A849096809788906C90F0029F8D0A54995
:100240000968097820229143A24A12681170704708
:1002500018B5024600200023009314E09D4B1B6854
:100260001B790B54431CD8B26B461B785B1CDCB269
:1002700000946B461B785B1CDCB200946B461B78C9
:100280005B1CDCB20094934B1B68DB78DB07DB0F55
:10029000002BE3D0107018BD10B58E480068807830
:1002A000082188438B4909688870062000F061F9AD
:1002B00010BD0CB5874800680078C006C00F002844
:1002C0000CD084480068007810218843814909686F
:1002D0000870694601A8FFF7BBFF00BF7D480068B2
:1002E00000788006C00F002807D07A4800680078A0
:1002F000202188437749096808707648006880782B
:100300008007C00F002808D072480068807802215A
:100310008843801C6F49096888700CBD10B56C4813
:100320000068007B80098001401D694909680873E5
:1003300067480068407B80098001801D6449096826
:100340004873634800682030407810218843604932
:100350000968203148705E480068203040782021CC
:1003600088435B490968203148705B4800688078A1
:10037000400840005849096888705748006800786C
:1003800000090001401C544909680870524800687F
:100390000078802188435049096808704E480068F9
:1003A0000078402188434C49096808704A48006831
:1003B000C07810218843103047490968C870464802
:1003C0000068807804218843001D434909688870CB
:1003D000414800688078202188433F490968887037
:1003E0003D4800688078102188433B49096888703F
:1003F00039480068807880218843374909688870C7
:1004000035480068807840218843334909688870FE
:10041000314800680078102188432F490968087026
:100420002D4800680078202188432B49096808700E
:1004300029480068807802218843801C2649096881
:10044000887025480068C0782021884320302249E0
:100450000968C870072000F07FF81F48006880789E
:100460000821884308301C490968887010BD1A4962
:100470000968487000BF1849096809788906C90FDA
:100480000029F8D014490968097820229143124ABA
:1004900012681170704718B50246002000230093BF
:1004A00014E00D4B1B681B790B54431CD8B26B46F0
:1004B0001B785B1CDCB200946B461B785B1CDCB2C7
:1004C00000946B461B785B1CDCB20094024B05E089
:1004D0000830002000300020043000201B68DB784A
:1004E000DB07DB0F002BDCD0107018BD10B52848DF
:1004F00000688078082188432549096888700720AA
:1005000000F037F810BD0CB5694601A8FFF7C3FF2E
:100510000CBD00B51E4800680078C006C00F00285A
:1005200009D01B48006800781021884318490968E1
:100530000870FFF7E8FF1648006880788007C00F52
:10054000002808D012480068807802218843801C67
:100550000F490968887000BD002809DB00BF00BF93
:10056000C206D20E012191400A4A116000BF00BFAD
:10057000704700280ADBC206D20E01219140054ACD
:1005800080321160BFF34F8FBFF36F8F7047000051
:100590000430002000E100E0002109E0002201E039
:1005A000531C9AB27D239B019A42F9DB4B1C99B2F2
:1005B0008142F3DB7047002107E0002201E0531C79
:1005C0009AB2082AFBDB4B1C99B28142F5DB7047DB
:1005D00010B50246002010E0012383401340002B99
:1005E0000AD0FE4B1B6819540123834014469C43D8
:1005F0002246002A00D102E0401C2028ECD300BF94
:1006000010BDFCB50346F64C221D0192002200925B
:10061000002B02D1F34A009203E0012B01D1F24AF0
:100620000092009A002A36D0002013E00122824076
:100630000D461540002D0CD02568009E375C012624
:10064000BE40354325600D4695432946002900D11B
:1006500002E0401C1828E9D300BF182017E001254C
:1006600085402A460D461540002D0FD0019D2D785E
:100670000646183E0127B7403D43EEB2019D2E705D
:100680000D4695432946002900D102E0401C202850
:10069000E5D300BF00BFFCBDFCB50346D04C221D16
:1006A000019200220092002B02D1CE4A009203E078
:1006B000012B01D1CC4A0092009A002A35D00020AB
:1006C00013E0012282400D461540002D0CD0256814
:1006D000009E375C0126BE40B54325600D4695431C
:1006E0002946002900D102E0401C1828E9D300BFA8
:1006F000182016E0012585402A460D461540002D9C
:100700000ED0019D2D780646183E0127B740BD4307
:10071000019E35700D4695432946002900D102E01F
:10072000401C2028E6D300BF00BFFCBDAF490968CC
:100730000A461378194653781B02194393781B0411
:100740001943D278120611438143A84A12681170E6
:100750000B0A53700B0C9370090ED170704710B5D3
:10076000A24A126813461C7822465C78240222436F
:100770009C7824042243DB781B061A4302439B4BDC
:100780001B681A70140A5C70140C9C70120EDA70DC
:10079000974A126813461C7822465C78240222434A
:1007A0009C7824042243DB781B061A430243904BB7
:1007B0001B681A70140A5C70140C9C70120EDA70AC
:1007C0008B4A12680823D3181C7822465C782402CE
:1007D00022439C7824042243DB781B061A4382437D
:1007E000834B1B681A72140A5C72140C9C72120EF2
:1007F000DA727F4A12680823D3181C7822465C7884
:10080000240222439C7824042243DB781B061A43EB
:100810000A43774B1B681A72140A5C72140C9C72A0
:10082000120EDA7210BD714909680A46137819462A
:1008300053781B02194393781B041943D27812068C
:1008400011430143694A126811700B0A53700B0C73
:100850009370090ED1707047654909680A4613788C
:10086000194653781B02194393781B041943D27815
:100870001206114301435E4A126811700B0A53704D
:100880000B0C9370090ED1707047594909680A46DC
:100890001378194653781B02194393781B041943A4
:1008A000D278120611438143514A126811700B0A23
:1008B00053700B0C9370090ED17070474D49096845
:1008C0000A461378194653781B02194393781B0480
:1008D0001943D278120611430143464A1268117037
:1008E0000B0A53700B0C9370090ED170704741497D
:1008F00009680A461378194653781B0219439378FE
:100900001B041943D278120611438143394A1268F5
:1009100011700B0A53700B0C9370090ED170704755
:10092000344909680A461378194653781B0219435B
:1009300093781B041943D2781206114341402D4A83
:10094000126811700B0A53700B0C9370090ED17062
:100950007047014626480068021D137818465378F0
:100960001B02184393781B041843D27812061043D5
:100970000840704710B50A461F4909681823CB186C
:100980001C7821465C78240221439C78240421436E
:10099000DB781B0619430140174B1B6819700C0AC2
:1009A0005C700C0C9C70090ED970134909681023F7
:1009B000CB181C7821465C78240221439C782404BF
:1009C0002143DB781B06194381430B4B1B681974C9
:1009D0000C0A5C740C0C9C74090E0FE008300020AB
:1009E0008010005020300020383000200C300020D3
:1009F000143000201030002018300020D9744E49E7
:100A0000096820310978490849004B4B1B6820339D
:100A100019704A490A600C21002909DB00BF00BF98
:100A2000CC06E40E0123A340454C236000BF00BF69
:100A300000BF10BD4049096810228A181378194672
:100A400053781B02194393781B041943D27812067A
:100A500011430143384A126811740B0A53740B0C8A
:100A60009374090ED17470470C2000280ADBC2066B
:100A7000D20E01219140324A80321160BFF34F8F74
:100A8000BFF36F8F00BF0020C0432B490968087473
:100A9000020A4A74020C8A74000EC8742648006860
:100AA0002030007840084000401C2349096820316C
:100AB0000870704710B520480068182141180A785E
:100AC00010464A78120210438A7812041043C978FB
:100AD000090608431849096810228A18137819462C
:100AE00053781B02194393781B041943D2781206DA
:100AF0001143884300281ED010480068002802D007
:100B00000E48006880470C480068182141180A7890
:100B100010464A78120210438A7812041043C978AA
:100B200009060843044909680870020A4A70020C61
:100B30008A70000EC87010BD183000201C300020D4
:100B400000E100E070B504460E461546002C1CD1AD
:100B500000212846FFF73CFD29460020FFF751FD04
:100B60000B213046FFF734FD0C212846FFF730FDFE
:100B7000FE480068407920218843FC490968487193
:100B80004F20FA490968C8701DE0012C1BD10021D3
:100B90002846FFF71DFD29460020FFF732FD0D21F5
:100BA0003046FFF715FD0E212846FFF711FDF048EE
:100BB0000068407920218843ED49096848714F2039
:100BC000EB490968C87070BDF8B504460D46164675
:100BD0001F4601200090E548006800798021884385
:100BE0008030E24909680871E04800688078FE2199
:100BF00088436100FE2211400843DC49096888707F
:100C0000DA480068007940218843A9014022114058
:100C10000843D64909680871D44800680670310A4B
:100C20004170D24800684079410949010698401E48
:100C3000C006C00E0143CD48006841713946CD4819
:100C4000069A006812F04CFFC8480068007920211D
:100C500088432030C5490968087100BFC34800684F
:100C600000790007C00F0028F8D0C048006800795C
:100C700008218843BD4909680871BC4800680079AB
:100C80004007C00F002809D0B84800680079042147
:100C90008843B6490968087100200090B34800688D
:100CA000007980218843B149096808710098F8BD2E
:100CB000F8B504460D4616461F4601200090AB4885
:100CC00000680079802188438030A849096808714C
:100CD000A64800688078FE2188436100FE2211400A
:100CE0000843A24909688870A0480068007940213B
:100CF0008843A9014022114008439C4909680871B2
:100D00009A4800680670310A417098480068407936
:100D1000410949010698401EC006C00E0143934890
:100D200000684171914800680079102188431030B3
:100D30008E490968087100BF8C4800680079000777
:100D4000C00F0028F8D0894800680079082188433E
:100D50008649096808718548006800794007C00F16
:100D600000280AD0814800680079042188437F491F
:100D7000096808710020009005E07F48069A016824
:100D8000384612F0ADFE794800680079802188432A
:100D90007649096808710098F8BDF8B504460D4613
:100DA00016461F4601200090714800680079802196
:100DB000884380306E49096808716D480068807802
:100DC000FE2188436100FE221140084368490968FA
:100DD000887067480068007940218843A901402253
:100DE000114008436249096808716148006806704B
:100DF000310A41705E48006840794109490106980E
:100E0000401EC006C00E0143594800684171394672
:100E10005A48069A006812F063FE55480068007947
:100E200020218843203052490968087100BF50488A
:100E3000006800790007C00F0028F8D04C4800680F
:100E40000079082188434A490968087148480068C0
:100E500000794007C00F002809D045480068007994
:100E600004218843424909680871002000904048E5
:100E700000680079802188433D490968087100981D
:100E8000F8BDF8B504460D4616461F4601200090F1
:100E900037480068007980218843803034490968E8
:100EA0000871334800688078FE2188436100FE2283
:100EB000114008432E49096888702D480068007960
:100EC00040218843A901402211400843284909686C
:100ED0000871274800680670310A4170244800688C
:100EE0004079410949010698401EC006C00E0143E1
:100EF0001F48006841711E4800680079102188432E
:100F000010301B490968087100BF19480068007952
:100F10000007C00F0028F8D01548006800790821A4
:100F2000884313490968087111480068007940072F
:100F3000C00F00280AD00E480068007904218843B9
:100F40000B49096808710020009005E00C48069ADA
:100F50000168384612F0C4FD054800680079802118
:100F600088430349096808710098F8BD5030002093
:100F70005C300020543000205830002060300020C9
:100F8000643000200A2814DCFE49096860310870CA
:100F9000020A4A70020C8A70020ECA70F949096886
:100FA000097A090909010207120F1143F54A12686B
:100FB0001172704730B504460D46230013F041FF0F
:100FC0000805325F8CB9E6FEFDFCEF4800688078CA
:100FD00080098001EC4909688870EC480068007855
:100FE00004218843001DE94909680870E848006841
:100FF000007804218843E64909680870E2480068DF
:101000002030007804218843DF49096820310870C6
:10101000DD4800688078800980011C30DA49096861
:1010200088703FE1D8480068C07880098001D649BF
:101030000968C870D54800680078082188430830DE
:10104000D24909680870D2480068007808218843AE
:10105000CF4909680870CC48006820300078082122
:101060008843C949096820310870C7480068C078BA
:10107000800980011C30C4490968C87012E1C24867
:101080000068007980098001BF4909680871BF487C
:1010900000680078102188431030BC490968087046
:1010A000BB480068007810218843B9490968087076
:1010B000B54800682030007810218843B24909689B
:1010C00020310870B04800680079800980011C3028
:1010D000AD4909680871E5E0AB48006840798009CE
:1010E0008001A94909684871A84800680078202152
:1010F00088432030A54909680870A5480068007831
:1011000020218843A249096808709F480068203060
:101110000078202188439C490968203108709A484A
:1011200000684079800980011C309749096848713E
:10113000B8E095480068007F8009800192490968FD
:10114000087792480068C0781021884310308F4992
:101150000968C8708E4800688078400840008C4953
:101160000968887088480068203000791021884319
:10117000854909682031087183480068007F80092B
:1011800080011C308049096808778BE07E48006840
:10119000407F800980017C49096848777B48006866
:1011A000C07820218843203078490968C870784881
:1011B0000068C078202102E073E045E017E0884332
:1011C00073490968C8707048006820300079202190
:1011D00088436D490968203108716B480068407F79
:1011E000800980011C306849096848775AE06648E0
:1011F0000068807F800980016349096888776348B7
:101200000068C07840218843403060490968C87050
:101210005F4800688078102188435D4909688870BC
:1012200059480068203000794021884356490968B0
:101230002031087154480068807F800980011C308B
:101240005149096888772DE04F480068C07F8009C0
:1012500080014D490968C8774C480068C0788021F2
:101260008843803049490968C87049480068C07897
:101270008021884346490968C87043480068203087
:1012800000798021884340490968203108713E482F
:101290000068C07F800980011C303B490968C8771D
:1012A00000E000BF00BF374800684030007F800981
:1012B00080011F30334909684031087731480068A0
:1012C0004030007B40084000401C2E4909684031F6
:1012D00008732C4800684030007A00090001401C67
:1012E00028490968403108720121264800682030E9
:1012F00001710021417127480078FFF743FE214822
:101300000068007D400840001E49096808751D48B6
:1013100000682030007F8009800118301949096871
:101320002031087717480068403000788009800134
:10133000001D1449096840310870012D12D111486F
:10134000006840300079C008C000C01D0D49096820
:101350004031087107210B480068203001720021DC
:1013600041721BE00748006840300079C008C000A7
:10137000401C044909684031087100210148006897
:10138000203009E068300020083000200C300020B8
:10139000143000206C3000200172417258480068FF
:1013A000007C4008400056490968087454480068A9
:1013B000007F40084000401C514909680877102010
:1013C000002809DB00BF00BFC206D20E01219140F8
:1013D0004C4A116000BF00BF00BF30BD002801D0E3
:1013E00049490860464909684031097B4908490074
:1013F000491C434A1268403211734149096809790E
:1014000049084900491C3E4A1268117170473C481E
:1014100000686030007C4007400F00283DD038480D
:101420000068007840084000401C35490968087091
:10143000334800682030007840084000401C3049A4
:101440000968203108702E480068007C4008400080
:101450002B490968087400BF294800686030007C87
:101460004007400F0028F7D100BF25480068007CE6
:10147000C007C00F0028F8D021480068007C400851
:1014800040001F49096808741D480068007F400833
:101490004000401C1A4909680877704718480068DE
:1014A0006030417B027B080210438005800D70474D
:1014B00010B513480068007CC007C00F00281DD07D
:1014C000FFF7ECFF04460E480068007C400840002F
:1014D0000B49096808740A4800684030007B4008DE
:1014E0004000074909684031087307480068002830
:1014F00003D0204604490968884700BF10BD00009A
:101500006830002000E100E0703000201C480068D6
:10151000012108431A4908607047194800680221F0
:1015200008431749086070471548006804210843BC
:101530001349086070471248006810210843104999
:101540000860704710B500230E4A7D210901012073
:1015500011F090FC00230C4A7D21C900022011F0FB
:1015600089FC0023094A7D21C900042011F082FC76
:101570000023074A0749102011F07CFC10BD000031
:10158000943100200D1500101B15001029150010B6
:1015900037150010204E000070B504460E46154663
:1015A0000E20FE4909680870681CFC4909684870EB
:1015B000FA48006884702A463146F8480068C01C22
:1015C00012F08EFA70BD08B510F0D3FD0020009027
:1015D000012269461620FFF7DFFF08BD38B5044633
:1015E000607821780002084301210903884200DD68
:1015F00038BD6078217800020843A17840180121A5
:101600000903884207DD6078217800020843012140
:101610000903081AA070A278617823780902194397
:10162000DF4BC818E11C12F05BFA00BFA3786078AA
:101630002178000208430246DAA100200EF0F2FFF2
:1016400000BF00200090012269461720FFF7A4FF89
:1016500000BFCDE77CB504460D461646684645708A
:10166000290A8170C670310A017104700522694629
:101670001420FFF791FF7CBD7CB504460025601C5B
:1016800012F08CFA064622783146C54810F041FF28
:10169000054600BF601C12F081FA064620783346EA
:1016A0002A46C7A1009000200EF0BCFF00BF002D0D
:1016B00002D10120019001E000200190012201A946
:1016C0001820FFF769FF7CBDF8B5054600BFC2488A
:1016D0000079002808D0C04A1179203A126A5001D6
:1016E000BD4A203A10F0B8FD00BF284612F056FA65
:1016F0000646687929790002084303463246B7A1B5
:1017000000200EF08FFF00BF284612F047FA064671
:1017100068792979000208430346324600210846C9
:1017200010F0A9FD044600BF2246B2A100200EF031
:1017300079FF00BF002C02D10120009001E00020C1
:101740000090012269461820FFF726FFF8BDF8B582
:10175000054600BF00BF284612F020FA0646687909
:10176000297900020843034632469CA100200EF06E
:1017700059FF00BF284612F011FA064668792A7907
:10178000000210430146304610F07AFD044600BFC7
:1017900022469DA100200EF045FF00BF002C02D183
:1017A0000120009001E000200090012269461820ED
:1017B000FFF7F2FEF8BD002804D00021974A11700F
:1017C000974A11700021974A1180974A1180974AD1
:1017D0001180974A1180974A11607047F8B5054605
:1017E0000E462C468F480088002803D08B4800788E
:1017F000002876D12078152843D008DC112822D083
:10180000122830D0132835D014281BD140E01628D8
:1018100006D0202866D0232878D02428F5D19EE051
:1018200000200CF0E1FD00BF83A100200EF0FAFEC5
:1018300000BF022011F062FC0120784908700020EE
:101840007C49086092E000200CF0CEFD00BF7EA134
:1018500000200EF0E7FE00BF042070490870002051
:101860007449086082E0A01CFFF7B8FE05206B49B0
:1018700008707BE0A01CFFF7FFFE06206749087098
:1018800074E0A01CFFF720FF0320644908706DE09E
:10189000E179A2790802104362490880617A227ACC
:1018A0000802104360490880A01C12F077F96149D2
:1018B000086000205D4908805D49088000BFA01CC9
:1018C00012F06CF90746617A227A08021043009000
:1018D000544803883A4661A100200EF0A3FE00BFE1
:1018E00044E044E000200CF07FFD00BF68A1002030
:1018F0000EF098FE00BF022011F000FC07204749BF
:10190000087000204B49086030E0FFE7E179A279D8
:101910000802104343490880617A227A0802104382
:1019200041490880A01C12F039F9424908600020A2
:101930003E4908803E49088000BFA01C12F02EF9E5
:101940000746617A227A08021043009035480388DE
:101950003A4654A100200EF065FE00BF06E0A01C30
:10196000FFF7F5FE03202D49087000BF3EE100207F
:101970002B490870002707E0E85D2D4909884018C9
:101980002B490880781C87B2B742F5DB2846E91757
:10199000890F091889108900691A9FE0903000208A
:1019A0004A070020636D64344B53455454494E47F5
:1019B00057726974652025782025780D0A0000008B
:1019C000436F64655570646174653D2564202578B6
:1019D0002025780D0A000000543200206F74612029
:1019E000737A3A257820636865636B73756D3A2561
:1019F00078200000436F64655570646174657632C9
:101A0000303D25640D0A0000436F646555706461C4
:101A100074657633303D25640D0A0000783000206F
:101A2000793000207A3000207E3000207C30002089
:101A30008030002084300020434D445F46575F458E
:101A4000524153450D0A0000344B53455454494EFE
:101A5000475F4552415345200D0A0000434D445F06
:101A600046575F57524954455F5354415254206F73
:101A700066667365743A25782C73697A653A2578B9
:101A800020636865636B73756D3A25780D0A0000F5
:101A9000464C415348444154415F455241534520CF
:101AA0000D0A0000464C415348444154415F57528F
:101AB0004954455F5354415254206F6666736574B0
:101AC0003A25782C73697A653A25782063686563CE
:101AD0006B73756D3A25780D0A00000029D03246E7
:101AE00029464D4811F0FCFF4C480078022803D0ED
:101AF0004A48007801280AD149490968494A1288A8
:101B00008818454A314610F0A7FB074635E04348A0
:101B10000078082803D04148007807282DD1404993
:101B20000968404A128888183B4A314610F005FB84
:101B300023E03A480078022803D03848007801288A
:101B40000AD137490968374A128888182A46314627
:101B500010F082FB074610E030480078082803D0D8
:101B60002E480078072808D12D4909682D4A128887
:101B700088182A46314610F0E0FA2A480088801971
:101B800028490880084600882749098888422CDBB4
:101B9000264800882649098888420CD123480288B3
:101BA000204801880020FFF755FD00BF21A100203B
:101BB0000EF038FD0CE01D4802881A48018801200B
:101BC000FFF748FD00BF1FA100200EF02BFD00BF56
:101BD00000BF17480388154802881EA100200EF098
:101BE00021FD00BF0020FFF7E6FD00BFF8BD70B586
:101BF00005460C46224800684078821C2149284648
:101C000011F06EFF1E4800684078801C20701D484F
:101C100000210160416070BD343200207830002026
:101C2000843000207C3000207A300020803000207A
:101C30007E30002073656374696F6E204F4B2120E6
:101C40000000000073656374696F6E206661696CE3
:101C5000652120006F74615F726563656976655FF9
:101C6000636865636B3A2578206F74615F736563A1
:101C700074696F6E5F636865636B3A25780D0A005F
:101C8000903000208830002010B500214020FEF761
:101C90009FFC4020FEF74AFD4020FEF70FFE10BDDE
:101CA00010B50122920451000020FEF74BFF0422E0
:101CB00008210120FEF746FF10BD10B50021FF20CE
:101CC0000130FEF785FCFF200130FEF72FFDFF20DD
:101CD0000130FEF7F3FD002101200005FEF778FC3E
:101CE00001200005FEF722FD01200005FEF7E6FDBC
:101CF000002101204004FEF76BFC01204004FEF7A8
:101D000015FD01204004FEF7F2FD00210120C0076F
:101D1000FEF75EFC0120C007FEF708FD0120C007AA
:101D2000FEF7CCFD10BD10B500211020FEF750FCD1
:101D300000211020FEF713FD10210020FEF761FCAA
:101D40001020FEF7A2FD1020FEF774FE00212020D7
:101D5000FEF73EFC20210846FEF701FD2021002071
:101D6000FEF74FFC2020FEF777FD02492020FEF70A
:101D700001FE10BDCDF5001010B511F058FB10BDDF
:101D800010B50449044811F000FB10BD10B511F066
:101D90004EFB10BDB9F50010CC0C000010B50024AE
:101DA00010F09CFB0446002C03D1122010F085FBA0
:101DB00002E0204610F081FB01210620FFF7FAF82F
:101DC00010BD0000F8B506460C4601236A462021E6
:101DD000304600F00DFA0546002D20D16846007807
:101DE00041084900E007C00F0143009168460078B0
:101DF000022188436100022211400143009168469C
:101E0000007804218843A100042211400843009077
:101E100001236A462021304600F0FDF90546284698
:101E2000F8BD10B504462046FEF7B6FB10BDFFB561
:101E300081B00C4615461E4601272B46224601213D
:101E400000960198FFF71DF80746002F02D10120E8
:101E500005B0F0BD0020FBE7FFB581B00C4615468C
:101E60001E4601272B462246012100960198FEF7C7
:101E700094FF0746002F02D1012005B0F0BD0020DD
:101E8000FBE71CB500210191284829490860294831
:101E9000486029488860192008736420FFF7C1FF53
:101EA00001A9234800F0ABFD0021214800F0CFFC40
:101EB00005211F4800F0AFFB10211D4801F0F3FA87
:101EC00010211B4801F01DFB0221194800F02FFBD7
:101ED0000121174800F002FD684600780821884378
:101EE00041180091684600780221884300906946B5
:101EF0000F4801F089F801210D48FFF763FF1CBD71
:101F000010B52020FEF725FD20210840002805D02F
:101F100000BF0AA100200EF085FB05E000BF0AA16A
:101F200000200EF07FFB00BF10BD0000591E001006
:101F30005C3200202F1E0010231E00104163745FCE
:101F400053746174650D0A00496E6163745F537464
:101F50006174650D0A00000010B504462046FEF7C6
:101F60001BFB10BDFFB581B00C4615461E46012770
:101F70002B462246012100960198FEF799FE07465E
:101F8000002F02D1012005B0F0BD0020FBE7FFB516
:101F900081B00C4615461E4601272B4622460121DC
:101FA00000960198FEF710FE0746002F02D101208F
:101FB00005B0F0BD0020FBE708B50021009179488D
:101FC0007949086079484860794888606A200873D0
:101FD000FF200130FEF78BFC6420FFF7BDFF694650
:101FE000714802F031FC684600786C2803D101206A
:101FF0007049087002E000206E49087001216A48AB
:1020000002F02EFC00BF6946674802F046FC6846B5
:1020100000780028F7D18021634803F02BFD0121CF
:10202000614801F0AEFE01215F4801F0B1FD0421DD
:102030005D4801F064FD03215B4802F0ACFD012125
:10204000594802F04AFD08BD5B490978491C5A4AC3
:10205000117011460978062920DB002111705749BB
:102060000988411A09B2564A1180114600228A5E37
:10207000002A03DA00228A5E514202E0504A00211F
:10208000515E1922D201914203DD0121494A917129
:1020900002E00021474A9171484908807047F0B535
:1020A00087B006A9404801F0A4FF6846007E0028DA
:1020B0000AD044493C4802F0EDF842490420085E49
:1020C00012F0BEF94049086040490420085E12F051
:1020D000B7F905463C480168284611F0A0FF0446C0
:1020E0004721090611F046FF374908600846016894
:1020F0004720000611F08FFF059012F031FA0646D6
:10210000334A344B12F024F9044612F065FA2E4992
:10211000086031492C48006811F085FF019012F0E9
:102120001FFA04462D4A2E4B12F0AAF80391029092
:102130002C48006812F014FA0646039B029A11F02C
:10214000EDFF0591049012F047FA26490860084611
:10215000006812F0A9F900B2164988800420085ED0
:10216000FFF772FF1348807901280FD11E491648E6
:10217000006811F058FF05461C4911F091FF044614
:1021800012F092F900B20B49488002E000200949A0
:10219000488007B0F0BD10B50121034802F060FB94
:1021A00010BD00008F1F00106C320020651F001052
:1021B000591F001088320020B4300020B6300020B3
:1021C000B83000209E300020B0300020AA3000201F
:1021D0006666666666664040CDCCCC3DE17A14AE5C
:1021E00047C1664094300020000070420000B443B4
:1021F000FFB581B004460D461746002C02D1401EA3
:1022000005B0F0BD207B66683A462946049BB0477E
:1022100000900098F4E7FFB581B004460D461746DC
:10222000002C02D1401E05B0F0BD207B26683A4646
:102230002946049BB04700900098F4E770B5044627
:10224000204612F0FDF806468321C90511F028FF4B
:1022500005467F21C90511F0E6FE70BD70B5044644
:10226000204612F0EDF806468321C90511F018FF4B
:1022700005460121890711F0D6FE70BD70B50446F0
:10228000204612F0DDF806468321C90511F008FF4B
:1022900005468121C90511F0C6FE70BD70B5044622
:1022A000204612F0CDF806468321C90511F0F8FE4C
:1022B0000546F74911F0B7FE70BDF8B50446204653
:1022C00012F0BEF807468521C90511F0E9FE064661
:1022D0008121C90511F0E4FE0546EE4911F04AFEE0
:1022E000F8BD70B50446204612F0AAF806468521CE
:1022F000C90511F0D5FE05468121C90511F093FEEF
:1023000070BD70B50446204612F09AF80646852145
:10231000C90511F0C5FE05464121090611F083FEED
:1023200070BD70B50446204612F08AF80646852135
:10233000C90511F0B5FE05468321C90511F073FEEC
:1023400070BD70B50446204612F07AF80646852125
:10235000C90511F0A5FE0546CF4911F064FE70BD18
:10236000F8B50446204612F06BF807468521C905EA
:1023700011F096FE06468121C90511F091FE054631
:10238000C44911F0F7FDF8BD70B50446204612F0BF
:1023900057F806468721C90511F082FE05468321BC
:1023A000C90511F040FE70BD70B50446204612F01C
:1023B00047F806468721C90511F072FE054621211E
:1023C000490611F030FE70BD70B50446204612F08B
:1023D00037F806468721C90511F062FE05468521BA
:1023E000C90511F020FE70BD70B50446204612F0FC
:1023F00027F806468721C90511F052FE0546A74970
:1024000011F011FE70BDF8B50446204612F018F820
:1024100007468721C90511F043FE06467F21C905FD
:1024200011F001FE05469B4911F0A4FDF8BD70B501
:1024300005460C460123224607212846FFF7D8FE11
:102440000646304670BDF8B505460C4601236A467F
:1024500007212846FFF7CCFE06466846007840076D
:10246000C00F20703046F8BDF8B505460C46012374
:102470006A4607212846FFF7BBFE064668460078F5
:102480004006C00F20703046F8BDF8B505460C4632
:1024900002236A460C212846FFF7AAFE0646684634
:1024A000407820802078010268460078081800B241
:1024B00020803046F8BDF8B506460C4601236A4632
:1024C0001F213046FFF794FE0546002D0FD16946C7
:1024D0000878C0218843A101C02211400843009020
:1024E00001236A461F213046FFF795FE0546284620
:1024F000F8BDF8B505460C4601236A461F2128465B
:10250000FFF776FE0646684600788009002802D06C
:10251000032806D102E00020207005E0032020708F
:1025200002E00020207000BF00BF3046F8BD7CB53F
:1025300006460C46012301AA20213046FFF758FE2B
:102540000546002D06D101236A4623213046FFF7B8
:102550004FFE0546002D2AD1002C09D1684600798E
:10256000082188430190684600788843083000902D
:10257000012C08D1684600790821884301906846FB
:10258000007888430090022C0AD16846007908211F
:1025900088434118019168460078082188430090DB
:1025A000012301AA20213046FFF735FE0546002D04
:1025B00006D101236A4623213046FFF72CFE05464B
:1025C00028467CBD7CB506460C46012301AA202185
:1025D0003046FFF70DFE0546002D1AD101236A464D
:1025E00023213046FFF704FE0546684600790007C0
:1025F000C00F002802D0022020700AE06846007850
:102600000007C00F002802D00020207001E0012048
:10261000207028467CBDF8B506460C4601236A4664
:1026200020213046FFF7E4FD0546002D0FD1694615
:102630000878F02188432101F022114008430090DE
:1026400001236A4620213046FFF7E5FD054628466E
:10265000F8BDF8B505460C4601236A4620212846F8
:10266000FFF7C6FD0646684600780009030012F031
:10267000E8FB0A06090C171A1D202326292C002026
:10268000207025E00120207022E0022020701FE051
:10269000000040410000C8410000404200004043AB
:1026A0000320207014E00420207011E00520207029
:1026B0000EE0062020700BE00720207008E00820C4
:1026C000207005E00920207002E00020207000BF8B
:1026D00000BF3046F8BDF8B506460C4601236A46F1
:1026E00021213046FFF784FD0546002D0FD16946B4
:1026F000087808218843E10008221140084300902F
:1027000001236A4621213046FFF785FD054628460C
:10271000F8BDF8B505460C4601236A462121284636
:10272000FFF766FD0646684600780007C00F207078
:102730003046F8BDF8B506460C4601236A4621210D
:102740003046FFF755FD0546002D0FD16946087844
:102750003021884321013022114008430090012399
:102760006A4621213046FFF756FD05462846F8BD4A
:10277000F8B505460C4601236A4621212846FFF795
:1027800037FD0646684600788006800F002806D090
:10279000012807D0022808D003280CD108E0002027
:1027A00020700BE00120207008E00220207005E07E
:1027B0000320207002E00320207000BF00BF3046DD
:1027C000F8BDF8B506460C4601236A46212130467D
:1027D000FFF70EFD0546002D0FD169460878C02190
:1027E0008843A101C02211400843009001236A469A
:1027F00021213046FFF70FFD05462846F8BDF8B504
:1028000005460C4601236A4621212846FFF7F0FCC5
:102810000646684600788009002806D0012807D0BF
:10282000022808D003280CD108E0002020700BE01B
:102830000120207008E00220207005E003202070B5
:1028400002E00020207000BF00BF3046F8BDF8B5A0
:1028500006460C4601236A4623213046FFF7C8FC92
:102860000546002D0FD169460878302188432101A3
:10287000302211400843009001236A46232130464C
:10288000FFF7C9FC05462846F8BDF8B505460C46D5
:1028900001236A4623212846FFF7AAFC064668461C
:1028A00000788006800F002806D0012807D0022873
:1028B00008D003280CD108E0002020700BE0012094
:1028C000207008E00220207005E00320207002E064
:1028D0000020207000BF00BF3046F8BDF8B50646A6
:1028E0000C4601236A4623213046FFF781FC05464A
:1028F000002D0FD16946087880218843E1018022AC
:1029000011400843009001236A4623213046FFF717
:1029100082FC05462846F8BDF8B505460C4601235D
:102920006A4623212846FFF763FC0646684600787E
:10293000C00920703046F8BD70B505460C4601232D
:10294000224626212846FFF766FC0646304670BD23
:1029500070B505460C460123224626212846FFF77E
:1029600047FC0646304670BDF8B505460C460123C7
:102970006A4627212846FFF73BFC06466846007852
:102980000007C00F20703046F8BDF8B505460C466C
:1029900001236A4627212846FFF72AFC0646684697
:1029A0000078C00920703046F8BD7CB505460C465D
:1029B00006236A4628212846FFF71AFC0646684681
:1029C000407820802078010268460078081800B21C
:1029D00020806846C0786080A078010268468078D0
:1029E000081800B2608068464079A0802079010212
:1029F00068460079081800B2A08030467CBD70B5EA
:102A000005460C46012322460F212846FFF7F0FB1E
:102A10000646304670BDF8B506460C4601236A46A8
:102A200023213046FFF7E4FB0546002D0FD1694610
:102A3000087806218843610006221140084300906F
:102A400001236A4623213046FFF7E5FB0546284669
:102A5000F8BDF8B505460C4601236A4623212846F1
:102A6000FFF7C6FB0646684600784007800F00283F
:102A700004D0012805D0022809D105E000202070EB
:102A800008E00120207005E00220207002E0002014
:102A9000207000BF00BF3046F8BDF8B506460C46B2
:102AA00001236A4623213046FFF7A2FB0546002D8D
:102AB0000FD16946087840218843A1014022114086
:102AC0000843009001236A4623213046FFF7A3FB09
:102AD00005462846F8BDF8B505460C4601236A466A
:102AE00023212846FFF784FB064668460078400607
:102AF000C00F002802D0012806D102E0002020707B
:102B000005E00120207002E00020207000BF00BF1F
:102B10003046F8BDF8B506460C4601236A46242126
:102B20003046FFF765FB0546002D0FD16946087852
:102B300080218843E1018022114008430090012355
:102B40006A4624213046FFF766FB05462846F8BD55
:102B5000F8B505460C4601236A4624212846FFF7AE
:102B600047FB064668460078C00920703046F8BD2D
:102B700070B505460C460123224627212846FFF75B
:102B800037FB0646304670BD70B505460C4601233E
:102B9000224630212846FFF73EFB0646304670BDF0
:102BA00070B505460C460123224630212846FFF722
:102BB0001FFB0646304670BD70B505460C46012326
:102BC000224631212846FFF713FB0646304670BDEA
:102BD000F8B506460C4601236A4632213046FFF717
:102BE00007FB0546002D0ED169460878C009C001D3
:102BF0006106490E0843009001236A46322130469F
:102C0000FFF709FB05462846F8BDF8B505460C4612
:102C100001236A4632212846FFF7EAFA064668464B
:102C200000784006400E20703046F8BDF8B50646E4
:102C30000C4601236A4633213046FFF7D9FA054690
:102C4000002D0ED169460878C009C0016106490E01
:102C50000843009001236A4633213046FFF7DBFA30
:102C600005462846F8BDF8B505460C4601236A46D8
:102C700033212846FFF7BCFA06466846007840062E
:102C8000400E20703046F8BD70B505460C46012355
:102C9000224634212846FFF7BEFA0646304670BD6C
:102CA00070B505460C460123224634212846FFF71D
:102CB0009FFA0646304670BD70B505460C460123A6
:102CC000224635212846FFF793FA0646304670BD66
:102CD000F8B506460C4601236A4636213046FFF712
:102CE00087FA0546002D0ED169460878C009C00153
:102CF0006106490E0843009001236A46362130469A
:102D0000FFF789FA05462846F8BDF8B505460C4692
:102D100001236A4636212846FFF76AFA06466846C6
:102D200000784006400E20703046F8BDF8B50646E3
:102D30000C4601236A4637213046FFF759FA05460B
:102D4000002D0ED169460878C009C0016106490E00
:102D50000843009001236A4637213046FFF75BFAAB
:102D600005462846F8BDF8B505460C4601236A46D7
:102D700037212846FFF73CFA0646684600784006A9
:102D8000400E20703046F8BDF8B506460C460123CB
:102D90006A4621213046FFF72BFA0546002D0ED159
:102DA00069460878C008C0006107490F08430090D1
:102DB00001236A4621213046FFF72DFA05462846B1
:102DC000F8BDF8B505460C4601236A462121284680
:102DD000FFF70EFA0646684600784007400F0300EA
:102DE00012F02FF80805080B110E14171A1D0020F9
:102DF000207017E00120207014E00220207011E004
:102E0000042020700EE0032020700BE005202070CD
:102E100008E00620207005E00720207002E0002076
:102E2000207000BF00BF3046F8BD70B505460C46A7
:102E30000123224622212846FFF7EDF906463046B7
:102E400070BD70B505460C46012322462221284656
:102E5000FFF7CEF90646304670BDF8B506460C467B
:102E600001236A4624213046FFF7C2F90546002DAA
:102E70000ED16946087840084000E107C90F0843B1
:102E8000009001236A4624213046FFF7C4F9054625
:102E90002846F8BDF8B505460C4601236A462421AC
:102EA0002846FFF7A5F9064668460078C007C00F18
:102EB00020703046F8BDF8B506460C4601236A4638
:102EC00024213046FFF794F90546002D0FD16946BD
:102ED00008780221884361000222114008430090D3
:102EE00001236A4624213046FFF795F90546284616
:102EF000F8BDF8B505460C4601236A46242128464C
:102F0000FFF776F90646684600788007C00F00286C
:102F100002D0012806D102E00020207005E0012047
:102F2000207002E00020207000BF00BF3046F8BDD6
:102F3000F8B506460C4601236A4624213046FFF7C1
:102F400057F90546002D0FD16946087804218843BA
:102F5000A100042211400843009001236A46242165
:102F60003046FFF758F905462846F8BDF8B505463E
:102F70000C4601236A4624212846FFF739F9064604
:102F8000684600784007C00F20703046F8BDF8B59D
:102F900006460C4601236A4624213046FFF728F9ED
:102FA0000546002D0FD16946087808218843E100C5
:102FB000082211400843009001236A46242130462C
:102FC000FFF729F905462846F8BDF8B505460C4631
:102FD00001236A4624212846FFF70AF90646684677
:102FE00000780007C00F002802D0012806D102E0B7
:102FF0000020207005E00120207002E000202070F9
:1030000000BF00BF3046F8BD70B505460C46012331
:10301000224625212846FFF7FEF80646304670BDB9
:1030200070B505460C460123224625212846FFF7A8
:10303000DFF80646304670BDF8B506460C4601235B
:103040006A4624213046FFF7D3F80546002D0FD1FC
:103050006946087840218843A10140221140084375
:10306000009001236A4624213046FFF7D4F8054634
:103070002846F8BDF8B505460C4601236A462421CA
:103080002846FFF7B5F80646684600784006C00FA8
:1030900020703046F8BDF8B506460C4601236A4656
:1030A0002E213046FFF7A4F80546002D0ED16946C3
:1030B000087840094001E106C90E08430090012349
:1030C0006A462E213046FFF7A6F805462846F8BD89
:1030D000F8B505460C4601236A462E212846FFF71F
:1030E00087F8064668460078C006C00E2070304655
:1030F000F8BDF8B506460C4601236A462E21304637
:10310000FFF776F80546002D0FD169460878202193
:1031100088436101202211400843009001236A4640
:103120002E213046FFF777F805462846F8BDF8B55A
:1031300005460C4601236A462E212846FFF758F81B
:103140000646684600788006C00F002802D0012895
:1031500006D102E00020207005E00120207002E08E
:103160000020207000BF00BF3046F8BDF8B506460D
:103170000C4601236A462E213046FFF739F80546F2
:10318000002D0FD169460878C0218843A101C022D3
:1031900011400843009001236A462E213046FFF774
:1031A0003AF805462846F8BDF8B505460C46012311
:1031B0006A462E212846FFF71BF806466846007827
:1031C0008009002806D0012807D0022808D003284B
:1031D0000CD108E0002020700BE00120207008E0F6
:1031E0000220207005E00320207002E00020207003
:1031F00000BF00BF3046F8BD70B505460C46012340
:1032000022462F212846FEF7F3FF0646304670BDC2
:10321000F8B505460C4601236A462F212846FEF7DD
:10322000E7FF064668460078C006C00E20703046AC
:10323000F8BDF8B505460C4601236A462F212846FD
:10324000FEF7D6FF0646684600788006C00F20705D
:103250003046F8BDF8B505460C4601236A462F21D5
:103260002846FEF7C5FF0646684600784006C00FB0
:1032700020703046F8BDF8B505460C4601236A4675
:103280002F212846FEF7B4FF064668460078C0099D
:1032900020703046F8BD70B505460C460123224625
:1032A00038212846FEF7B7FF0646304670BD70B598
:1032B00005460C460123224638212846FEF798FF92
:1032C0000646304670BD70B505460C4601232246C1
:1032D00039212846FEF78CFF0646304670BDF8B50A
:1032E00006460C4601236A463A213046FEF780FF27
:1032F0000546002D0ED169460878C009C001610657
:10330000490E0843009001236A463A213046FEF7F1
:1033100082FF05462846F8BDF8B505460C46012350
:103320006A463A212846FEF763FF0646684600785B
:103330004006400E20703046F8BDF8B506460C46F3
:1033400001236A463A213046FEF752FF0546002D1A
:103350000FD16946087880218843E101802211401D
:103360000843009001236A463A213046FEF753FF96
:1033700005462846F8BDF8B505460C4601236A46C1
:103380003A212846FEF734FF064668460078C00911
:10339000002802D0012806D102E00020207005E0BC
:1033A0000120207002E00020207000BF00BF3046E6
:1033B000F8BDF8B506460C4601236A463B21304667
:1033C000FEF716FF0546002D0ED169460878C009A4
:1033D000C0016106490E0843009001236A463B2163
:1033E0003046FEF718FF05462846F8BDF8B50546F5
:1033F0000C4601236A463B212846FEF7F9FE0646A5
:10340000684600784006400E20703046F8BDF8B59A
:1034100006460C4601236A463C213046FEF7E8FE8C
:103420000546002D08D1E0B2009001236A463C21F8
:103430003046FEF7F0FE05462846F8BDF8B50546CD
:103440000C4601236A463C212846FEF7D1FE06467B
:103450006846007820703046F8BDF8B506460C4640
:1034600001236A463D213046FEF7C2FE0546002D87
:1034700008D1E0B2009001236A463D213046FEF7B4
:10348000CAFE05462846F8BDF8B505460C46012398
:103490006A463D212846FEF7ABFE064668460078A0
:1034A00020703046F8BDF8B506460C4601236A4642
:1034B0003E213046FEF79CFE0546002D0ED16946A2
:1034C0000878C009C0016106490E08430090012335
:1034D0006A463E213046FEF79EFE05462846F8BD68
:1034E000F8B505460C4601236A463E212846FEF7FC
:1034F0007FFE0646684600784006400E2070304643
:10350000F8BDF8B506460C4601236A463F21304611
:10351000FEF76EFE0546002D08D1E0B200900123B3
:103520006A463F213046FEF776FE05462846F8BD3E
:10353000F8B505460C4601236A463F212846FEF7AA
:1035400057FE06466846007820703046F8BDF8B54C
:1035500006460C4601236A461E213046FEF748FE09
:103560000546002D0FD16946087880218843E10186
:10357000802211400843009001236A461E213046F4
:10358000FEF749FE05462846F8BDF8B505460C4647
:1035900001236A461E212846FEF72AFE0646684693
:1035A0000078C009002803D0012804D1207005E06C
:1035B0000020207002E00120207000BF00BF3046D4
:1035C000F8BDF8B506460C4601236A46232130466D
:1035D000FEF70EFE0546002D0ED16946087840081C
:1035E0004000E107C90F0843009001236A462321E8
:1035F0003046FEF710FE05462846F8BDF8B50546EC
:103600000C4601236A4623212846FEF7F1FD0646B3
:1036100068460078C007C00F002802D0012806D1F4
:1036200002E00020207005E00120207002E0002070
:10363000207000BF00BF3046F8BD0000FFB581B06C
:1036400004460D461746002C02D1401E05B0F0BDC1
:10365000207B66683A462946049BB0470090009854
:10366000F4E7FFB581B004460D461746002C02D1A1
:10367000401E05B0F0BD207B26683A462946049BD3
:10368000B04700900098F4E7002803D0002901D04B
:103690000A780270704770B50446204610F0D0FEDC
:1036A0000546F84910F0BFFC70BD70B504462046D1
:1036B00010F0C6FE0546F44910F0B5FC70BD70B5BB
:1036C0000446204610F0BCFE0546F04910F0ABFC65
:1036D00070BD70B50446204610F0B2FE0546EC49B8
:1036E00010F0A1FC70BD70B50446204610F0A8FE95
:1036F0000546E84910F097FC70BD70B504462046B9
:1037000010F09EFE0546E44910F08DFC70BD70B5CA
:103710000446204610F094FE0546E04910F083FC74
:1037200070BD70B50446204610F08AFE0546DC499F
:1037300010F079FC70BD70B50446204610F080FE94
:103740000546D84910F06FFC70BD70B504462046A0
:1037500010F076FE06468721C90510F0A1FC05464B
:10376000D14910F007FC70BD70B50446204610F03A
:1037700067FE0546CD4910F056FC70BDF8B506460B
:103780000C4601236A4610213046FFF757FF0546D5
:10379000002D0FD1694608780C218843A1000C2226
:1037A00011400843009001236A4610213046FFF77C
:1037B00058FF05462846F8BDF8B505460C460123D6
:1037C0006A4610212846FFF739FF0646684600780A
:1037D0000007800F002806D0012807D0022808D053
:1037E00003280CD108E0002020700BE0012020709D
:1037F00008E00220207005E00320207002E0002095
:10380000207000BF00BF3046F8BDF8B505460C4635
:103810000020009069460878C0218843A101C02299
:1038200011400843009001236A4619462846FFF7D5
:1038300018FF06463046F8BDF8B506460C4602218C
:103840003046FFF7E2FF0546002D01D02846F8BDBF
:1038500001236A465F213046FFF7F0FE0546002D42
:1038600000D01DE068460078C006800F002806D012
:10387000012807D0022808D003280CD108E0002036
:1038800020700BE00120207008E00220207005E08D
:103890000320207002E00020207000BF00BF00BFA6
:1038A00000213046FFF7B1FF45192846CFE770B534
:1038B00006460D4602213046FFF7A7FF04460223C5
:1038C0002A4646213046FFF7B9FE0419002130464A
:1038D000FFF79BFF0419204670BDFEB506460C4657
:1038E000274602A93046FFF7E2FF0546002D01D02A
:1038F0002846FEBD6946087AC007C00F097A8907C5
:10390000C90F08436946097A4907C90F0843694640
:10391000097A0907C90F08436946097AC906C90F18
:1039200008436946097A8906C90F08436946097A36
:103930004906C90F08436946097AC9090843694617
:10394000497AC907C90F08436946497A8907C90FE7
:1039500008436946497A4907C90F08436946497AC5
:103960000907C90F08436946497AC906C90F0843C0
:103970006946497A8906C90F08436946497A490662
:10398000C90F08436946497AC9090843002846D047
:1039900001A93046FFF750FF0546002D01D028460B
:1039A000A7E768460079002806D001280AD0022837
:1039B00012D0032830D11DE0002C01D1012700E0F6
:1039C00027462BE0002C01D1022704E0012C01D175
:1039D000022700E0274621E0002C01D1032708E060
:1039E000012C01D1032704E0022C01D1032700E0C0
:1039F000274613E0002C01D104270CE0012C01D153
:103A0000042708E0022C01D1042704E0032C01D193
:103A1000042700E0274601E0274600BF00BF01233E
:103A20006A4610213046FFF709FE054669460878C8
:103A3000F02188433901F02211400843009001230E
:103A40006A4610213046FFF70CFE4519284650E71C
:103A5000F8B505460C4601236A4610212846FFF7B3
:103A6000EDFD0646684600780009030011F0E9F90B
:103A70000C07202326292C2F3235383B3E410020CD
:103A8000207039E023DB793D23DBF93D23DB793EF0
:103A900023DBF93E00008C4000008C4100000C410B
:103AA00000000C4200008C420000C8410050C34698
:103AB0000120207020E0022020701DE003202070F3
:103AC0001AE00420207017E00520207014E0062082
:103AD000207011E0072020700EE0082020700BE01D
:103AE0000920207008E00A20207005E00B202070DB
:103AF00002E00020207000BF00BF3046F8BDF8B5DE
:103B000006460C4601236A4611213046FFF796FD12
:103B10000546002D0FD1694608780E2188436100C3
:103B20000E2211400843009001236A4611213046BD
:103B3000FFF797FD05462846F8BDF8B505460C4643
:103B400001236A4611212846FFF778FD064668469C
:103B500000780007400F030011F073F90705080B08
:103B6000140E14111400002020700EE001202070AB
:103B70000BE00220207008E00420207005E0062001
:103B8000207002E00020207000BF00BF3046F8BD6A
:103B9000FEB506460C46274602A93046FFF787FECB
:103BA0000546002D01D02846FEBD6946087AC007AB
:103BB000C00F097A8907C90F08436946097A49077E
:103BC000C90F08436946097A0907C90F08436946BE
:103BD000097AC906C90F08436946097A8906C90FD7
:103BE00008436946097A4906C90F08436946097AB4
:103BF000C90908436946497AC907C90F0843694694
:103C0000497A8907C90F08436946497A4907C90FA4
:103C100008436946497A0907C90F08436946497A42
:103C2000C906C90F08436946497A8906C90F08437E
:103C30006946497A4906C90F08436946497AC9095C
:103C40000843002846D001A93046FFF7F5FD054698
:103C5000002D01D02846A7E768460079002806D045
:103C600001280AD0022812D0032830D11DE0002CF0
:103C700001D1012700E027462BE0002C01D10227CB
:103C800004E0012C01D1022700E0274621E0002CAE
:103C900001D1032708E0012C01D1032704E0022C05
:103CA00001D1032700E0274613E0002C01D10427AF
:103CB0000CE0012C01D1042708E0022C01D10427DB
:103CC00004E0032C01D1042700E0274601E0274649
:103CD00000BF00BF01236A4611213046FFF7AEFC4A
:103CE000054669460878F02188433901F0221140E1
:103CF0000843009001236A4611213046FFF7B1FCCA
:103D00004519284650E7F8B505460C4601236A4692
:103D100011212846FFF792FC064668460078000904
:103D2000030011F08EF80B070A0D101316191C1F53
:103D3000222528000020207020E0012020701DE0B6
:103D4000022020701AE00320207017E00420207069
:103D500014E00520207011E0062020700EE00720FE
:103D600020700BE00820207008E00920207005E09A
:103D70000A20207002E00020207000BF00BF304603
:103D8000F8BDF8B506460C4601236A4612213046B6
:103D9000FFF754FC0546002D0FD1694608784021F5
:103DA0008843A101402211400843009001236A4644
:103DB00012213046FFF755FC05462846F8BDF8B5F8
:103DC00005460C4601236A4612212846FFF736FCB9
:103DD0000646684600784006C00F20703046F8BDA1
:103DE000F8B506460C4601236A4615213046FFF712
:103DF00025FC0546002D0FD1694608780821884327
:103E0000E100082211400843009001236A46152171
:103E10003046FFF726FC05462846F8BDF8B50546AE
:103E20000C4601236A4615212846FFF707FC064683
:103E3000684600780007C00F002802D0012806D18C
:103E400002E00020207005E00120207002E0002048
:103E5000207000BF00BF3046F8BD7CB506460D4659
:103E6000012301AA14213046FFF7E8FB0446002C89
:103E700001D020467CBD6946087980218843022113
:103E800029404908C90180221140084301900123BB
:103E900001AA14213046FFF7E4FB0446002C01D0B0
:103EA0002046E7E701236A4615213046FFF7C6FBA7
:103EB0000446002C01D02046DCE769460878102132
:103EC00088432901102211400843009001236A46CB
:103ED00015213046FFF7C5FB04462046CAE77CB5EE
:103EE00006460C46012301AA14213046FFF7A6FB23
:103EF0000546002D22D101236A4615213046FFF7E1
:103F00009DFB054669460879C00940000978C90645
:103F1000C90F0843002804D0012805D0022809D180
:103F200005E00020207008E00120207005E002205C
:103F3000207002E00020207000BF00BF28467CBD3A
:103F4000F8B506460C4601236A4616213046FFF7AF
:103F500075FB0546002D0FD16946087880218843FE
:103F6000E101802211400843009001236A46162196
:103F70003046FFF776FB05462846F8BDF8B50546FE
:103F80000C4601236A4616212846FFF757FB0646D2
:103F900068460078C009002802D0012806D102E056
:103FA0000020207005E00120207002E00020207039
:103FB00000BF00BF3046F8BD70B505460C46012372
:103FC00022461E212846FFF739FB0646304670BDC3
:103FD000F8B505460C4601236A461E212846FFF720
:103FE0002DFB064668460078C007C00F207030469B
:103FF000F8BDF8B505460C4601236A461E21284641
:10400000FFF71CFB0646684600788007C00F20704B
:104010003046F8BDF8B505460C4601236A461E2118
:104020002846FFF70BFB0646684600784007C00F9E
:1040300020703046F8BD70B505460C460123224677
:1040400073212846FFF70DFB0646304670BD70B55C
:1040500005460C460123224673212846FFF7EEFA57
:104060000646304670BD70B505460C460123224613
:1040700074212846FFF7F5FA0646304670BD70B544
:1040800005460C460123224674212846FFF7D6FA3E
:104090000646304670BD70B505460C4601232246E3
:1040A00075212846FFF7DDFA0646304670BD70B52B
:1040B00005460C460123224675212846FFF7BEFA25
:1040C0000646304670BDF8B506460C4601236A46E2
:1040D00016213046FFF7B2FA0546002D0FD169468A
:1040E00008780221884361000222114008430090B1
:1040F00001236A4616213046FFF7B3FA05462846E3
:10410000F8BDF8B505460C4601236A461621284637
:10411000FFF794FA0646684600788007C00F2070C3
:104120003046F8BD38B50446AA20009001236A46FF
:1041300042212046FFF795FA38BDF8B506460C46F1
:1041400001236A4619213046FFF778FA0546002D0B
:104150000FD169460878202188436101202211404F
:104160000843009001236A4619213046FFF779FA87
:1041700005462846F8BDF8B505460C4601236A46B3
:1041800019212846FFF75AFA064668460078800645
:10419000C00F20703046F8BDF8B505460C46042324
:1041A0006A4640212846FFF749FA06466846C07825
:1041B0002060206801026846807808182060206826
:1041C00001026846407808182060206801026846AD
:1041D0000078081820603046F8BDF8B506460C4651
:1041E00001236A4614213046FFF728FA0546002DC0
:1041F0000FD169460878602188436101602211402F
:104200000843009001236A4614213046FFF729FA3B
:1042100005462846F8BDF8B505460C4601236A4612
:1042200014212846FFF70AFA064668460078400639
:10423000800F002806D0012807D0022808D00328C4
:104240000CD108E0002020700BE00120207008E075
:104250000220207005E00320207002E00020207082
:1042600000BF00BF3046F8BDF8B505460C46022336
:104270006A4620212846FFF7E1F90646684640785D
:1042800020802078010268460078081800B220805B
:104290003046F8BD7CB505460C4606236A46222109
:1042A0002846FFF7CBF906466846407820802078FC
:1042B000010268460078081800B220806846C0787D
:1042C0006080A078010268468078081800B260809B
:1042D00068464079A0802079010268460079081874
:1042E00000B2A08030467CBD7CB505460C46062356
:1042F0006A4628212846FFF7A1F906466846407815
:1043000020802078010268460078081800B22080DA
:104310006846C0786080A0780102684680780818F6
:1043200000B2608068464079A0802079010268462A
:104330000079081800B2A08030467CBD70B50546F3
:104340000C460623224679212846FFF777F90646D0
:10435000304670BDF8B506460C4602213046FFF7E0
:1043600054FA0546002D01D02846F8BD02236A46BE
:1043700062213046FFF762F90546002D00D009E0C2
:104380006846407820802078010268460078081846
:10439000208000BF00213046FFF737FA4519284634
:1043A000E3E738B5054602212846FFF72EFA044612
:1043B000002C01D0204638BD01236A4664212846DE
:1043C000FFF73CF90446002C00D00DE06946087860
:1043D000802188438030009001236A46642128466A
:1043E000FFF73FF9044600BF00212846FFF70DFA0A
:1043F00004192046DFE7F8B506460C4601236A4655
:1044000063213046FFF71AF90546002D08D1E0B2C6
:10441000009001236A4663213046FFF722F90546E2
:104420002846F8BDF8B505460C4601236A466321C7
:104430002846FFF703F906466846007820703046A4
:10444000F8BDF8B505460C4601236A4619462846CC
:10445000FFF7F4F80646684600788009002804D083
:10446000012805D0022809D105E00020207008E0CD
:104470000120207005E00220207002E00020207062
:1044800000BF00BF3046F8BDFFB585B00F46380508
:10449000000F0190FDB202210598FFF7B6F904461E
:1044A000002C02D0204609B0F0BD012304AA172138
:1044B0000598FFF7C3F804466946087C60218843E5
:1044C00040300490012304AA17210598FFF7C9F88A
:1044D0000419002C00D097E0012303AA02210598BB
:1044E000FFF7ACF804466846007BF0218843019949
:1044F0000901F0221140014303916846007B000945
:104500000001401C0390012303AA02210598FFF734
:10451000A8F80419002C00D076E0E8B2029001233C
:1045200002AA08210598FFF79CF80419002C00D076
:104530006AE000263AE007988219012309210598CC
:10454000FFF78FF80446002C00D05DE0681CC5B270
:10455000002D29D1002C27D10198401CC0B2019018
:10456000012303AA02210598FFF768F80419002C1B
:1045700000D049E06846007BF02188430199090199
:10458000F0221140014303916846007B00090001BD
:10459000401C0390012303AA02210598FFF761F84C
:1045A0000446002C00D02FE0701CC6B2089886424A
:1045B00001DA002CBFD06846007BF02188430390CD
:1045C0006846007B00090001401C0390012303AAF8
:1045D00002210598FFF745F80446002C00D013E0AF
:1045E000012304AA17210598FFF728F80446694615
:1045F000087C602188430490012304AA17210598B0
:10460000FFF72FF8041900BF00210598FFF7FDF808
:104610000419204647E770B504460D4616460123A7
:10462000324629462046FFF72FFF70BDFFB585B003
:104630000F463805000F0190FDB202210598FFF7E3
:10464000E4F80446002C02D0204609B0F0BD012356
:1046500004AA17210598FEF7F1FF04466946087C75
:104660006021884320300490012304AA1721059873
:10467000FEF7F7FF0419002C00D097E0012303AAEE
:1046800002210598FEF7DAFF04466846007BF02118
:10469000884301990901F0221140014303916846C2
:1046A000007B00090001401C0390012303AA0221A2
:1046B0000598FEF7D6FF0419002C00D076E00026FE
:1046C00046E0E8B20290012302AA08210598FEF70D
:1046D000C8FF0446002C00D068E007988219012327
:1046E00009210598FEF7AAFF0419002C00D05DE00F
:1046F000681CC5B2002D29D1002C27D10198401C7F
:10470000C0B20190012303AA02210598FEF796FF8B
:104710000419002C00D049E06846007BF021884352
:1047200001990901F0221140014303916846007B81
:1047300000090001401C0390012303AA02210598EF
:10474000FEF78FFF0419002C00D02FE0701CC6B2BA
:104750000898864201DA002CB3D06846007BF0212D
:10476000884303906846007B00090001401C0390C9
:10477000012303AA02210598FEF773FF0446002CCB
:1047800000D013E0012304AA17210598FEF756FF75
:1047900004466946087C602188430490012304AAEA
:1047A00017210598FEF75DFF041900BF0021059849
:1047B000FFF72BF80419204647E770B504460D466D
:1047C00016460123324629462046FFF72FFF70BDCB
:1047D000F8B506460C4601236A460B213046FEF723
:1047E0002DFF0546002D0FD16946087880218843AA
:1047F000E101802211400843009001236A460B2109
:104800003046FEF72EFF05462846F8BDF8B50546AA
:104810000C4601236A460B212846FEF70FFF064689
:1048200068460078C009002802D0012806D102E0BD
:104830000020207005E00120207002E000202070A0
:1048400000BF00BF3046F8BD70B505460C460123D9
:1048500022460F212846FEF7F1FE0646304670BD7F
:10486000F8B506460C4601236A4612213046FEF78B
:10487000E5FE0546002D0ED1694608784008400047
:10488000E107C90F0843009001236A461221304610
:10489000FEF7E7FE05462846F8BDF8B505460C4686
:1048A00001236A4612212846FEF7C8FE06466846DE
:1048B0000078C007C00F20703046F8BDF8B5064636
:1048C0000C4601236A4612213046FEF7B7FE054624
:1048D000002D0FD16946087804218843A1000422E5
:1048E00011400843009001236A4612213046FEF72A
:1048F000B8FE05462846F8BDF8B505460C46012326
:104900006A4612212846FEF799FE06466846007858
:104910004007C00F20703046F8BDF8B506460C467B
:1049200001236A4612213046FEF788FE0546002D17
:104930000FD16946087880218843E1018022114027
:104940000843009001236A4612213046FEF789FE93
:1049500005462846F8BDF8B505460C4601236A46CB
:1049600012212846FEF76AFE064668460078C0090E
:1049700020703046F8BDF8B506460C4601236A465D
:1049800014213046FEF75AFE0546002D0ED1694629
:10499000087880088000A107890F08430090012350
:1049A0006A4614213046FEF75CFE05462846F8BDEF
:1049B000F8B505460C4601236A4614212846FEF741
:1049C0003DFE0646684600788007800F002804D028
:1049D000012805D0022809D105E00020207008E058
:1049E0000120207005E00220207002E000202070ED
:1049F00000BF00BF3046F8BDF8B506460C4601239F
:104A00006A4614213046FEF719FE0546002D0FD1E7
:104A1000694608780C218843A1000C221140084304
:104A2000009001236A4614213046FEF71AFE05461F
:104A30002846F8BDF8B505460C4601236A46142100
:104A40002846FEF7FBFD0646684600780007800F03
:104A5000002804D0012805D0032809D105E0002052
:104A6000207008E00120207005E00320207002E0A3
:104A70000020207000BF00BF3046F8BDF8B50646E4
:104A80000C4601236A4610213046FEF7D7FD054645
:104A9000002D0FD169460878022188436100022267
:104AA00011400843009001236A4610213046FEF76A
:104AB000D8FD05462846F8BDF8B505460C46012345
:104AC0006A4610212846FEF7B9FD0646684600787A
:104AD0008007C00F20703046F8BDF8B506460C467A
:104AE00001236A4613213046FEF7A8FD0546002D36
:104AF0000FD16946087802218843610002221140E3
:104B00000843009001236A4613213046FEF7A9FDB1
:104B100005462846F8BDF8B505460C4601236A4609
:104B200013212846FEF78AFD06466846007880076E
:104B3000C00F20703046F8BDF8B506460C4601237C
:104B40006A4613213046FEF779FD0546002D0FD148
:104B50006946087808218843E1000822114008438B
:104B6000009001236A4613213046FEF77AFD054680
:104B70002846F8BDF8B505460C4601236A461321C0
:104B80002846FEF75BFD0646684600780007C00F22
:104B900020703046F8BDF8B506460C4601236A463B
:104BA00015213046FEF74AFD0546002D0ED1694617
:104BB0000878C008C0006107490F0843009001232E
:104BC0006A4615213046FEF74CFD05462846F8BDDD
:104BD000F8B505460C4601236A4615212846FEF71E
:104BE0002DFD0646684600784007400F030010F090
:104BF00028F90805080B0E1114171A1D0020207043
:104C000017E00120207014E00220207011E0032042
:104C100020700EE0042020700BE00520207008E0DA
:104C20000620207005E00720207002E000202070A0
:104C300000BF00BF3046F8BDF8B506460C4601235C
:104C40006A4617213046FEF7F9FC0546002D0ED1C5
:104C50006946087840084000E107C90F0843009002
:104C600001236A4617213046FEF7FBFC054628461D
:104C7000F8BDF8B505460C4601236A4617212846BB
:104C8000FEF7DCFC064668460078C007C00F2070BF
:104C90003046F8BDF8B506460C4601236A46172192
:104CA0003046FEF7CBFC0546002D27D1684600783C
:104CB0000421884310212140090989000422114060
:104CC000014300916846007810218843202121404B
:104CD00049090901102211400143009168460078FA
:104CE000E02188436101E022114008430090012344
:104CF0006A4617213046FEF7B4FC05462846F8BD43
:104D0000F8B505460C4601236A4617212846FEF7EA
:104D100095FC064668460078C006C00F410168460B
:104D200000784007C00F0001084369460978490927
:104D30000843132832D00DDC030010F082F813234F
:104D40005356595C5F626568686868686868682679
:104D5000292C6800322833D00CDC162827D004DC3C
:104D600014281ED0152852D11EE0172822D0312831
:104D70004DD122E03338030010F063F80525282BCD
:104D80002E3149000020207044E01020207041E0C6
:104D9000112020703EE0122020703BE01320207094
:104DA00038E01420207035E01520207032E0162005
:104DB00020702FE0172020702CE03120207029E097
:104DC0003220207026E03320207023E03420207031
:104DD00020E0352020701DE0362020701AE03720BA
:104DE000207017E00120207014E00220207011E0F4
:104DF000032020700EE0042020700BE005202070BE
:104E000008E00620207005E00720207002E0002066
:104E1000207000BF00BF3046F8BDF8B506460C460E
:104E200001236A4617213046FEF708FC0546002D8F
:104E30000FD16946087808218843E1000822114013
:104E40000843009001236A4617213046FEF709FC0B
:104E500005462846F8BDF8B505460C4601236A46C6
:104E600017212846FEF7EAFB064668460078000749
:104E7000C00F20703046F8BDF8B506460C46012339
:104E80006A4656213046FEF7D9FB0546002D0FD164
:104E900069460878102188432101102211400843F7
:104EA000009001236A4656213046FEF7DAFB05469C
:104EB0002846F8BDF8B505460C4601236A4656213A
:104EC0002846FEF7BBFB064668460078C006C00FC2
:104ED000002802D0012806D102E00020207005E061
:104EE0000120207002E00020207000BF00BF30468B
:104EF000F8BDF8B506460C4601236A461621304631
:104F0000FEF79CFB0546002D1BD16846007840212A
:104F1000884380212140C909890140221140014371
:104F200000916846007830218843210130221140E9
:104F30000843009001236A4616213046FEF791FB94
:104F400005462846F8BDF8B505460C4601236A46D5
:104F500016212846FEF772FB064668460078400692
:104F6000C00FC101684600788006800F08188128AC
:104F700010D004DC002807D0802814D107E0822854
:104F80000BD083280FD10BE0002020700EE0802092
:104F900020700BE08120207008E08220207005E066
:104FA0008320207002E00020207000BF00BF304648
:104FB000F8BDF8B506460C4601236A460221304684
:104FC000FEF73CFB0546002D0FD16946087880218D
:104FD0008843E101802211400843009001236A4682
:104FE00002213046FEF73DFB05462846F8BDF8B5E0
:104FF00005460C4601236A4602212846FEF71EFBA1
:10500000064668460078C009002802D0012806D16B
:1050100002E00020207005E00120207002E0002066
:10502000207000BF00BF3046F8BDF8B506460C46FC
:1050300001236A4616213046FEF700FB0546002D87
:1050400017D16846007804218843A100042211404A
:10505000014300916846007840084000E107C90F0D
:105060000843009001236A4616213046FEF7F9FAFC
:1050700005462846F8BDF8B505460C4601236A46A4
:1050800016212846FEF7DAFA064668460078C00779
:10509000C00F002803D0012804D1207005E00020B3
:1050A000207002E00120207000BF00BF3046F8BD34
:1050B000F8B506460C4601236A4617213046FEF72E
:1050C000BDFA0546002D0FD16946087802218843B4
:1050D0006100022211400843009001236A46172113
:1050E0003046FEF7BEFA05462846F8BDF8B5054637
:1050F0000C4601236A4617212846FEF79FFA06460A
:10510000684600788007C00F002802D0012806D129
:1051100002E00020207005E00120207002E0002065
:10512000207000BF00BF3046F8BD70B505460C4684
:10513000012322461E212846FEF780FA0646304605
:1051400070BDF8B505460C4601236A461E21284667
:10515000FEF774FA064668460078C007C00F207054
:105160003046F8BDF8B505460C4601236A461E21B7
:105170002846FEF763FA0646684600788007C00FA7
:1051800020703046F8BDF8B505460C4601236A4646
:105190001E212846FEF752FA064668460078400768
:1051A000C00F20703046F8BDF8B506460C46012306
:1051B0006A466F213046FEF741FA0546002D0ED1B2
:1051C0006946087880088000A107890F084300908D
:1051D00001236A466F213046FEF743FA054628460A
:1051E000F8BDF8B505460C4601236A466F212846EE
:1051F000FEF724FA0646684600788007800F0028EC
:1052000004D0012805D0022809D105E00020207033
:1052100008E00120207005E00220207002E000205C
:10522000207000BF00BF3046F8BDF8B506460C46FA
:1052300001236A466F213046FEF700FA0546002D2D
:105240000FD169460878202188436101202211404E
:105250000843009001236A466F213046FEF701FAA9
:1052600005462846F8BDF8B505460C4601236A46B2
:105270006F212846FEF7E2F9064668460078800668
:10528000C00F002802D0012806D102E000202070C3
:1052900005E00120207002E00020207000BF00BF68
:1052A0003046F8BD7CB506460D4601236A466F219F
:1052B0003046FEF7C3F90446694608784021884322
:1052C000A901402211400843009001236A466F2142
:1052D0003046FEF7C6F90419002C01D020467CBDEB
:1052E000012301AA70213046FEF7A8F90446694659
:1052F0000879402188430221294049088901402238
:10530000114008430190012301AA70213046FEF7A5
:10531000A8F904192046E2E77CB506460C460123AD
:105320006A466F213046FEF789F90546002D01D007
:1053300028467CBD012301AA70213046FEF77EF984
:105340000546002D01D02846F3E76846007940065F
:10535000C00F4100684600784006C00F08180028BA
:1053600004D0022808D0032809D102E000202070D0
:1053700008E00320207005E00220207002E00020F9
:10538000207000BF00BF2846D3E7F8B506460C469C
:1053900001236A466F213046FEF750F90546002D7D
:1053A0000FD16946087880218843E10180221140AD
:1053B0000843009001236A466F213046FEF751F9F9
:1053C00005462846F8BDF8B505460C4601236A4651
:1053D0006F212846FEF732F9064668460078C00974
:1053E00020703046F8BDF8B506460C4601236A46E3
:1053F00070213046FEF722F90546002D1AD1684685
:10540000007841084900E007C00F01430091684659
:105410000078102188430221214049080901102207
:1054200011400843009001236A4670213046FEF780
:1054300018F905462846F8BDF8B505460C4601237F
:105440006A4670212846FEF7F9F80646694608784C
:10545000C006C00F40000978C907C90F08430028DB
:1054600004D0012805D0032809D105E000202070D0
:1054700008E00120207005E00320207002E00020F9
:10548000207000BF00BF3046F8BDF8B506460C4698
:1054900001236A4670213046FEF7D0F80546002DFC
:1054A0000FD1694608780E21884361000E22114011
:1054B0000843009001236A4670213046FEF7D1F878
:1054C00005462846F8BDF8B505460C4601236A4650
:1054D00070212846FEF7B2F80646684600780007B5
:1054E000400F03000FF0ADFC0705080B140E14115C
:1054F0001400002020700EE0012020700BE002203C
:10550000207008E00420207005E00620207002E0F2
:105510000020207000BF00BF3046F8BDF8B5064639
:105520000C4601236A4670213046FEF787F805468F
:10553000002D0FD16946087820218843610120227F
:1055400011400843009001236A4670213046FEF75F
:1055500088F805462846F8BDF8B505460C460123EF
:105560006A4670212846FEF769F8064668460078C4
:105570008006C00F002802D0012806D102E00020DA
:10558000207005E00120207002E00020207000BFA4
:1055900000BF3046F8BDF8B506460C4601236A4602
:1055A00071213046FEF74AF80546002D0FD16946B5
:1055B00008780621884361000622114008430090C4
:1055C00001236A4671213046FEF74BF8054628460E
:1055D000F8BDF8B505460C4601236A4671212846F8
:1055E000FEF72CF80646684600784007800F002832
:1055F00006D0012807D0022808D003280CD108E0E3
:10560000002020700BE00120207008E002202070B4
:1056100005E00320207002E00020207000BF00BFE2
:105620003046F8BDF8B506460C4601236A4671219E
:105630003046FEF703F80546002D18D1684600787D
:1056400030218843210130221140014300916846F6
:1056500000784008400010212140090908430090CB
:1056600001236A4671213046FDF7FBFF05462846B7
:10567000F8BDF8B505460C4601236A467121284657
:10568000FDF7DCFF064669460878C007C00E0978BA
:105690008906890F0843112810D004DC002807D0A0
:1056A000102814D107E012280BD013280FD10BE0DB
:1056B000002020700EE0102020700BE011202070E0
:1056C00008E01220207005E01320207002E0002086
:1056D000207000BF00BF3046F8BDF8B506460C4646
:1056E00001236A4672213046FDF7A8FF0546002DCA
:1056F0000ED16946087840084000E107C90F084309
:10570000009001236A4672213046FDF7AAFF054644
:105710002846F8BDF8B505460C4601236A467221B5
:105720002846FDF78BFF064668460078C007C00F85
:10573000002802D0012806D102E00020207005E0F8
:105740000120207002E00020207000BF00BF304622
:10575000F8BDF8B506460C4601236A46722130466C
:10576000FDF76CFF0546002D0FD16946087806212C
:1057700088436100062211400843009001236A46D5
:1057800072213046FDF76DFF05462846F8BDF8B595
:1057900005460C4601236A4672212846FDF74EFF56
:1057A0000646684600784007800F002804D001288C
:1057B00005D0032809D105E00020207008E0012071
:1057C000207005E00320207002E00020207000BF60
:1057D00000BF3046F8BDF8B506460C4601236A46C0
:1057E00072213046FDF72AFF0546002D0FD169468C
:1057F000087838218843E10038221140084300909E
:1058000001236A4672213046FDF72BFF05462846E4
:10581000F8BDF8B505460C4601236A4672212846B4
:10582000FDF70CFF0646684600788006400F03002F
:105830000FF007FB0805080B0E1114171A1D0020A6
:10584000207017E00120207014E00220207011E089
:10585000032020700EE0042020700BE00520207053
:1058600008E00620207005E00720207002E00020FC
:10587000207000BF00BF3046F8BDF8B506460C46A4
:1058800001236A4672213046FDF7D8FE0546002DF9
:105890000FD169460878C0218843A101C022114078
:1058A0000843009001236A4672213046FDF7D9FE75
:1058B00005462846F8BDF8B505460C4601236A465C
:1058C00072212846FDF7BAFE064668460078800930
:1058D000002806D0012807D0022808D003280CD1C0
:1058E00008E0002020700BE00120207008E002207A
:1058F000207005E00320207002E00020207000BF2F
:1059000000BF3046F8BDF8B506460C4601236A468E
:1059100002213046FDF792FE0546002D0FD1694663
:10592000087840218843A10140221140084300909B
:1059300001236A4602213046FDF793FE05462846BC
:10594000F8BDF8B505460C4601236A4602212846F3
:10595000FDF774FE0646684600784006C00F002832
:1059600002D0012806D102E00020207005E00120CD
:10597000207002E00020207000BF00BF3046F8BD5C
:10598000F8B506460C4601236A4612213046FDF75B
:1059900055FE0546002D0FD1694608780821884339
:1059A000E100082211400843009001236A461221B9
:1059B0003046FDF756FE05462846F8BDF8B50546C3
:1059C0000C4601236A4612212846FDF737FE06469B
:1059D000684600780007C00F002802D0012806D1D1
:1059E00002E00020207005E00120207002E000208D
:1059F000207000BF00BF3046F8BDF8B506460C4623
:105A000001236A4613213046FDF718FE0546002D96
:105A10000FD16946087804218843A100042211406F
:105A20000843009001236A4613213046FDF719FE12
:105A300005462846F8BDF8B505460C4601236A46DA
:105A400013212846FDF7FAFD064668460078400710
:105A5000C00F002802D0012806D102E000202070EB
:105A600005E00120207002E00020207000BF00BF90
:105A70003046F8BD7CB506460D4601236A4618211E
:105A80003046FDF7DBFD044669460878022188436D
:105A900080212940C9094900022211400843009091
:105AA00001236A4618213046FDF7DBFD0419002C5E
:105AB00001D020467CBD012301AA62213046FDF7BA
:105AC000BDFD04466946087918218843E90018227B
:105AD000114008430190012301AA62213046FDF7DD
:105AE000C0FD04192046E5E77CB506460C460123B7
:105AF00001AA18213046FDF7A1FD054601236A469B
:105B000062213046FDF79AFD4519002D01D0284647
:105B10007CBD694608798007C00FC0010978C906B5
:105B2000890F0843022811D004DC002808D001287E
:105B300012D108E003280CD080280DD120700EE08F
:105B4000002020700BE00120207008E0022020706F
:105B500005E00320207002E08020207000BF00BF1D
:105B60002846D5E7F8B506460C4601236A46622169
:105B70003046FDF763FD0546002D0ED169460878D5
:105B800040084000E107C90F0843009001236A461E
:105B900062213046FDF765FD05462846F8BDF8B59B
:105BA00005460C4601236A4662212846FDF746FD5C
:105BB000064668460078C007C00F002802D00128BA
:105BC00006D102E00020207005E00120207002E0F4
:105BD0000020207000BF00BF3046F8BDF8B5064673
:105BE0000C4601236A4612213046FDF727FD054683
:105BF000002D0FD169460878102188432101102219
:105C000011400843009001236A4612213046FDF7F7
:105C100028FD05462846F8BDF8B505460C46012383
:105C20006A4612212846FDF709FD064668460078B7
:105C3000C006C00F002802D0012806D102E00020D3
:105C4000207005E00120207002E00020207000BFDD
:105C500000BF3046F8BDF8B506460C4601236A463B
:105C600012213046FDF7EAFC0546002D0FD16946AA
:105C700008782021884361012022114008430090C8
:105C800001236A4612213046FDF7EBFC0546284603
:105C9000F8BDF8B505460C4601236A461221284690
:105CA000FDF7CCFC0646684600788006C00F002849
:105CB00002D0012806D102E00020207005E001207A
:105CC000207002E00020207000BF00BF3046F8BD09
:105CD000F8B506460C4601236A4613213046FDF707
:105CE000ADFC0546002D0FD1694608782021884378
:105CF0006101202211400843009001236A461321CC
:105D00003046FDF7AEFC05462846F8BDF8B5054619
:105D10000C4601236A4613212846FDF78FFC0646F0
:105D2000684600788006C00F20703046F8BD7CB50C
:105D300006460D46012301AA56213046FDF77EFC9A
:105D400004466846007941084900E807C00F01434E
:105D500001916846007940218843A9014022114001
:105D600008430190012301AA56213046FDF779FC32
:105D70000419002C01D020467CBD02213046FDF7DD
:105D800044FD0446002C01D02046F5E701236A4675
:105D900017213046FDF752FC0446694608788021F9
:105DA0008843022129404908C90180221140084343
:105DB000009001236A4617213046FDF752FC041972
:105DC00000213046FDF721FD04192046D4E77CB5BB
:105DD00006460C46012301AA56213046FDF72EFC4B
:105DE0000546002D01D028467CBD02213046FDF736
:105DF0000CFD054601236A4617213046FDF71EFCBF
:105E00004519002D00D028E069460878C0094000F7
:105E10000979C907C90F0843002806D0012807D00F
:105E2000022808D003280CD108E0002020700BE0E5
:105E30000120207008E00220207005E0032020707F
:105E400002E00020207000BF00BF01236A46172136
:105E50003046FDF7F3FB451900BF00213046FDF742
:105E6000D4FC45192846BFE7F8B506460C46012381
:105E70006A465C213046FDF7E1FB0546002D0FD157
:105E800069460878102188432101102211400843F7
:105E9000009001236A465C213046FDF7E2FB05468F
:105EA0002846F8BDF8B505460C4601236A465C2134
:105EB0002846FDF7C3FB064668460078C006C00FBB
:105EC000002802D0012806D102E00020207005E061
:105ED0000120207002E00020207000BF00BF30468B
:105EE000F8BDF8B506460C4601236A465B213046EC
:105EF000FDF7A4FB0546002D0ED169460878800900
:105F00008001A106890E0843009001236A465B21A7
:105F10003046FDF7A6FB05462846F8BDF8B5054610
:105F20000C4601236A465B212846FDF787FB06469F
:105F3000684600788006800E20703046F8BDF8B5BF
:105F400006460C4601236A465B213046FDF776FB88
:105F50000546002D0FD16946087840218843A101EC
:105F6000402211400843009001236A465B213046DD
:105F7000FDF777FB05462846F8BDF8B505460C4603
:105F800001236A465B212846FDF758FB0646684612
:105F900000784006C00F20703046F8BDF8B50646C0
:105FA0000C4601236A465C213046FDF747FB054657
:105FB000002D0FD169460878602188436101602275
:105FC00011400843009001236A465C213046FDF7EA
:105FD00048FB05462846F8BDF8B505460C460123A2
:105FE0006A465C212846FDF729FB0646684600788C
:105FF0004006800F20703046F8BDF8B506460C46C6
:1060000001236A4613213046FDF718FB0546002D93
:106010000FD16946087840218843A10140221140F0
:106020000843009001236A4613213046FDF719FB0F
:1060300005462846F8BDF8B505460C4601236A46D4
:1060400013212846FDF7FAFA06466846007840060E
:10605000C00F20703046F8BDF8B506460C46012347
:106060006A4656213046FDF7E9FA0546002D0FD164
:1060700069460878202188436101202211400843A5
:10608000009001236A4656213046FDF7EAFA05469C
:106090002846F8BDF8B505460C4601236A46562148
:1060A0002846FDF7CBFA0646684600788006C00F02
:1060B000002802D0012806D102E00020207005E06F
:1060C0000120207002E00020207000BF00BF304699
:1060D000F8BDF8B506460C4601236A4658213046FD
:1060E000FDF7ACFA0546002D0FD16946087860210E
:1060F00088436101602211400843009001236A46F1
:1061000058213046FDF7ADFA05462846F8BDF8B5EA
:1061100005460C4601236A4658212846FDF78EFAAB
:106120000646684600784006800F002806D0012801
:1061300007D0022808D003280CD108E000202070E6
:106140000BE00120207008E00220207005E0032011
:10615000207002E00020207000BF00BF3046F8BD74
:10616000F8B506460C4601236A465C213046FDF729
:1061700065FA0546002D0ED1694608780009000130
:106180002107090F0843009001236A465C2130462D
:10619000FDF767FA05462846F8BDF8B505460C46F2
:1061A00001236A465C212846FDF748FA0646684600
:1061B00000780007000F20703046F8BDF8B506469D
:1061C0000C4601236A4656213046FDF737FA05464C
:1061D000002D0FD169460878022188436100022210
:1061E00011400843009001236A4656213046FDF7CE
:1061F00038FA05462846F8BDF8B505460C46012391
:106200006A4656212846FDF719FA06466846007880
:106210008007C00F20703046F8BDF8B506460C4622
:1062200001236A4656213046FDF708FA0546002D3F
:106230000FD16946087804218843A1000422114047
:106240000843009001236A4656213046FDF709FABB
:1062500005462846F8BDF8B505460C4601236A46B2
:1062600056212846FDF7EAF90646684600784007B9
:10627000C00F20703046F8BDF8B506460C46012325
:106280006A4656213046FDF7D9F90546002D0FD153
:106290006946087808218843E10008221140084334
:1062A000009001236A4656213046FDF7DAF905468B
:1062B0002846F8BDF8B505460C4601236A46562126
:1062C0002846FDF7BBF90646684600780007C00F70
:1062D00020703046F8BDF8B506460C4601236A46E4
:1062E00057213046FDF7AAF90546002D0ED1694623
:1062F000087840094001E106C90E084300900123D7
:106300006A4657213046FDF7ACF905462846F8BDE8
:10631000F8B505460C4601236A4657212846FDF785
:106320008DF9064668460078C006C00E20703046DB
:10633000F8BDF8B506460C4601236A46572130469B
:10634000FDF77CF90546002D0FD169460878E0215C
:1063500088436101E02211400843009001236A460E
:1063600057213046FDF77DF905462846F8BDF8B5BA
:1063700005460C4601236A4657212846FDF75EF97B
:10638000064668460078400903000EF05AFD0705EE
:10639000080B0E17111417000020207011E00120C7
:1063A00020700EE0022020700BE00320207008E037
:1063B0000520207005E00620207002E000202070FB
:1063C00000BF00BF3046F8BDF8B506460C460123B5
:1063D0006A4658213046FDF731F90546002D0ED1A9
:1063E0006946087840094001E106C90E084300905B
:1063F00001236A4658213046FDF733F90546284601
:10640000F8BDF8B505460C4601236A4658212846D2
:10641000FDF714F9064668460078C006C00E2070E5
:106420003046F8BDF8B506460C4601236A465921A8
:106430003046FDF703F90546002D0ED16946087870
:1064400040094001E106C90E0843009001236A4655
:1064500059213046FDF705F905462846F8BDF8B53F
:1064600005460C4601236A4659212846FDF7E6F801
:10647000064668460078C006C00E20703046F8BD5B
:10648000F8B506460C4601236A465A213046FDF708
:10649000D5F80546002D0ED16946087880088000A1
:1064A000A107890F0843009001236A465A2130460C
:1064B000FDF7D7F805462846F8BDF8B505460C4661
:1064C00001236A465A212846FDF7B8F80646684671
:1064D00000788007800F20703046F8BDF8B506467A
:1064E0000C4601236A465A213046FDF7A7F80546B7
:1064F000002D0FD1694608780C218843A1000C2299
:1065000011400843009001236A465A213046FDF7A6
:10651000A8F805462846F8BDF8B505460C460123FF
:106520006A465A212846FDF789F8064668460078EB
:106530000007800F20703046F8BDF8B506460C46BF
:1065400001236A465A213046FDF778F80546002DAA
:106550000FD169460878F02188432101F0221140CB
:106560000843009001236A465A213046FDF779F826
:1065700005462846F8BDF8B505460C4601236A468F
:106580005A212846FDF75AF8064668460078000961
:1065900020703046F8BDF8B506460C4601236A4621
:1065A0005B213046FDF74AF80546002D0FD16946BC
:1065B000087880218843E10180221140084300903F
:1065C00001236A465B213046FDF74BF80546284615
:1065D000F8BDF8B505460C4601236A465B212846FE
:1065E000FDF72CF8064668460078C009002802D05E
:1065F000012806D102E00020207005E00120207073
:1066000002E00020207000BF00BF3046F8BDF8B5A2
:1066100006460C4601236A4659213046FDF70EF81E
:106620000546002D0FD16946087860218843610135
:10663000602211400843009001236A4659213046E8
:10664000FDF70FF805462846F8BDF8B505460C4697
:1066500001236A4659212846FCF7F0FF06466846A2
:1066600000784006800F002806D0012807D00228B5
:1066700008D003280CD108E0002020700BE0012096
:10668000207008E00220207005E00320207002E066
:106690000020207000BF00BF3046F8BDF8B50646A8
:1066A0000C4601236A4659213046FCF7C7FF0546D0
:1066B000002D0FD16946087880218843E1018022AE
:1066C00011400843009001236A4659213046FCF7E7
:1066D000C8FF05462846F8BDF8B505460C46012317
:1066E0006A4659212846FCF7A9FF06466846007805
:1066F000C00920703046F8BDF8B506460C460123A7
:106700006A465D213046FCF799FF0546002D0ED103
:1067100069460878C008C0006107490F0843009027
:1067200001236A465D213046FCF79BFF054628465B
:10673000F8BDF8B505460C4601236A465D2128469A
:10674000FCF77CFF0646684600784007400F0300D0
:106750000EF077FB0805080B0E1114171A1D002008
:10676000207017E00120207014E00220207011E05A
:10677000032020700EE0042020700BE00520207024
:1067800008E00620207005E00720207002E00020CD
:10679000207000BF00BF3046F8BD7CB506460D46F0
:1067A000012301AA5C213046FCF748FF044601237F
:1067B0006A465D213046FCF741FF0419002C01D0E8
:1067C00020467CBD684600798021884320212940ED
:1067D0004909C901802211400143019168460078AE
:1067E000F8218843E900F822114008430090012372
:1067F00001AA5C213046FCF734FF044601236A46B7
:106800005D213046FCF72DFF04192046D9E77CB501
:1068100006460C46012301AA5C213046FCF70EFF18
:106820000546002D0FD101236A465D213046FCF755
:1068300005FF054668460079C009410168460078B1
:10684000C0080818207028467CBD7CB506460C465A
:1068500001236A4608213046FCF7F0FE0546002D6C
:1068600001D028467CBDE1B201916846007840081D
:106870004000FF2101312140090A08430090012313
:1068800001AA07213046FCF7ECFE054601236A46C3
:1068900008213046FCF7E5FE45192846E2E77CB5BD
:1068A00006460C46012301AA07213046FCF7C6FE26
:1068B0000546002D0ED101236A4608213046FCF71B
:1068C000BDFE054668460078C007C10D68460079E0
:1068D0000818208028467CBDF8B506460D460221E2
:1068E0003046FCF792FF0446002C01D02046F8BD4C
:1068F00001236A4667213046FCF7A0FE044669463C
:10690000087808218843E9000822114008430090D4
:1069100001236A4667213046FCF7A3FE04190021D3
:106920003046FCF772FF04192046E0E7F8B506464A
:106930000D4602213046FCF768FF044601236A46F3
:1069400067213046FCF77AFE041900213046FCF737
:106950005CFF0419684600780007C00F28702046C5
:10696000F8BDF8B506460C4601236A4608213046B4
:10697000FCF764FE0546002D1BD1684600784021D7
:1069800088430421214089088901402211400143A4
:106990000091684600780621884361000622114074
:1069A0000843009001236A4608213046FCF759FE4F
:1069B00005462846F8BDF8B505460C4601236A464B
:1069C00008212846FCF73AFE064669460878400644
:1069D000C00F800009784907890F084303000EF0B3
:1069E00030FA0805141414080B0E1114002020703E
:1069F0000EE0042020700BE00520207008E0062047
:106A0000207005E00720207002E00020207000BF09
:106A100000BF3046F8BDF8B506460C4601236A466D
:106A200008213046FCF70AFE0546002D0FD16946C5
:106A3000087810218843210110221140084300905A
:106A400001236A4608213046FCF70BFE054628461E
:106A5000F8BDF8B505460C4601236A4608212846CC
:106A6000FCF7ECFD064668460078C006C00F2070B3
:106A70003046F8BDF8B506460C4601236A460821A3
:106A80003046FCF7DBFD0546002D0FD1694608783E
:106A900040218843A1014022114008430090012376
:106AA0006A4608213046FCF7DCFD05462846F8BD5D
:106AB000F8B505460C4601236A4608212846FCF72E
:106AC000BDFD0646684600784006C00F207030467F
:106AD000F8BDF8B506460C4601236A460821304643
:106AE000FCF7ACFD0546002D0FD1694608788021E2
:106AF0008843E101802211400843009001236A4647
:106B000008213046FCF7ADFD05462846F8BDF8B52E
:106B100005460C4601236A4608212846FCF78EFDEF
:106B2000064668460078C00920703046F8BDF8B5C2
:106B300006460C4601236A4609213046FCF77EFDD5
:106B40000546002D0ED1694608780009000121078D
:106B5000090F0843009001236A4609213046FCF7DB
:106B600080FD05462846F8BDF8B505460C460123CC
:106B70006A4609212846FCF761FD0646684600780A
:106B80000007000F03000EF05CF90C070A0D10134C
:106B900016191C1F2225282B0020207023E001201D
:106BA000207020E0022020701DE0032020701AE0F9
:106BB0000420207017E00520207014E006202070CB
:106BC00011E0072020700EE0082020700BE0092063
:106BD000207008E00A20207005E00B20207002E001
:106BE0000020207000BF00BF3046F8BDF8B5064653
:106BF0000C4601236A4609213046FCF71FFD054675
:106C0000002D0FD169460878F02188432101F02238
:106C100011400843009001236A4609213046FCF7E1
:106C200020FD05462846F8BDF8B505460C4601236B
:106C30006A4609212846FCF701FD064668460078A9
:106C4000000903000EF0FDF80C070A0D10131619C9
:106C50001C1F2225282B0020207023E001202070FB
:106C600020E0022020701DE0032020701AE00420A4
:106C7000207017E00520207014E00620207011E03D
:106C8000072020700EE0082020700BE00920207003
:106C900008E00A20207005E00B20207002E00020B0
:106CA000207000BF00BF3046F8BDF8B506460C4660
:106CB00001236A460A213046FCF7C0FC0546002D38
:106CC0000ED169460878C008C0006107490F084323
:106CD000009001236A460A213046FCF7C2FC0546B3
:106CE0002846F8BDF8B505460C4601236A460A2138
:106CF0002846FCF7A3FC0646684600784007400F8C
:106D000003000EF09EF8080508170B0E1711141754
:106D10000020207011E0012020700EE00320207080
:106D20000BE00420207008E00620207005E007201A
:106D3000207002E00020207000BF00BF3046F8BD88
:106D4000F8B506460C4601236A460A213046FCF790
:106D500075FC0546002D0FD169460878302188431F
:106D60002101302211400843009001236A460A2184
:106D70003046FCF776FC05462846F8BDF8B50546D2
:106D80000C4601236A460A212846FCF757FC0646B2
:106D9000684600788006800F002806D0012807D0BA
:106DA000022808D003280CD108E0002020700BE056
:106DB0000120207008E00220207005E003202070F0
:106DC00002E00020207000BF00BF3046F8BDF8B5DB
:106DD00006460C4601236A460A213046FCF72EFC83
:106DE0000546002D0FD169460878C0218843A101CE
:106DF000C02211400843009001236A460A21304610
:106E0000FCF72FFC05462846F8BDF8B505460C46AC
:106E100001236A460A212846FCF710FC064668460C
:106E200000788009002806D0012807D0022808D061
:106E300003280CD108E0002020700BE00120207016
:106E400008E00220207005E00320207002E000200E
:106E5000207000BF00BF3046F8BDF8B506460C46AE
:106E600001236A460B213046FCF7E8FB0546002D5E
:106E70000FD1694608782021884361012022114002
:106E80000843009001236A460B213046FCF7E9FBDA
:106E900005462846F8BDF8B505460C4601236A4666
:106EA0000B212846FCF7CAFB064668460078800698
:106EB000C00F002802D0012806D102E00020207077
:106EC00005E00120207002E00020207000BF00BF1C
:106ED0003046F8BDF8B506460C4601236A460B213C
:106EE0003046FCF7ABFB0546002D0FD1694608780C
:106EF00040218843A1014022114008430090012312
:106F00006A460B213046FCF7ACFB05462846F8BD27
:106F1000F8B505460C4601236A460B212846FCF7C6
:106F20008DFB0646684600784006C00F207030464C
:106F3000F8BD7CB506460D46012301AA0B2130465B
:106F4000FCF77CFB0446002C01D020467CBDE9B256
:106F5000009168460079C008C00007210902294055
:106F6000C9B2091208430190012301AA0B2130463E
:106F7000FCF777FB041901236A460C213046FCF725
:106F800070FB04192046E1E77CB506460C46012358
:106F900001AA0B213046FCF751FB0546002D0ED10E
:106FA00001236A460C213046FCF748FB054668463B
:106FB00000794007410D684600780818208028466F
:106FC0007CBDF3B581B00C466E46771C02236A4641
:106FD0003A210198FCF732FB0546002D08D138789C
:106FE0008007800F208020780002317840182080B0
:106FF0002846FEBDF8B506460C4600AF0137022311
:107000006A463A213046FCF719FB0546002D01D1AE
:10701000387820702846F8BDF8B506460C4600AF13
:10702000013702236A463A213046FCF707FB054642
:10703000002D03D138788006C00F20702846F8BD97
:10704000F8B506460C4600AF013702236A463A21DE
:107050003046FCF7F3FA0546002D03D13878400698
:10706000C00F20702846F8BDF8B506460C4600AFA4
:10707000013702236A463A213046FCF7DFFA05461B
:10708000002D02D13878C00920702846F8BDF8B527
:1070900005460C4601236A4678212846FCF7CEFABD
:1070A000064668460078C00803000DF0CAFE1A5074
:1070B0000E1114171A1D202326292C2F3235383B88
:1070C0003E4144474A5050504D500120207041E00D
:1070D000022020703EE0032020703BE0042020705E
:1070E00038E00520207035E00620207032E00720CF
:1070F00020702FE0082020702CE00920207029E06B
:107100000A20207026E00B20207023E00C20207045
:1071100020E00D2020701DE00E2020701AE00F20CE
:10712000207017E01020207014E01120207011E072
:10713000122020700EE0132020700BE0142020702D
:1071400008E01520207005E01920207002E00120E1
:10715000207000BF00BF3046F8BDF8B506460D46AA
:1071600002213046FCF751FB0446002C01D020469A
:10717000F8BD01236A4644213046FCF75FFA044615
:107180006946087840218843A901402211400843FC
:10719000009001236A4644213046FCF762FA041944
:1071A00000213046FCF731FB04192046E0E7F8B532
:1071B00006460D4602213046FCF727FB0446002C0C
:1071C00001D02046F8BD01236A4644213046FCF731
:1071D00035FA0446684600784006C00F2870002142
:1071E0003046FCF712FB04192046EBE7F8B50746DA
:1071F0000D46164601213846FCF707FB0446002CD5
:1072000001D02046F8BD680028181730C1B201230C
:107210006A463846FCF712FA04466946087808219F
:107220008843F100082211400843009068002818A4
:107230001730C1B201236A463846FCF712FA041926
:1072400000213846FCF7E1FA04192046DAE7F8B5E0
:1072500007460D46164601213846FCF7D6FA044685
:10726000002C01D02046F8BD680028181730C1B2A4
:1072700001236A463846FCF7E1F90446684600787F
:107280000007C00F307000213846FCF7BEFA041921
:107290002046E8E7F8B506460C4601236A46152164
:1072A0003046FCF7CBF90546002D0FD1694608782A
:1072B000E02188436101E02211400843009001234E
:1072C0006A4615213046FCF7CCF905462846F8BD3C
:1072D000F8B505460C4601236A4615212846FCF7F9
:1072E000ADF9064668460078400903000DF0A9FD97
:1072F0000705140E0B1114081400002020700EE076
:10730000062020700BE00320207008E0022020708F
:1073100005E00420207002E00020207000BF00BFC4
:107320003046F8BDF8B506460C4601236A461821DA
:107330003046FCF783F90546002D0FD169460878E1
:1073400004218843A1000422114008430090012336
:107350006A4618213046FCF784F905462846F8BDF0
:10736000F8B505460C4601236A4618212846FCF765
:1073700065F90646684600784007C00F002802D02D
:10738000012806D102E00020207005E001202070D5
:1073900002E00020207000BF00BF3046F8BDF8B505
:1073A00006460C4601236A4618213046FCF746F98A
:1073B0000546002D0FD16946087818218843E10061
:1073C000182211400843009001236A4618213046D4
:1073D000FCF747F905462846F8BDF8B505460C46C2
:1073E00001236A4618212846FCF728F90646684614
:1073F0000078C006800F002804D0012805D002289C
:1074000009D105E00020207008E00120207005E08F
:107410000220207002E00020207000BF00BF304634
:10742000F8BDF8B506460C4601236A4618213046D9
:10743000FCF704F90546002D0FD169460878202194
:1074400088436101202211400843009001236A46CD
:1074500018213046FCF705F905462846F8BDF8B571
:1074600005460C4601236A4618212846FCF7E6F833
:107470000646684600788006C00F20703046F8BD8A
:10748000F8B506460C4601236A4618213046FCF73B
:10749000D5F80546002D0FD169460878402188436C
:1074A000A101402211400843009001236A4618219F
:1074B0003046FCF7D6F805462846F8BDF8B505462F
:1074C0000C4601236A4618212846FCF7B7F8064601
:1074D000684600784006C00F20703046F8BDF8B509
:1074E00006460C4601236A4618213046FCF7A6F8EA
:1074F0000546002D0FD16946087880218843E101B7
:10750000802211400843009001236A46182130462A
:10751000FCF7A7F805462846F8BDF8B505460C4621
:1075200001236A4618212846FCF788F80646684673
:107530000078C00920703046F8BDF8B506460C4604
:107540006A46FF2184313046FDF737F90546002DA4
:107550001BD1684600780421884310212140090985
:1075600089000422114001430091684600784008D8
:107570004000202121404909084300906A46FF212C
:1075800084313046FDF747F805462846F8BDF8B582
:1075900005460C466A46FF2184312846FDF70DF961
:1075A000064669460878C007800E09784907C90F62
:1075B00009010843002804D0102805D0302809D13B
:1075C00005E00020207008E01020207005E0302049
:1075D000207002E00020207000BF00BF3046F8BDE0
:1075E000F8B506460D4602213046FCF70EF9044672
:1075F000002C01D02046F8BD01236A4612213046F6
:10760000FCF71CF80446684600780007C00F287095
:1076100000213046FCF7F9F804192046EBE770B575
:1076200005460C462246FF2185312846FCF7F3FF2C
:107630000646304670BD70B505460C462246FF2111
:1076400085312846FDF7B9F80646304670BDF8B5D5
:1076500006460C462004010E684641704078000240
:10766000201AC1B2684601706A46FF21D131304606
:10767000FCF7D1FF054600AA0132FF21D231304686
:10768000FCF7C9FF45192846F8BDF8B506460C4673
:107690006A46FF21D1313046FDF78FF8054600AA32
:1076A0000132FF21D2313046FDF787F8451968468F
:1076B00040782080207801026846007808182080F1
:1076C0002846F8BDF8B506460C466A46FF218431C7
:1076D0003046FDF772F80546002D0FD1694608784F
:1076E00008218843E10008221140084300906A46BF
:1076F000FF2184313046FCF78EFF05462846F8BD51
:10770000F8B505460C466A46FF2184312846FDF748
:1077100054F80646684600780007C00F002802D0DB
:10772000012806D102E00020207005E00120207031
:1077300002E00020207000BF00BF3046F8BDF8B561
:1077400006460D4602213046FCF75FF80446002C41
:1077500001D02046F8BD01236A4612213046FBF7CE
:107760006DFF0446684600788006C00F287000212F
:107770003046FCF74AF804192046EBE7F8B5064610
:107780000D4602213046FCF740F80446002C01D09B
:107790002046F8BD01236A4612213046FBF74EFF12
:1077A000044668460078C006C00F287000213046A5
:1077B000FCF72BF804192046EBE7F8B506460C4613
:1077C0002004010E6846417040780002201AC1B2C0
:1077D000684601706A46BA213046FCF71CFF054630
:1077E00000AA0132BB213046FCF715FF4519284697
:1077F000F8BDF8B506460C466A46BA213046FCF795
:10780000DCFF054600AA0132BB213046FCF7D5FF5C
:107810004519684640782080207801026846007843
:10782000081820802846F8BD7CB505460C462088FF
:107830000004010E68464170217840780002081A61
:10784000C1B26846017060880004010E6846C170CC
:10785000A178C0780002081AC1B268468170A08879
:107860000004010E68464171217940790002081A2E
:10787000C1B26846017106236A46C0212846FCF75A
:1078800003FE7CBD7CB505460C4606236A46C02136
:107890002846FCF7CBFE06466846407820802078D4
:1078A000010268460078081800B220806846C07857
:1078B0006080A078010268468078081800B2608075
:1078C00068464079A080207901026846007908184E
:1078D00000B2A08030467CBD3EB505460C462088EF
:1078E0000004010E68464170217840780002081AB1
:1078F000C1B26846017060880004010E6846C1701C
:10790000A178C0780002081AC1B268468170A088C8
:107910000004010E68464171217940790002081A7D
:10792000C1B268460171E0880004010E6846C17169
:10793000A179C0790002081AC1B268468171208914
:107940000004010E68464172217A407A0002081A4A
:10795000C1B26846017260890004010E6846C172B6
:10796000A17AC07A0002081AC1B2684681720C235B
:107970006A46C6212846FCF787FD3EBDFEB5054692
:107980000C460C236A46C6212846FCF74FFE0646E5
:107990006846407820802078010268460078081800
:1079A00000B220806846C0786080A07801026846F6
:1079B0008078081800B2608068464079A0802079FD
:1079C000010268460079081800B2A0806846C079B4
:1079D000E080A079010268468079081800B2E08052
:1079E0006846407A2081207A01026846007A0818A9
:1079F00000B220816846C07A6081A07A01026846A0
:107A0000807A081800B260813046FEBDF8B506469F
:107A10000C466A46D4213046FCF7CFFE0546002DC1
:107A20000DD169460878C008C0006107490F0843B6
:107A300000906A46D4213046FCF7EDFD0546284605
:107A4000F8BDF8B505460C466A46D4212846FCF731
:107A5000B4FE0646684600784007400F03000DF06C
:107A6000F0F90604070A0D1013160020207011E02B
:107A7000012020700EE0022020700BE00320207017
:107A800008E00420207005E00520207002E00020BE
:107A9000207000BF00BF3046F8BDF8B506460C4662
:107AA0006A46D4213046FCF788FE0546002D0ED1EB
:107AB00069460878702188432101702211400843EB
:107AC00000906A46D4213046FCF7A5FD05462846BD
:107AD000F8BDF8B505460C466A46D4212846FCF7A1
:107AE0006CFE0646684600784006400F03000DF025
:107AF000A8F90604070A0D1013160020207011E0E3
:107B0000012020700EE0022020700BE00320207086
:107B100008E00420207005E00520207002E000202D
:107B2000207000BF00BF3046F8BDF8B506460C46D1
:107B30006A46D5213046FCF740FE0546002D0DD1A2
:107B400069460878C008C0006107490F08430090E3
:107B50006A46D5213046FCF75EFD05462846F8BD4D
:107B6000F8B505460C466A46D5212846FCF725FEA1
:107B70000646684600784007400F03000DF061F9A3
:107B80000604070A0D1013160020207011E00120D2
:107B900020700EE0022020700BE00320207008E02F
:107BA0000420207005E00520207002E000202070F5
:107BB00000BF00BF3046F8BDF8B506460D460221AD
:107BC0003046FBF722FE0446002C01D02046F8BDCB
:107BD00001236A4612213046FBF730FD0446684611
:107BE0000078C009287000213046FBF70EFE04190A
:107BF0002046ECE770B506460D4602213046FBF7FD
:107C000004FE0446002C01D0204670BD01232A4604
:107C100046213046FBF725FD044601236A1C472117
:107C20003046FBF71EFD041900213046FBF7EDFD41
:107C300004192046E9E7F8B506460C462004010E73
:107C40006846417040780002201AC1B2684601704F
:107C500002213046FBF7D9FD054602236A4648213A
:107C60003046FBF7FEFC451900213046FBF7CDFD01
:107C700045192846F8BDF8B506460C46022130469F
:107C8000FBF7C3FD054602236A4648213046FBF751
:107C9000D5FC451900213046FBF7B7FD451968466C
:107CA00040782080207801026846007808182080FB
:107CB0002846F8BDF8B506460D4602213046FBF7CA
:107CC000A4FD0446002C01D02046F8BD01236A46DD
:107CD0004A213046FBF7B2FC044669460878800822
:107CE0008000A907890F0843009001236A464A21B2
:107CF0003046FBF7B6FC041900213046FBF785FD42
:107D000004192046E1E7F8B506460C460221304644
:107D1000FBF77BFD0546002D01D02846F8BD012369
:107D20006A464A213046FBF789FC0546002D00D003
:107D300018E0684600788007800F002804D00128EA
:107D400005D0022809D105E00020207008E00120BC
:107D5000207005E00220207002E00020207000BFAB
:107D600000BF00BF00213046FBF74FFD45192846F4
:107D7000D4E770B506460D4602213046FBF745FDB7
:107D8000044610232A464C213046FBF757FC0419C1
:107D900000213046FBF739FD0419204670BDF8B5C7
:107DA00006460D4602213046FBF72FFD0446002C07
:107DB00001D02046F8BD01236A465F213046FBF71B
:107DC0003DFC0446002C00D01DE068460078C10848
:107DD000C900C91C009168460078E021884301462B
:107DE000403100916846007818218843E900182244
:107DF00011400843009001236A465F213046FBF79B
:107E000030FC044600BF00213046FBF7FEFC04199D
:107E10002046CFE7F8B506460D4602213046FBF76F
:107E2000F4FC0446002C01D02046F8BD01236A462C
:107E300067213046FBF702FC0446002C00D00FE01F
:107E40006946087840084000E907C90F08430090D8
:107E500001236A4667213046FBF703FC044600BF56
:107E600000213046FBF7D1FC04192046DDE7F8B5C8
:107E700006460D4602213046FBF7C7FC0446002C9F
:107E800001D02046F8BD01236A4667213046FBF742
:107E9000D5FB044668460078C007C00F2870002153
:107EA0003046FBF7B2FC04192046EBE7F8B506466E
:107EB0000C462004010E6846417040780002201AEA
:107EC000C1B2684601706A46FF217B313046FCF73B
:107ED000A2FB054600AA0132FF217C313046FCF7A7
:107EE0009AFB45192846F8BDF8B506460C466A4681
:107EF000FF217B313046FCF760FC054600AA0132C9
:107F0000FF217C313046FCF758FC45196846407823
:107F100020802078010268460078081820802846D2
:107F2000F8BD73B5044601AAFF217D312046FCF758
:107F300072FB054628467CBD70B505460C462246B8
:107F4000FF217D312846FCF738FC0646304670BDDF
:107F5000F8B506460C462004010E6846417040788C
:107F60000002201AC1B2684601706A46FF217F31C3
:107F70003046FCF750FB054600AA0132FF21803154
:107F80003046FCF748FB45192846F8BDF8B50646CB
:107F90000C466A46FF217F313046FCF70EFC054651
:107FA00000AA0132FF2180313046FCF706FC45195A
:107FB00068464078208020780102684600780818DA
:107FC00020802846F8BDF8B507460D461646012123
:107FD0003846FBF71AFC044633462A460221384647
:107FE000FBF72CFB041900213846FBF70EFC0419A3
:107FF0002046F8BDF8B506460D4601213046FBF790
:1080000004FC0446002C01D02046F8BD01236A463A
:1080100014213046FBF712FB0446694608788008B5
:108020008000A907890F0843009001236A461421A4
:108030003046FBF716FB041900213046FBF7E5FB41
:1080400004192046E1E7F8B506460C460121304602
:10805000FBF7DBFB0546002D01D02846F8BD0123C8
:108060006A4614213046FBF7E9FA0546684600786F
:108070008007800F002806D0012807D0022808D0EA
:1080800003280CD108E0002020700BE001202070B4
:1080900008E00220207005E00320207002E00020AC
:1080A000207000BF00BF00213046FBF7AEFB451932
:1080B0002846D3E7F8B506460D4601213046FBF7C2
:1080C000A4FB0446002C01D02046F8BD01236A46DB
:1080D00014213046FBF7B2FA0446694608780421B9
:1080E0008843A900042211400843009001236A46F6
:1080F00014213046FBF7B5FA041900213046FBF78E
:1081000084FB04192046E0E7F8B506460D46012138
:108110003046FBF77AFB0446002C01D02046F8BD20
:1081200001236A4614213046FBF788FA0446684664
:1081300000784007C00F287000213046FBF765FB30
:1081400004192046EBE7F8B506460D4601213046F6
:10815000FBF75BFB0446002C01D02046F8BD012351
:108160006A4614213046FBF769FA044669460878E6
:1081700008218843E90008221140084300900123A8
:108180006A4614213046FBF76CFA04190021304688
:10819000FBF73BFB04192046E0E7F8B506460C4622
:1081A00001213046FBF731FB0546002D01D0284662
:1081B000F8BD01236A4614213046FBF73FFA054615
:1081C000684600780007C00F002802D0012806D1B9
:1081D00002E00020207005E00120207002E0002075
:1081E000207000BF00BF00213046FBF70EFB451991
:1081F0002846DDE7F8B506460D4601213046FBF777
:1082000004FB0446002C01D02046F8BD01236A4639
:1082100014213046FBF712FA04466946087810210B
:1082200088432901102211400843009001236A4627
:1082300014213046FBF715FA041900213046FBF7EC
:10824000E4FA04192046E0E7F8B506460D46012198
:108250003046FBF7DAFA0446002C01D02046F8BD80
:1082600001236A4614213046FBF7E8F904466846C4
:108270000078C006C00F287000213046FBF7C5FA11
:1082800004192046EBE7F8B506460D4601213046B5
:10829000FBF7BBFA0446002C01D02046F8BD0123B1
:1082A0006A4614213046FBF7C9F904466946087846
:1082B00020218843690120221140084300900123B6
:1082C0006A4614213046FBF7CCF9041900213046E8
:1082D000FBF79BFA04192046E0E7F8B506460C4682
:1082E00001213046FBF791FA0546002D01D02846C2
:1082F000F8BD01236A4614213046FBF79FF9054675
:10830000684600788006C00F002803D0012804D1F9
:10831000207005E00020207002E00120207000BFE6
:1083200000BF00213046FBF770FA45192846DFE709
:10833000F8B506460D4601213046FBF766FA0446BD
:10834000002C01D02046F8BD01236A461421304696
:10835000FBF774F904466946087840218843A9016F
:10836000402211400843009001236A461421304600
:10837000FBF777F9041900213046FBF746FA041998
:108380002046E0E7F8B506460C4601213046FBF7EB
:108390003CFA0546002D01D02846F8BD01236A4667
:1083A00014213046FBF74AF9054668460078400636
:1083B000C00F002802D0012806D102E00020207062
:1083C00005E00120207002E00020207000BF00BF07
:1083D00000213046FBF719FA45192846DDE738B584
:1083E000054601212846FBF710FA0446002C01D06F
:1083F000204638BD01236A4614212846FBF71EF9A2
:108400000446694608788021884380300090012323
:108410006A4614212846FBF724F90419002C01D0E0
:108420002046E6E7694608788021884300900123CA
:108430006A4614212846FBF714F904460021284611
:10844000FBF7E3F904192046D3E7F8B506460D46D5
:1084500001213046FBF7D9F90446002C01D0204613
:10846000F8BD01236A4614213046FBF7E7F80446BD
:1084700068460078C009287000213046FBF7C5F92E
:1084800004192046ECE7F8B506460D4601213046B2
:10849000FBF7BBF90446002C01D02046F8BD0123B0
:1084A0006A4617213046FBF7C9F804466946087842
:1084B000C0218843A901C022114008430090012334
:1084C0006A4617213046FBF7CCF8041900213046E4
:1084D000FBF79BF904192046E0E7F8B506460C4681
:1084E00001213046FBF791F90546002D01D02846C1
:1084F000F8BD01236A4617213046FBF79FF8054671
:10850000684600788009002806D0012807D0022894
:1085100008D003280CD108E0002020700BE00120D7
:10852000207008E00220207005E00320207002E0A7
:108530000020207000BF00BF00213046FBF765F926
:1085400045192846D4E7F8B506460D4601213046C0
:10855000FBF75BF90446002C01D02046F8BD6846C5
:108560000078FE21884329784900FE22114001430A
:1085700000916846007840084000009001236A4658
:1085800015213046FBF76DF80446002C00D011E0B1
:1085900001236A1C16213046FBF763F80446002CC1
:1085A00000D007E00123AA1C21213046FBF759F82F
:1085B000044600BF00213046FBF727F90419204686
:1085C000CCE7FEB507460D46164601213846FBF7B7
:1085D0001CF90446002C01D02046FEBD68460079F7
:1085E000FE21884331784900FE2211400143019168
:1085F0006846007940084000401C01906800281837
:108600001530C1B2012301AA3846FBF72AF8044607
:10861000002C00D02AE0680028181630C1B20123CF
:10862000721C3846FBF71DF80446002C00D01DE0F4
:10863000680028181730C1B201236A463846FAF795
:10864000FDFF044669460878C008C000B1784907B4
:10865000490F08430090680028181730C1B2012361
:108660006A463846FAF7FDFF041900BF0021384674
:10867000FBF7CBF804192046AFE770B505460C466A
:108680000123224639212846FAF7D8FF064630460C
:1086900070BDF8B505460C4616460027002D06D0DD
:1086A000012332460F212846FAF7C8FF0746002C5F
:1086B00006D00123721C0F212046FAF7BFFFC7190D
:1086C0003846F8BDFEB506460C4602213046FBF79B
:1086D0009CF80546002D01D02846FEBD012301AAC5
:1086E00067213046FAF7AAFF054668460079082157
:1086F0008843E10008221140014301916846007956
:1087000041084900E007C00F01430191012301AA7C
:1087100067213046FAF7A5FF4519012302AA662111
:108720003046FAF78BFF45196846007A08218843DE
:10873000202121404911C900082211400143029122
:108740006846007A1021884340212140891109019F
:1087500010221140014302916846007A202188438B
:1087600080212140C9114901202211400843029073
:10877000012302AA66213046FAF773FF451900214A
:108780003046FBF742F84519002D01D02846A4E7F2
:1087900001236A4612213046FAF750FF0546012CA4
:1087A00001D0022C1AD1002D18D168460078802102
:1087B0008843E1018022114001430091684600781E
:1087C0004008400002212140491008430090012345
:1087D0006A4612213046FAF744FF0546002C20D1A4
:1087E000684600784006C00F002805D0684600782B
:1087F0004007C00F002814D1002D12D16846007820
:10880000402188434118009168460078042188433C
:10881000001D009001236A4612213046FAF721FF1D
:108820000546284659E7F7B586B007460E460025A7
:10883000002E23D0012305AA70213046FAF7FEFE50
:10884000054608A84078042108408408002D15D169
:108850006846007D8006C00FA0420FD06946087DA3
:108860002021884361012022114008430590012303
:1088700005AA70213046FAF7F4FE0546002F7DD098
:10888000002D06D1012303AA18213846FAF7D6FE97
:10889000054608A80078042108408408002D15D159
:1088A0006846007B8007C00FA0420FD06946087B56
:1088B00002218843610002221140084303900123F2
:1088C00003AA18213846FAF7CCFE0546002D06D13A
:1088D000012304AA62213846FAF7B0FE054608A82B
:1088E0000078302108400409002D15D16846007C2D
:1088F000C006800FA0420FD06946087C182188432B
:10890000E1001822114008430490012304AA6221C7
:108910003846FAF7A6FE0546002D06D1012301AA26
:1089200013213846FAF78AFE054608A80078022186
:1089300008404408002D15D1684600794007C00F53
:10894000A0420FD06946087904218843A10004227F
:10895000114008430190012301AA13213846FAF778
:1089600080FE0546002D06D1012302AA12213846B9
:10897000FAF764FE054608A8007800E019E0C4078D
:10898000E40F002D15D16846007A0007C00FA04201
:108990000FD06946087A08218843E1000822114077
:1089A00008430290012302AA12213846FAF759FE21
:1089B0000546284609B0F0BDF0B585B007460E461D
:1089C00014460025002E19D0012304AA7021304638
:1089D000FAF734FE05466846007C8006C00F002882
:1089E00002D0012806D102E00020607005E00120DD
:1089F000607002E00020607000BF00BF002F68D0F0
:108A0000002D06D1012302AA18213846FAF716FED6
:108A10000546002D06D1012303AA62213846FAF744
:108A20000DFE0546002D06D101236A461321384666
:108A3000FAF704FE0546002D4BD1012301AA1221AD
:108A40003846FAF7FBFD05466846007BC006800FF6
:108A500001016846007A8007C00F8000084069461F
:108A600009784907C90F490008406946097909078B
:108A7000C90F0840072816D008DC00280DD00228AE
:108A800017D0042812D006281FD109E0122813D0CD
:108A9000222814D0322818D114E00020207017E0CA
:108AA0000620207014E00720207011E004202070C0
:108AB0000EE0022020700BE01220207008E022203F
:108AC000207005E03220207002E00020207000BFFE
:108AD00000BF284605B0F0BDFEB506460D4614465B
:108AE0000027002D28D0012302AA1E212846FAF7CC
:108AF000A5FD07462078202188436946097A490167
:108B00002022114008432070207840218843694684
:108B1000097A8907C90F8901402211400843207052
:108B20002078802188436946097A4907C90FC9011D
:108B30008022114008432070002E51D001236A4644
:108B400012213046FAF77AFD0746207840084000A7
:108B500069460978C907C90F0843207020780221A7
:108B60008843694609780906C90F49000222114065
:108B700008432070002F33D168460078C007C00F2B
:108B800000282DD168460078C009002828D101238B
:108B900001AA1E213046FAF751FD0746207804212C
:108BA00088436946097989000422114008432070EE
:108BB000207808218843694609798907C90FC900C7
:108BC000082211400843207020781021884369460C
:108BD00009794907C90F0901102211400843207083
:108BE0003846FEBD33B583B00546012301AA0221F4
:108BF0002846FAF723FD0446694608798021884310
:108C00006946097C8907C90FC943C90180221140FF
:108C10000843019069460879402188436946097CE8
:108C200089014022114008430190012301AA022139
:108C30002846FAF716FD0419002C02D0204605B08C
:108C400030BD01236A4612212846FAF7F7FC044694
:108C500069460878102188436946097C4907C90F8D
:108C6000C9430901102211400843009001236A46BC
:108C700012212846FAF7F5FC0419002C01D02046F1
:108C8000DDE7012302AA62212846FAF7D7FC044651
:108C90006846007A410849006846007C0007C20F18
:108CA0000120904301430291012302AA6221284638
:108CB000FAF7D7FC04192046C1E7FEB506460C4674
:108CC000012301AA02213046FAF7B8FC0546002D1F
:108CD00001D02846FEBD20780221884369460979E3
:108CE000C909C94349000222114008432070207875
:108CF00002218843694609794906C90F4900114094
:108D00000843207001236A4612213046FAF796FC88
:108D10000546002D01D02846DCE720780421884351
:108D200069460978C906C90FC94389000422114060
:108D300008432070012302AA62213046FAF77EFC24
:108D400005462078082188436946097AC943C90045
:108D500008221140084320702846BBE733B583B092
:108D6000054601236A4612212846FAF767FC0446A5
:108D700069460878202188436946097C49012022F8
:108D800011400843009001236A4612212846FAF751
:108D900068FC0419002C02D0204605B030BD012328
:108DA00002AA56212846FAF749FC04466846007A8A
:108DB000410849006846007C8007C00F01430291CA
:108DC0006846007C8007C10F6846007C4007C00FE2
:108DD00001438801402108406946097A40229143B5
:108DE00008430290012302AA56212846FAF739FCCB
:108DF0000419002C01D02046CFE702212846FAF7BB
:108E000004FD0446002C01D02046C6E7012301AA38
:108E100017212846FAF712FC044669460879802192
:108E200088436946097C4907C90FC901802211405E
:108E300008430190012301AA17212846FAF711FCE3
:108E4000041900212846FAF7E0FC04192046A4E79B
:108E5000FEB506460C4601236A4612213046FAF753
:108E6000EDFB0546002D01D02846FEBD20784008C8
:108E70004000694609788906C90F0843207001231C
:108E800002AA56213046FAF7D9FB0546002D01D03B
:108E90002846EAE76946087A4106C90F08404000BB
:108EA00002210840217802229143084320700221C8
:108EB0003046FAF7AAFC0546002D01D02846D4E733
:108EC000012301AA17213046FAF7B8FB0546694687
:108ED0000879C009097A4906C90F084080000421B1
:108EE0000840217804229143084320700021304635
:108EF000FAF78BFC45192846B7E7F0B587B0074667
:108F00000E4614460025002E0FD001236A466F211D
:108F10003046FAF793FB0546207840084000694642
:108F200009780906C90F08432070002F71D0002D61
:108F300004D102213846FAF768FC0546002D06D117
:108F4000012306AA0E213846FAF778FB0546002DC4
:108F500006D1012305AA0F213846FAF76FFB054613
:108F6000002D06D1012304AA10213846FAF766FB2A
:108F70000546002D04D100213846FAF746FC054687
:108F8000002D06D1012303AA0E213846FAF756FB1D
:108F90000546002D06D1012302AA5F213846FAF7C3
:108FA0004DFB0546002D06D1012301AA13213846A9
:108FB000FAF744FB0546684600798006C00F002892
:108FC00028D1002D12D1012303AA0E213846FAF729
:108FD00035FB05462078082188436946097B490707
:108FE000C90FC9000822114008432070002D19D173
:108FF000012302AA5F213846FAF720FB0546607874
:10900000400840006946097AC907C90F08436070E3
:1090100008E081E1207808218843207060784008CA
:10902000400060702078022188436946097B49002E
:1090300002221140084320702078042188436946A9
:10904000097B8907C90F8900042211400843207059
:109050002078082188436946097B4907C90FC90060
:109060000822114008432070207810218843694667
:10907000097B0907C90F090110221140084320701C
:109080002078202188436946097BC906C90F490118
:1090900020221140084320702078402188436946EF
:1090A000097B8906C90F89014022114008432070BD
:1090B0002078802188436946097B4906C90FC90188
:1090C00080221140084320706078400840006946C3
:1090D000097AC907C90F0843607060780221884384
:1090E0006946097A4907C90F49000222114008431D
:1090F00060706078042188436946097A0907C90FBE
:109100008900042211400843607060780821884378
:109110006946097AC906C90FC900082211400843E7
:1091200060706078102188436946097A8906C90F02
:1091300009011022114008436070607820218843A3
:109140006946097A4906C90F49012022114008439E
:1091500060706078402188436946097A0906C90F22
:109160008901402211400843607060788021884363
:109170006946097E0907C90FC901802211400843C9
:109180006070A078400840006946097EC906C90F92
:109190000843A070A078042188436946097E090627
:1091A000C90F8900042211400843A070A07808214B
:1091B00088436946097DC900082211400843A07010
:1091C000A078102188436946097D8907C90F0901E4
:1091D000102211400843A070A078202188436946DE
:1091E000097D4907C90F4901202211400843A07099
:1091F000A078402188436946097D0907C90F890184
:10920000402211400843A070A0788021884369461D
:10921000097DC906C90FC901802211400843A07009
:10922000E078400840006946097D8906C90F084377
:10923000E070E078022188436946097D4906C90F3C
:109240004900022211400843E070E078042188437D
:109250006946097D0906C90F8900042211400843A7
:10926000E070E078082188436946097CC90008223B
:1092700011400843E070E078102188436946097C7A
:109280008907C90F0901102211400843E070E078F6
:10929000202188436946097C4907C90F49012022DA
:1092A00011400843E070E078402188436946097C1A
:1092B0000907C90F8901402211400843E070E07896
:1092C000802188436946097CC906C90FC9018022EB
:1092D00011400843E0702079400840006946097C4D
:1092E0008906C90F08432071207902218843694605
:1092F000097C4906C90F4900022211400843207128
:109300002079042188436946097C0906C90F890030
:109310000422114008432071284607B0F0BD37B53C
:109320008CB00546002006906846007E4108490042
:1093300008A8007DC007C00F014306916846007E63
:109340000221884308A9097D8907C90F4900022223
:109350001140084306906946087E0421884308A905
:10936000097D0907C90F89000422114008430690AE
:109370006946087E0821884308A9097DC906C90FE6
:10938000C90008221140084306906946087E102152
:10939000884308A9097D8906C90F090110221140D7
:1093A000084306906946087E2021884308A9097D64
:1093B0004906C90F49012022114008430690694619
:1093C000087E4021884308A9097D0906C90F890143
:1093D00040221140084306906946087E8021884358
:1093E00008A9497DC9018022114008430690012344
:1093F00006AA0D212846FAF734F90446002C02D0BB
:1094000020460FB030BD012301AA13212846FAF7E8
:1094100015F90446002C01D02046F2E708A9087D82
:109420004007C00F497D4907C90F0843002806D0EF
:1094300069460879202188432030019004E069467C
:109440000879202188430190012301AA132128468D
:10945000FAF707F90446002C01D02046D1E7012392
:1094600005AA0E212846FAF7E9F804466946087D60
:109470000421884308A9097D4907C90F89000422EE
:10948000114008430590012305AA0E212846FAF74A
:10949000E8F80419002C01D02046B2E7012303AA02
:1094A0005F212846FAF7CAF804466846007B41085F
:1094B000490008A8407D4007C00F014303910123E4
:1094C00003AA5F212846FAF7CCF80419002C01D032
:1094D000204696E708A80079C108C900099108A8A4
:1094E00000790821884308A9897D8907C90FC90027
:1094F000082211400843099008A9087910218843DF
:1095000008A9897D4907C90F0901102211400843A4
:10951000099008A908792021884308A9897D0907AD
:10952000C90F4901202211400843099008A9087970
:1095300040218843099008A908798021884308A917
:10954000897DC906C90FC9018022114008430990CD
:1095500008A800784108490008A8807D8006C00F4F
:109560000143089108A800780221884308A9897D51
:109570004906C90F4900022211400843089008A972
:1095800008780421884308A9897D0906C90F890044
:10959000042211400843089008A90878082188434C
:1095A00008A9C97DC900082211400843089008A9EC
:1095B00008781021884308A9C97D8907C90F0901C6
:1095C000102211400843089008A9087820218843F8
:1095D00008A9C97D4907C90F490120221140084344
:1095E000089008A908784021884308A9C97D09077F
:1095F000C90F8901402211400843089008A9087842
:109600008021884308A9C97DC906C90FC9018022E4
:109610001140084308906946087F4008400008A9A7
:10962000C97D8906C90F084307906946087F022152
:10963000884308A9C97D4906C90F49000222114083
:10964000084307906946087F0421884308A9C97D1B
:109650000906C90F89000422114008430790694692
:10966000087F0821884308A9097EC9000822114003
:10967000084307906946087F1021884308A9097E9E
:109680008907C90F09011022114008430790694654
:10969000087F2021884308A9097E4907C90F49018D
:1096A00020221140084307906946087F40218843E3
:1096B00008A9097E0907C90F890140221140084302
:1096C00007906946087F8021884308A9097EC9065A
:1096D000C90FC90180221140084307900221284682
:1096E000FAF793F80446002C01D0204689E60123BE
:1096F00009AA0A212846F9F7B4FF0446012308AA5B
:109700000B212846F9F7ADFF0419012307AA0C2104
:109710002846F9F7A6FF041900212846FAF775F83C
:109720000419002C01D020466BE66846007A4108F7
:10973000490008A8407D8007C00F01430291684698
:10974000007A0421884308A9497D0907C90F8900C7
:1097500004221140084302906946087A0821884390
:1097600008A9497DC906C90FC9000822114008434C
:1097700002906946087A1021884308A9497D890624
:10978000C90F090110221140084302906946087A66
:109790002021884308A9497D4906C90F4901202293
:1097A0001140084302906946087A4021884308A97D
:1097B000497D0906C90F89014022114008430290E2
:1097C0006946087A8021884308A9897DC9018022D9
:1097D00011400843029008A90879C009097989064F
:1097E000C90F084308A909790907C90F084308A93F
:1097F0000979C906C90F084308A90978C907C90F1B
:10980000084308A909788907C90F084308A90978F6
:109810004907C90F084308A909780907C90F084370
:1098200008A90978C906C90F084308A90978890653
:10983000C90F084308A909784906C90F084308A9B0
:109840000978C90908436946097FC907C90F084350
:109850006946097F8907C90F08436946097F490797
:10986000C90F08436946097F0907C90F08436946BC
:10987000097FC906C90F08436946097F8906C90FD0
:1098800008436946097F4906C90F08436946097FAD
:10989000C9090843002806D06946087A022188438E
:1098A000801C029004E06946087A022188430290F5
:1098B000012302AA5E212846F9F7D3FE0446002CB4
:1098C00001D020469DE5012304AA58212846F9F736
:1098D000B5FE04460AAA00212846FFF70EFB04192C
:1098E000002C01D020468CE508A9087AC009097A25
:1098F0004907C90F084308A9097A0907C90F08438E
:1099000008A9097A8907C90F084308A9097A4906ED
:10991000C90F084308A9097A8906C90F084308A98D
:10992000097AC906C90F084308A9497A8907C90FE6
:10993000084308A9497A4907C90F084308A9497A81
:109940000907C90F084308A9497AC906C90F08437E
:1099500008A9497A8906C90F084308A9497A49061E
:10996000C90F08436946097EC90908436946097E4B
:109970004907C90F08436946097E4906C90F0843CC
:109980006946097E8907C90F08436946097EC907E8
:10999000C90F08436946097E8906C90F084369460D
:1099A000097EC906C90F08436946097E0907C90F20
:1099B00008436946097AC907C90F08436946097A05
:1099C0004907C90F08436946097A0907C90F0843BF
:1099D0006946097AC906C90F08436946097A8906A2
:1099E000C90F08436946097A4906C90F0843694601
:1099F000097AC9090843002806D06946087C8021F5
:109A000088438030049004E06946087C80218843C4
:109A10000490012304AA58212846F9F722FE04469F
:109A20002046EEE470B588B006460C46022130466A
:109A3000F9F7EBFE0546002D02D0284608B070BDB0
:109A4000012307AA0A213046F9F7F8FD054601234C
:109A500006AA0B213046F9F7F1FD4519012305AAA5
:109A60000C213046F9F7EAFD451900213046F9F797
:109A7000CCFE4519002D01D02846DFE7012304AABA
:109A80000D213046F9F7DAFD0546002D01D02846B4
:109A9000D4E7012301AA5E213046F9F7CFFD054640
:109AA000002D01D02846C9E701236A46132130461C
:109AB000F9F7C4FD0546002D01D02846BEE76846EB
:109AC00000788006C00F002824D0012303AA0E21AD
:109AD0003046F9F7B3FD05462078042188436946EE
:109AE000097B4907C90F89000422114008432070EF
:109AF000012302AA5F213046F9F7A0FD45196078DD
:109B0000042188436946097A8900042211400843E8
:109B1000607006E0207804218843207060788843D4
:109B20006070002D01D0284688E72078400840006A
:109B30006946097CC907C90F0843207020780221B3
:109B400088436946097C8907C90F490002221140F0
:109B5000084320702078082188436946097C49071A
:109B6000C90FC90008221140084320702078102135
:109B700088436946097C0907C90F09011022114071
:109B8000084320702078202188436946097CC90653
:109B9000C90F49012022114008432070207840213C
:109BA00088436946097C8906C90F89014022114012
:109BB000084320702078802188436946097C490643
:109BC000C90FC90180221140084320706078400805
:109BD00040006946097C0906C90F08436070607837
:109BE000022188436946097949000222114008434D
:109BF0006070607808218843694609794907C90F70
:109C0000C900082211400843607060781021884321
:109C1000694609790907C90F090110221140084353
:109C2000607060782021884369460979C906C90FA8
:109C30004901202211400843607060784021884328
:109C4000694609798906C90F8901402211400843F4
:109C50006070607880218843694609794906C90F98
:109C6000C9018022114008436070A078400840007C
:109C7000694609790906C90F0843A070A078022136
:109C800088436946097F0907C90F4900022211402C
:109C90000843A070A078042188436946097FC9065B
:109CA000C90F8900042211400843A070A078082140
:109CB00088436946097F8906C90FC90008221140F7
:109CC0000843A070A078102188436946097F0906DF
:109CD000C90F0901102211400843A070A07820216B
:109CE00088436946097E4901202211400843A0703B
:109CF000A078402188436946097E8907C90F8901F8
:109D0000402211400843A070A07880218843694612
:109D1000097E4907C90FC901802211400843A0707C
:109D2000E078400840006946097E0907C90F0843EA
:109D3000E070E078022188436946097EC906C90FB0
:109D40004900022211400843E070E0780421884372
:109D50006946097E8906C90F89000422114008431B
:109D6000E070E078082188436946097E4906C90FFA
:109D7000C900082211400843E070E07810218843B0
:109D80006946097E0906C90F0901102211400843DE
:109D9000E070E078202188436946097D490120224E
:109DA00011400843E070E078402188436946097D0E
:109DB0008907C90F8901402211400843E070E0780B
:109DC000802188436946097D4907C90FC90180225E
:109DD00011400843E0702079400840006946097D41
:109DE0000907C90F08432071207902218843694679
:109DF000097DC906C90F490002221140084320719C
:109E00002079042188436946097D8906C90F8900A4
:109E100004221140084320712079082188436946B3
:109E2000097D4906C90FC900082211400843207165
:109E30002079102188436946097D0906C90F090167
:109E400010221140084320712846F7E57FB58AB0FB
:109E500006460D460024002D1DD001236A466F21C1
:109E60002846F9F7EBFB04466946087880218843C9
:109E700008A9097CC90180221140084300900123F0
:109E80006A466F212846F9F7ECFB0419002C02D032
:109E900020460EB070BD002E7ED06846007C410882
:109EA000490008A8007C8007C00F01430491684660
:109EB000007C0221884308A9097C4907C90F490091
:109EC00002221140084304906946087C042188431B
:109ED00008A9097C0907C90F890004221140084319
:109EE00004906946087C0821884308A9097CC906B2
:109EF000C90FC90008221140084304906946087C34
:109F00001021884308A9097C8906C90F090110227C
:109F10001140084304906946087C2021884308A921
:109F2000097C4906C90F49012022114008430490C9
:109F30006946087C4021884308A9097C0906C90FA5
:109F4000890140221140084304906946087C802121
:109F500088430490012304AA0E213046F9F781FBBF
:109F60000446002C01D0204693E76846007A410859
:109F7000490008A8407CC007C00F01430291684611
:109F8000007A0421884308A9497C8907C90F890000
:109F900004221140084300E0A1E202906946087AD9
:109FA0000821884308A9497C4907C90FC90008222C
:109FB0001140084302906946087A1021884308A995
:109FC000497C0907C90F090110221140084302907A
:109FD0006946087A2021884308A9497CC906C90F27
:109FE000490120221140084302906946087A402125
:109FF000884308A9497C8906C90F8901402211407C
:10A00000084302906946087A8021884308A9497C60
:10A010004906C90FC90180221140084302906946D0
:10A02000087FC008C0000790087F0821884308A95E
:10A03000497C0906C90FC90008221140084307904E
:10A040006946087F1021884308A9897C09011022EC
:10A050001140084307906946087F2021884308A9DA
:10A06000897C8907C90F49012022114008430790C4
:10A070006946087F4021884307906946087F802110
:10A08000884308A9897C4907C90FC901802211406A
:10A09000084307906846007E4108490008A8807C74
:10A0A0000007C00F014306916846007E02218843E5
:10A0B00008A9897CC906C90F49000222114008433A
:10A0C00006906946087E0421884308A9897C890690
:10A0D000C90F890004221140084306906946087E92
:10A0E0000821884308A9897C4906C90FC9000822AC
:10A0F0001140084306906946087E1021884308A94C
:10A10000897C0906C90F09011022114008430690F5
:10A110006946087E2021884308A9C97C490120227C
:10A120001140084306906946087E4021884308A9EB
:10A13000C97C8907C90F8901402211400843069054
:10A140006946087E8021884308A9C97C4907C90F50
:10A15000C90180221140084306906946087D4008E5
:10A16000400008A9C97C0907C90F08430590694642
:10A17000087D0221884308A9C97CC906C90F490086
:10A1800002221140084305906946087D0421884356
:10A1900008A9C97C8906C90F890004221140084317
:10A1A00005906946087D0821884308A9C97C4906AD
:10A1B000C90FC90008221140084305906946087D6F
:10A1C0001021884308A9C97C0906C90F090110227A
:10A1D0001140084305906946087D2021884308A95D
:10A1E000097D490120221140084305906946087DF8
:10A1F0004021884308A9097D8907C90F89014022A8
:10A200001140084305906946087D8021884308A9CC
:10A21000097D4907C90FC9018022114008430590F3
:10A22000012301AA13213046F9F708FA044608A9C8
:10A23000087C0007C00F497CC907C90F08430028E4
:10A2400004D069460879202188430190012301AA9E
:10A2500013213046F9F705FA0419002C01D02046E5
:10A2600017E602213046F9F7D0FA0446012307AA7F
:10A270000E213046F9F7F5F90419012306AA0F213A
:10A280003046F9F7EEF90419012305AA10213046EA
:10A29000F9F7E7F9041900213046F9F7B6FA04197D
:10A2A000002C01D02046F4E56946087FC009097FEB
:10A2B0008906C90F08436946097F0907C90F084382
:10A2C0006946097FC906C90F08436946097EC9075F
:10A2D000C90F08436946097E8907C90F08436946C3
:10A2E000097E4907C90F08436946097E0907C90F56
:10A2F00008436946097EC906C90F08436946097EB5
:10A300008906C90F08436946097E4906C90F0843F3
:10A310006946097EC90908436946097DC907C90F0D
:10A3200008436946097D8907C90F08436946097DC5
:10A330004907C90F08436946097D0907C90F084342
:10A340006946097DC906C90F08436946097D890622
:10A35000C90F08436946097D4906C90F0843694684
:10A36000097DC9090843002806D06946087A0221F8
:10A370008843801C029004E06946087A02218843E1
:10A380000290012302AA5F213046F9F76AF90446D8
:10A39000002C01D020467CE5012303AA5821304639
:10A3A000F9F74CF9044608A93046FFF73BFB0419BE
:10A3B00008A9087CC009097C4907C90F084308A9F6
:10A3C000097C0907C90F084308A9097C8907C90F37
:10A3D000084308A9097C4906C90F084308A9097C54
:10A3E0008906C90F084308A9097CC906C90F084393
:10A3F00008A9497C8907C90F084308A9497C49076E
:10A40000C90F084308A9497C0907C90F084308A9CF
:10A41000497CC906C90F084308A9497C8906C90FA8
:10A42000084308A9497C4906C90F084308A9497887
:10A43000C907C90F084308A909780907C90F0843C4
:10A4400008A90978C909084308A909788907C90F23
:10A45000084308A90978C907C90F084308A909785A
:10A460004906C90F084308A909788906C90F084396
:10A4700008A90978C906C90F084308A94978090736
:10A48000C90F084308A94978C906C90F084308A994
:10A4900049788906C90F084308A949784906C90FB0
:10A4A000084308A94978C909084308A98978C90750
:10A4B000C90F0843002806D06946087B80218843DD
:10A4C0008030039004E06946087B80218843039034
:10A4D000012303AA58213046F9F7C3F8041920468E
:10A4E000D7E470B58EB006460C46052301AA1A21A2
:10A4F0003046F9F7A3F80546002D02D028460EB0E5
:10A5000070BD01A907A8F9F7BFF801A9013106A894
:10A51000F9F7BAF801A9023104A8F9F7B5F801A9C9
:10A52000033103A8F9F7B0F802A905A8F9F7ACF8C8
:10A530002078102188436946097F0906C90F09015F
:10A5400010221140084320702078802188436946FA
:10A55000097EC901802211400843207060784008BC
:10A5600040006946097E8907C90F0843607060781A
:10A57000022188436946097E4907C90F4900022222
:10A580001140084360702078402188436946097E65
:10A590000907C90F89014022114008432070E07863
:10A5A000400840006946097EC906C90F0843E070AB
:10A5B0002078202188436946097E8906C90F490110
:10A5C0002022114008432070A078802188436946EA
:10A5D000097E4906C90FC901802211400843A070B5
:10A5E0006078402188436946097C4907C90F890181
:10A5F00040221140084360706078202188436946FA
:10A60000097C8907C90F4901202211400843607065
:10A610006078102188436946097C090110221140A5
:10A62000084360706078802188436946097C090787
:10A63000C90FC90180221140084360706078082169
:10A6400088436946097CC906C90FC9000822114020
:10A65000084360706078042188436946097C890654
:10A66000C90F89000422114008436070A0780221BC
:10A6700088436946097B4900022211400843A070C3
:10A68000A078042188436946097B8907C90F89009E
:10A69000042211400843A070A0780821884369462D
:10A6A000097B4907C90FC900082211400843A0705F
:10A6B000A078102188436946097B0907C90F090161
:10A6C000102211400843A070A078202188436946D9
:10A6D000097BC906C90F4901202211400843A07017
:10A6E000A078402188436946097B8906C90F890102
:10A6F000402211400843A070A078400840006946FD
:10A70000097B4906C90F0843A070207808218843B7
:10A710006946097B0906C90FC90008221140084390
:10A7200020702078400840006946097DC907C90F9C
:10A73000084320702078022188436946097D8907F3
:10A74000C90F4900022211400843207020780421DB
:10A7500088436946097D4907C90F890004221140D1
:10A7600008432070032301AA35213046F8F766FF1D
:10A770000546002D01D02846C1E601A90DA8F8F72D
:10A7800083FF01A901310BA8F8F77EFF01A902316F
:10A790000AA8F8F779FFE0780221884308A9097D23
:10A7A0000907C90F4900022211400843E070E07810
:10A7B0000421884308A9097DC906C90F890004221C
:10A7C00011400843E070E0780821884308A9097D1A
:10A7D0008906C90FC900082211400843E070E078DB
:10A7E0001021884308A9097D0906C90F0901102213
:10A7F00011400843E070E0782021884308A9097BD4
:10A800004901202211400843E070E078402188434C
:10A8100008A9097B8907C90F890140221140084313
:10A82000E070E0788021884308A9097B4907C90FB7
:10A83000C901802211400843E0702079400840009F
:10A8400008A9097B0907C90F084320712079022153
:10A85000884308A9097BC906C90F49000222114093
:10A860000843207120790421884308A9097B8906BF
:10A87000C90F890004221140084320712079082162
:10A88000884308A9097B4906C90FC900082211405D
:10A890000843207120791021884308A9097B090603
:10A8A000C90F09011022114008432071207920218D
:10A8B000884308A9097A49012022114008432071E0
:10A8C00020794021884308A9097A8907C90F89019D
:10A8D000402211400843207120798021884308A933
:10A8E000097A4907C90FC901802211400843207124
:10A8F00060794008400008A9097A0907C90F084390
:10A90000607160790221884308A9097AC906C90FD4
:10A910004900022211400843607160790421884394
:10A9200008A9097A8906C90F890004221140084341
:10A93000607160790821884308A9097A4906C90F1E
:10A94000C9000822114008436071607910218843D2
:10A9500008A9097A0906C90F090110221140084304
:10A960006071032301AA39213046F8F767FE0546D6
:10A97000002D01D02846C2E501A90CA8F8F784FEF5
:10A9800001A9013109A8F8F77FFE01A9023108A841
:10A99000F8F77AFEA0792021884308A9097C4901AB
:10A9A000202211400843A071A0794021884308A9C2
:10A9B000097C0907C90F8901402211400843A07191
:10A9C000A0798021884308A9097CC906C90FC9015B
:10A9D000802211400843A071E0794008400008A996
:10A9E000097C8906C90F0843E071E0790221884398
:10A9F00008A9097C4906C90F4900022211400843F1
:10AA0000E071E0790421884308A9097C0906C90F8F
:10AA10008900042211400843E07108A90878000267
:10AA2000097940188005800D2189890A8902084327
:10AA30002081607A0421884308A909780907C90F91
:10AA40008900114008436072607A0821884308A990
:10AA50000978C906C90FC90008221140084360726D
:10AA6000607A1021884308A909788906C90F09016D
:10AA70001022114008436072607A2021884308A99F
:10AA800009784906C90F4901202211400843607224
:10AA9000607A4021884308A909780906C90F89010D
:10AAA0004022114008436072284628E5F7B592B06D
:10AAB000144600200F900A900990002608A8007AFA
:10AAC000022188430A9008A80079400840000990B4
:10AAD00020781021084000090590207820210840A6
:10AAE00040090390207807073F0F0398002804D0FF
:10AAF00000216171E1710020A0706079012801D10D
:10AB00000121E171A0781021084000090490A0788B
:10AB100005072D0F1298002849D0082301AA129882
:10AB2000F8F78CFD0646002E02D0304615B0F0BD79
:10AB300001A90DA8F8F7A8FD01A901310BA8F8F7A4
:10AB4000A3FD01A902310AA8F8F79EFD01A903316E
:10AB500009A8F8F799FD02A908A8F8F795FD02A938
:10AB6000013107A8F8F790FD02A9023106A8F8F70D
:10AB70008BFD02A903310CA8F8F786FD012311AA69
:10AB800019461298F8F75AFD064608A80078C10938
:10AB9000039881420BD008A9087DF02188430D90CD
:10ABA00001230DAA10211298F8F75BFD06461398B1
:10ABB000002819D0032301AA70211398F8F73EFD4D
:10ABC0000646002E01D03046B0E701A910A8F8F7DC
:10ABD0005BFD01A901310FA8F8F756FD01A902316B
:10ABE0000EA8F8F751FD1BE01298002818D0032397
:10ABF00001AA70211298F8F721FD0646002E01D017
:10AC0000304693E701A910A8F8F73EFD01A90131EC
:10AC10000FA8F8F739FD01A902310EA8F8F734FDA5
:10AC2000607A002849D0A07A002806D0012813D0E5
:10AC3000022820D003283CD12CE0607A022802D0E0
:10AC4000002F00D10127607A012804D0002D02D105
:10AC50000020039001252FE0607A022802D0022F05
:10AC600000D20227607A012804D0022D02D20020EF
:10AC70000390022520E0607A022802D0032F00D240
:10AC80000327607A012804D0032D02D2002003900C
:10AC9000032511E0607A022802D0042F00D2042795
:10ACA000607A012804D0042D02D2002003900425EC
:10ACB00002E00027002500BF00BF08A80078C009F7
:10ACC00041016846007FC006C00F0001084308A983
:10ACD000097D0909084303000AF0B3F82C171A1D6F
:10ACE000202326292C2F32355C5C5C5C5C5C3B3E6F
:10ACF0004144475C5C5C5C5C385C5C5C5C5C4D501B
:10AD00005356595C5C5C5C5C4A5C0020207044E0FB
:10AD10000120207041E0022020703EE003202070DE
:10AD20003BE00420207038E00520207035E006204C
:10AD3000207032E0072020702FE0082020702CE0E7
:10AD40000920207029E00A20207026E01B202070B6
:10AD500023E01120207020E0122020701DE013203D
:10AD600020701AE01420207017E01520207014E0E5
:10AD70002B20207011E0212020700EE02220207076
:10AD80000BE02320207008E02420207005E025201F
:10AD9000207002E00020207000BF00BF6946087EDE
:10ADA000C009000108A9097B0909084303000AF04A
:10ADB00048F8160C12181E242A2D303336393C3C24
:10ADC0003C3C3C3C0F151B21273C0020A0702FE091
:10ADD0001120A0702CE00120A07029E01220A070AA
:10ADE00026E00220A07023E01320A07020E00320C2
:10ADF000A0701DE01420A0701AE00420A07017E0DD
:10AE00001520A07014E00520A07011E00620A070AD
:10AE10000EE00720A0700BE00820A07008E00920D9
:10AE2000A07005E00A20A07002E00020A07000BF22
:10AE300000BF6078012802D0A079012803D1012049
:10AE400060700121A1716078012805D108A9087CF2
:10AE5000022188430C9005E008A9087C0221884360
:10AE6000801C0C906846007E0421884321790129CA
:10AE700000D100E00021890004221140084306901F
:10AE80002079002802D0012854D129E010A80078A8
:10AE90000E218843217A49000E221140014310916E
:10AEA000E07961790843C107C90F10A8007840080C
:10AEB00040000143109110A8007810218843617967
:10AEC0000901102211400143109108A8007EC02101
:10AED0008843A1798901C022114008430E9053E0B4
:10AEE00010A800780E218843217A49000E221140D3
:10AEF00001431091E07961790843C107C90F6846A1
:10AF0000007E400840000143069110A800781021FF
:10AF1000884361790901102211400143109108A86A
:10AF2000007EC0218843A1798901C02211400843D5
:10AF30000E9029E010A800780E218843217A49005C
:10AF40000E22114001431091E07961790843C10755
:10AF5000C90F10A80078400840000143109110A8C4
:10AF600000781021884361790901102211400143C2
:10AF7000109108A8007EC0218843A1798901C022D0
:10AF8000114008430E9000BF00BF08A8007DF021CB
:10AF900088433901F022114001430D9108A8007D3A
:10AFA0000C218843617889000C22114001430D91E6
:10AFB00008A80078802188430399C90180221140A4
:10AFC000014308916846007F1021884305990901D3
:10AFD00010221140014307916846007E802188437A
:10AFE0000499C901802211400143069108A8007B01
:10AFF000F02188432901F022114001430B9108A858
:10B00000007B0E218843E17849000E22114008435D
:10B010000B901298002837D00DA901A8F8F734FB3F
:10B020000BA901A80130F8F72FFB0AA901A80230EB
:10B03000F8F72AFB09A901A80330F8F725FB08A9AE
:10B0400002A8F8F721FB07A902A80130F8F71CFBBA
:10B0500006A902A80230F8F717FB0CA902A80330D2
:10B06000F8F712FB082301AA10211298F8F7F9FA51
:10B070000646012311AA19461298F8F7F2FA861922
:10B08000002E01D0304651E51398002814D010A9A5
:10B0900001A8F8F7F9FA0FA901A80130F8F7F4FAB6
:10B0A0000EA901A80230F8F7EFFA032301AA7021D4
:10B0B0001398F8F7D6FA0646304637E5F0B591B062
:10B0C00006460F4614460025002E6BD007236A461D
:10B0D00010213046F8F7B2FA0546002D02D0284676
:10B0E00011B0F0BD694608A8F8F7CEFA00A9013101
:10B0F00007A8F8F7C9FA00A9023106A8F8F7C4FAB8
:10B1000000A9033105A8F8F7BFFA01A904A8F8F7C8
:10B11000BBFA01A9013103A8F8F7B6FA01A9023177
:10B1200002A8F8F7B1FA01230FAA19463046F8F73A
:10B1300085FA0546002D01D02846D1E70221304688
:10B14000F8F763FB0546002D01D02846C8E7012328
:10B150006A465F213046F8F771FA0546694610A83D
:10B16000F8F792FA01230EAA05213046F8F766FA9D
:10B17000451900A901310CA8F8F786FA02236A469E
:10B1800046213046F8F75AFA451969460DA8F8F7EE
:10B190007BFA00213046F8F738FB4519002D01D025
:10B1A00028469DE7002F19D003236A4670213846B0
:10B1B000F8F744FA0546002D01D0284690E7694685
:10B1C0000BA8F8F761FA00A901310AA8F8F75CFAB0
:10B1D00000A9023109A8F8F757FA1AE0002E18D092
:10B1E00003236A4670213046F8F728FA0546002DF9
:10B1F00001D0284674E769460BA8F8F745FA00A97C
:10B2000001310AA8F8F740FA00A9023109A8F8F7B5
:10B210003BFA6846007CC00941016846007BC006D5
:10B22000C00F0001084308A9097809090843030071
:10B2300009F007FE2C171A1D202326292C2F323542
:10B240005C5C5C5C5C5C3B3E4144475C5C5C5C5CC5
:10B25000385C5C5C5C5C4D505356595C5C5C5C5C7F
:10B260004A5C0020207044E00120207041E0022070
:10B2700020703EE0032020703BE00420207038E086
:10B280000520207035E00620207032E00720207075
:10B290002FE0082020702CE00920207029E00A20EF
:10B2A000207026E01B20207023E01120207020E079
:10B2B000122020701DE0132020701AE0142020704E
:10B2C00017E01520207014E02B20207011E02120C1
:10B2D00020700EE0222020700BE02320207008E078
:10B2E0002420207005E02520207002E0002020703E
:10B2F00000BF00BF08A800780007800F002806D014
:10B3000001280DD0022805D003280CD105E000202B
:10B3100060700BE00220607008E00320607005E0C0
:10B320000120607002E00020607000BF00BF69462D
:10B33000087AC0090001097F09090843030009F0E0
:10B3400080FD160C12181E242A2D303336393C3C51
:10B350003C3C3C3C0F151B21273C0020A0702FE0FB
:10B360001120A0702CE00120A07029E01220A07014
:10B3700026E00220A07023E01320A07020E003202C
:10B38000A0701DE01420A0701AE00420A07017E047
:10B390001520A07014E00520A07011E00620A07018
:10B3A0000EE00720A0700BE00820A07008E0092044
:10B3B000A07005E00A20A07002E00020A07000BF8D
:10B3C00000BF6846007F0007400F030009F039FD09
:10B3D0000708050B140E141114000121E1700EE092
:10B3E0000021E1700BE00221E17008E00421E1702E
:10B3F00005E00621E17002E00121E17000BF00BF1D
:10B4000008A9087DC007C00F097D8907C90F084337
:10B4100008A9097D4907C90F084308A9097D09073B
:10B42000C90F084308A9097DC906C90F084308A91F
:10B43000097D8906C90F084308A9097D4906C90F76
:10B44000084308A9097DC909084308A9097CC90757
:10B45000C90F084308A9097C8907C90F084308A92F
:10B46000097C4907C90F084308A9097C0907C90FC6
:10B47000084308A9097CC906C90F084308A9097C23
:10B480008906C90F084308A9097C4906C90F084362
:10B4900008A9097CC9090843002829D010A8007808
:10B4A000C006800F002806D0012807D0022808D047
:10B4B00003280CD108E00021A1720BE00121A17248
:10B4C00008E00221A17205E00321A17202E000213F
:10B4D000A17200BF00BF03206072A078002801D1D4
:10B4E000012060722078002804D10220607201E0FF
:10B4F000002060726846007A4007C00F002802D022
:10B5000001286ED161E008A800798009002806D0E2
:10B5100001280DD0022805D003280CD105E0002118
:10B52000A1710BE00221A17108E00321A17105E0E6
:10B530000121A17102E00021A17100BF00BF08A894
:10B54000007BC006C00F002802D0012806D102E00F
:10B550000021617105E00121617102E0002161714A
:10B5600000BF00BF08A8007B0007400F002806D0DE
:10B57000022807D0042808D006280CD108E00021B2
:10B5800021720BE00221217208E00421217205E002
:10B590000621217202E00021217200BF00BF08A82D
:10B5A000007BC007C00F002802D0012806D102E0AE
:10B5B0000021E17105E00121E17102E00021E1716A
:10B5C00000BF00BF002020716AE008A80079800950
:10B5D000002807D001280ED0022806D003280DD15C
:10B5E00006E055E00021A1710BE00221A17108E005
:10B5F0000321A17105E00121A17102E00021A171E7
:10B6000000BF00BF08A8007BC006C00F002802D002
:10B61000012806D102E00021617105E0012161717C
:10B6200002E00021617100BF00BF08A8007B000795
:10B63000400F002806D0022807D0042808D006288A
:10B640000CD108E0002121720BE00221217208E0F8
:10B650000421217205E00621217202E000212172FD
:10B6600000BF00BF08A8007BC007C00F002802D0A1
:10B67000012806D102E00021E17105E00121E1711C
:10B6800002E00021E17100BF00BF0120207107E04E
:10B6900000212172E1716171A1710020207100BF50
:10B6A00000BF28461CE5FFB585B017461D460020A3
:10B6B0000090059800280CD00E2301AA202105989F
:10B6C000F7F7BCFF00900098002802D0009809B05E
:10B6D000F0BD002601A9701C095CA9852C20405DE5
:10B6E000000201A9895D401801B2A985B61C2C2071
:10B6F000285EF8F72AF8A86200245CE001A9701C13
:10B70000095C62002846203081526100405C0002E2
:10B7100001A9895D401801B262002846203081529B
:10B72000B01CC6B2F878030009F08BFB0705101BAC
:10B730003C263C313C00620029462031885EF7F708
:10B74000E6FFA20029461431885031E06200294604
:10B750002031885EF7F7C7FFA200294614318850D0
:10B7600026E0620029462031885EF7F7C6FFA20076
:10B770002946143188501BE0620029462031885E3A
:10B78000F7F7CFFFA20029461431885010E062007D
:10B7900029462031885EF7F7CEFFA20029461431F2
:10B7A000885005E00021A20028461430815000BFD7
:10B7B00000BF601CC4B2032CA0D3002448E001A940
:10B7C000701C095C620028460C3081526100405CAC
:10B7D000000201A9895D401801B2620028460C30C0
:10B7E0008152B01CC6B27878002806D001281FD03C
:10B7F00002280BD0032824D111E0620029460C3125
:10B80000885EF7F748FFA10068501EE062002946F5
:10B810000C31885EF7F749FFA100685015E062001F
:10B8200029460C31885EF7F74AFFA10068500CE00A
:10B83000620029460C31885EF7F74BFFA100685083
:10B8400003E00020A100685000BF00BF601CC4B22C
:10B85000032CB4D3069800280BD00C2301AA222174
:10B860000698F7F7EBFE00900098002801D00098AA
:10B870002DE70026002461E001A9701C095C62002C
:10B880002846503081526100405C000201A9895D68
:10B89000401801B26200284650308152B01CC6B236
:10B8A000387A030009F0CDFA0705111D4129413509
:10B8B0004100620029465031885EF7F728FF0146B3
:10B8C000A20028464430815035E0620029465031BC
:10B8D000885EF7F708FF0146A200284644308150F1
:10B8E00029E0620029465031885EF7F706FF0146DD
:10B8F000A2002846443081501DE0620029465031A4
:10B90000885EF7F70EFF0146A200284644308150BA
:10B9100011E0620029465031885EF7F70CFF0146BE
:10B92000A20028464430815005E00021A2002846AC
:10B930004430815000BF00BF601CC4B2032C9BD3B5
:10B94000002452E001A9701C095C620028463C30CA
:10B9500081526100405C000201A9895D401801B27A
:10B96000620028463C308152B01CC6B2B87900282B
:10B9700006D0012825D002280DD003282CD115E0AF
:10B98000620029463C31885EF7F785FEA200294611
:10B990003031885026E0620029463C31885EF7F756
:10B9A00084FEA2002946303188501BE062002946FF
:10B9B0003C31885EF7F783FEA2002946303188507B
:10B9C00010E0620029463C31885EF7F782FEA20053
:10B9D00029463031885005E00021A2002846303049
:10B9E000815000BF00BF601CC4B2032CAAD30098D2
:10B9F0006DE67CB506460C4602213046F7F705FF9A
:10BA00000546002D01D028467CBD012301AA042152
:10BA10003046F7F713FE054601236A4605213046F6
:10BA2000F7F70CFE4519002D00D051E0684600786C
:10BA3000400840002178C906C90F014300916846BB
:10BA400000791021884321788907C90F0901102244
:10BA5000114001430191684600790821884321780B
:10BA60004907C90FC90008221140014301916846E6
:10BA700000781021884321780907C90F0901102295
:10BA800011400143009168460079202188432178C4
:10BA900049012022114001430191684600780821A4
:10BAA000884321788906C90FC9000822114008433C
:10BAB0000090012301AA04213046F7F7D2FD054684
:10BAC00001236A4605213046F7F7CBFD451900BF33
:10BAD00000213046F7F799FE4519284694E77CB5D2
:10BAE00006460C4602213046F7F78FFE0546002D2C
:10BAF00001D028467CBD012301AA04213046F7F776
:10BB00009DFD054601236A4605213046F7F796FD5F
:10BB100045192078102188436946097809011022C7
:10BB20001140084320702078022188436946097932
:10BB3000C906C90F4900022211400843207020782D
:10BB400004218843694609790907C90F890004223D
:10BB500011400843207020780821884369460978FD
:10BB6000C906C90FC9000822114008432070207877
:10BB700040084000694609798906C90F08432070CA
:10BB8000207820218843694609780907C90F4901AF
:10BB9000202211400843207000213046F7F735FE7F
:10BBA00045192846A6E77CB5054602212846F7F741
:10BBB0002CFE0446002C01D020467CBD012301AAA6
:10BBC00004212846F7F73AFD044601236A46052179
:10BBD0002846F7F733FD0419002C00D02CE0684606
:10BBE0000078410849000091684600791021884397
:10BBF00001906846007908218843019068460078E2
:10BC000010218843009068460079202188430190E4
:10BC100068460078082188430090012301AA042186
:10BC20002846F7F71EFD044601236A4605212846EB
:10BC3000F7F717FD041900BF00212846F7F7E5FDC7
:10BC400004192046B9E70000F7480068F64949683A
:10BC5000401870470146002900D17047087B102822
:10BC600001D10120F9E70020F7E700B502461046B0
:10BC7000FFF7F0FF002800D100BD1069FCE7014686
:10BC8000002900D17047087B082801D10120F9E77D
:10BC90000020F7E700B502461046FFF7F0FF002846
:10BCA00001D1E24900BDD1699069FBE708B50E20DA
:10BCB00007230122DEA10090E04809F097F8DF4851
:10BCC00008BD70B504460D46002C01D0002D01D1F1
:10BCD000012070BDAC4201D10020FAE705E02078D8
:10BCE000002800D1F5E7641C6D1C207807F0F2FEF7
:10BCF0000646287807F0EEFE8642F0D0207807F05E
:10BD0000E9FE0646287807F0E5FE301AE1E7F8B5C7
:10BD100004460D4600260027002C00D1F8BD204621
:10BD200007F002FF461C3046296888470746002F67
:10BD300000D1F3E732462146384607F0D1FE3846B7
:10BD4000ECE7002807D1BE49BE4A1160BE495160E8
:10BD5000BE4991607047BA49BA4A1160016800292A
:10BD600001D001681160B849B64A516041680029A4
:10BD700001D0416851600021B24A916011460968C2
:10BD8000AF4A914207D1AF494968AF4A914202D1C7
:10BD9000AE49AC4A916000BFDCE770B5044628208C
:10BDA000216888470546002D03D02821284607F042
:10BDB000B0FE284670BD70B5044600252BE025680E
:10BDC000FF210131E0680840002805D1A068002863
:10BDD00002D0A068FFF7EFFFFF210131E0680840C3
:10BDE000002806D12069002803D0964A20695168AE
:10BDF000884701214902E0680840002806D1206AEE
:10BE0000002803D08F4A206A516888478D484168CE
:10BE1000204688472C46002CD1D170BD2E2070477B
:10BE2000F3B593B00C4600BF00201290FFF7F6FF69
:10BE300001900025002C02D02068002802D10020AB
:10BE400015B0F0BD00253CE0A16820684018405DB9
:10BE500034281FD009DC2B38030008F0F2FF092139
:10BE60002F222B2F1718191A2F00382816D006DC6E
:10BE7000352810D036280FD037281FD10DE03928AB
:10BE80000DD045280FD0652818D10BE000BF00BFAA
:10BE900000BF00BF00BF00BF00BF00BF00BF00BFAA
:10BEA00000BF00BF00BFA16820684018405D02A924
:10BEB000485504E002A90198485500E00BE000BF96
:10BEC0006D1C3F2D06D2002C04D0A068401961687B
:10BED0008842B9D300BF002002A9485512A902A880
:10BEE00009F0E8FC06460F4602A81299884201D1E3
:10BEF0000020A5E71398C7618661554A554B304627
:10BF0000394608F055FB03D853491398416111E0B5
:10BF10000022524B3046394608F036FB04D8012146
:10BF2000C9071398416105E03046394608F0D6FA52
:10BF30001399486108211398C160A06802AA129958
:10BF4000891A4018A06001207AE770B506461446A9
:10BF50001D463F4A3F4B2046294608F029FB02D8A0
:10BF60003D4870610FE000223C4B2046294608F016
:10BF70000BFB03D80120C007706104E0204629466E
:10BF800008F0ACFA706120462946F561B46170BDD5
:10BF900010B504462B4841682046884710BDF8B5C7
:10BFA00004460E4600251021E0680840002804D011
:10BFB0000901E0680840002801D00020F8BD3046A3
:10BFC00007F0B2FD0746206907F0AEFD874205D8AD
:10BFD0003146206907F0CAFD2069EFE7194930466C
:10BFE000FFF795FE0546002D00D1E7E72069002800
:10BFF00002D02069FFF7CCFF25612846DEE7F8B5BF
:10C0000004460D4600260027002C02D02068002898
:10C0100001D10020F8BD6068002821D06168A068C7
:10C0200088421DD30020F5E7BC3000200000F87FD7
:10C0300025692E25692E2569000000009432002014
:10C04000C14E0110C43000205D4E01104158011056
:10C050000000C0FFFFFFDF41FFFFFF7F0000E0C1E6
:10C06000F648854201D90020D4E7A068401C451954
:10C070006068A84203D3A16820684018CAE7206915
:10C08000002801D00020C5E7ED48854206D9EB48DD
:10C09000854201D8074602E00020BBE76F00206A16
:10C0A00000280DD03946226A206890470646002EA7
:10C0B0001CD1E16920688847002060602060A9E702
:10C0C0003846A16988470646002E06D1E1692068F6
:10C0D00088470020606020609CE7A068421C3046D2
:10C0E000216807F0FDFCE1692068884767602660E9
:10C0F000A06880198EE770B504460025002C02D098
:10C100002068002800D170BDA16820684518284625
:10C1100007F00AFDA1684018A06000BFF3E7F0B582
:10C1200087B004460D4616461F4678004008029622
:10C130000390680040083246009401902046039B1B
:10C14000019908F035FA03D269004908204602E057
:10C15000304679004908059104900022B94B0599B1
:10C16000049808F08DF832463B4603910290204631
:10C17000294608F077F84900490801910090039B8F
:10C18000029A08F001FA02D8012007B0F0BD0020A1
:10C19000FBE7F3B58FB00F4600200D900F99CE69E5
:10C1A0008D690C9000241C2105A807F0B2FCFFF754
:10C1B00035FE0490002002900390002F01D111B0B1
:10C1C000F0BD01960095009A0199002A01D0012244
:10C1D00000E0002208461043410049089A4A511ADB
:10C1E000C90F00290ED10196009501984000510019
:10C1F000884204D10098002801D1012000E00020ED
:10C20000002805D091A105A808F0F0FD0C901CE0D5
:10C210002A4633468FA105A808F0E8FD0C9002AA33
:10C220008EA105A807F0CEFC012807D12A46334687
:10C2300003990298FFF773FF002806D12A46334678
:10C2400087A105A808F0D2FD0C900C98002802DB0D
:10C250000C98192801DD0020B1E70C99491C3846DB
:10C26000FFF7CDFE0D900D98002800D1A7E7002420
:10C270000EE005A8015D0498814203D12E210D989E
:10C28000015504E005A8015D0D98015500BF641C2F
:10C290000C988442EDD300210D980155B9680C9893
:10C2A0000818B86001208AE702460023002100BF79
:10C2B00023E0505C302806DB505C392803DC505CFE
:10C2C0003038C31815E0505C412806DB505C462826
:10C2D00003DC505C3738C3180BE0505C612806DB88
:10C2E000505C662803DC505C5738C31801E000201E
:10C2F0007047032900D21B01491C0429D9D31846D1
:10C30000F6E7F7B586B01546002400260698059096
:10C310000020049003900290019007990598081A54
:10C32000062800DA88E00598801CFFF7BDFF064666
:10C3300037208002864203D34B48864200D87BE0F8
:10C340001B20C00286422CD34848864229D8059833
:10C35000871D002000900C2002900798C01B062823
:10C3600000DA69E038785C2802D17878752800D046
:10C3700062E0B81CFFF798FF00903721890200980F
:10C38000884203D338490098884200D954E0B00568
:10C39000000B00998905890D0843012109044418FF
:10C3A00002E0062002903446802C02D20120049044
:10C3B0001AE00120C002844204D202200490C0206E
:10C3C000019011E001200004844204D20320049073
:10C3D000E020019008E02648844204D8042004901C
:10C3E000F020019000E027E00498401EC0B20390C6
:10C3F0000CE0204680210843BF2108402A680399A9
:10C400005054A4090398401EC0B20390039800281A
:10C41000EFDC0498012804DD0198204329680870A6
:10C4200003E06006400E296808702968049808181F
:10C430002860029809B0F0BD0020FBE7FFFFFF7FF6
:10C44000FFFFFF3F0000B03C0000F07F6E756C6C9A
:10C450000000000025312E3135670000256C670093
:10C4600025312E3137670000FFDF0000FFDB0000C1
:10C47000FFFF1000F3B583B00C46A1682068401898
:10C48000461CA16820684018451C00200290002727
:10C49000A1682068405C222800D0AAE0002001901A
:10C4A00000900EE028785C280AD1681C2168401AA8
:10C4B0006168884200D39CE00098401C00906D1C8D
:10C4C0006D1C2068281A6168884202D228782228C8
:10C4D000E8D12068281A6168884202D22878222888
:10C4E00000D086E0A16820684018291A0098081A30
:10C4F000019021690198401C88470746002F00D110
:10C5000077E0029762E030785C2807D030780299B3
:10C510000870761C0298401C029057E0022001909F
:10C52000A81B012800DA64E07078662819D008DCBE
:10C53000222832D02F2832D05C282FD0622840D138
:10C5400008E06E2814D0722819D074281ED07528DF
:10C5500037D12BE00820029908700298401C029005
:10C5600030E00C20029908700298401C029029E0EB
:10C570000A20029908700298401C029022E00D20C7
:10C58000029908700298401C02901BE00920029951
:10C5900008700298401C029014E000BF00BF707841
:10C5A000029908700298401C02900BE002AA2946EA
:10C5B0003046FFF7A6FE01900198002800D118E050
:10C5C00000E016E000BF0198361800BFAE429AD3D3
:10C5D00000200299087010210398C1600398076138
:10C5E0002068281AA060A068401CA060012005B047
:10C5F000F0BD002F02D0384661698847002E02D076
:10C600002068301AA0600020F1E7F3B583B0074638
:10C6100000240026002500200290019004980028A4
:10C6200001D105B0F0BD002F0DD103210498FFF713
:10C63000E6FC0646002E00D1F3E7F7A1304607F0EE
:10C6400095FA0120EDE73C4624E020780C2811D033
:10C6500006DC08280DD009280FD00A2811D10AE0DD
:10C660000D2809D0222802D05C280AD100E000BFA2
:10C6700000BF00BF00BF00BF00BF0198401C019079
:10C6800006E02078202802DA0198401D019000BFC2
:10C6900000BF641C20780028D7D1E11B019808183E
:10C6A00002900299C91C0498FFF7A9FC0646002EC7
:10C6B00000D1B6E70198002810D122203070394609
:10C6C000701C029A07F00CFA22210298401C315487
:10C6D00000210298801C31540120A2E722203070F2
:10C6E000751C3C463DE020781F2808DD2078222874
:10C6F00005D020785C2802D0207828702FE05C20BC
:10C7000028706D1C20780C2815D006DC08280FD066
:10C71000092819D00A281AD110E00D2811D0222892
:10C7200003D05C2813D1287018E02220287015E06F
:10C730006220287012E0662028700FE06E202870BA
:10C740000CE07220287009E07420287006E022783E
:10C75000B2A1284608F04AFB2D1D00BF00BF641C93
:10C760006D1C20780028BED122210298401C315433
:10C7700000210298801C3154012052E770B5044614
:10C780000D4629462069FFF740FF70BD014600298C
:10C7900002D00868002801D100207047002903D08A
:10C7A0004A688868904201D30846F6E702E0886844
:10C7B000401C8860002908D04A688868904204D2EA
:10C7C0008A680868805C2028F1DD4A6888689042A1
:10C7D00002D18868401E88600846DEE710B504462E
:10C7E000002C05D02068002802D0A068002801D0C5
:10C7F000002010BD002C10D0A068001D6168884288
:10C800000BD2A26821688818032286A107F0B7F925
:10C81000002802D1A068C01CA0602046E9E7F3B55B
:10C8200081B00C46002600257D21C900E0688842C1
:10C8300001D30020FEBDE068401CE060002C08D061
:10C840006168A068884204D2A1682068405C7B28A7
:10C8500000D087E0A068401CA0602046FFF796FF4C
:10C86000002C09D06168A068884205D2A1682068C0
:10C87000405C7D2800D165E0002C03D06168A06891
:10C88000884203D3A068401EA0606BE0A068401EF1
:10C89000A06000BF20461030FFF77FFA0746002F48
:10C8A00000D15FE0002E02D13E463D4602E02F60FF
:10C8B0007D603D46A068401CA0602046FFF766FFF3
:10C8C00021462846FFF7D6FD002800D14AE0204641
:10C8D000FFF75CFF2869286200202861002C08D03F
:10C8E0006168A068884204D2A1682068405C3A2848
:10C8F00000D037E0A068401CA0602046FFF746FF4C
:10C900002146284600F0C2F8002800D12AE020463F
:10C91000FFF73CFF002C08D06168A068884204D271
:10C92000A1682068405C2C28B4D0002C08D0616835
:10C93000A068884204D2A1682068405C7D2800D0AD
:10C9400010E000BFE068401EE060002E00D075607F
:10C9500040210198C16001988660A068401CA060D9
:10C96000012067E7002E02D03046FFF724FA0020AE
:10C9700060E7F3B581B00C46002500277D21C90092
:10C98000E068884201D30020FEBDE068401CE06002
:10C99000A1682068405C5B2800D070E0A068401C63
:10C9A000A0602046FFF7F2FE002C09D06168A06865
:10C9B000884205D2A1682068405C5D2800D14EE025
:10C9C000002C03D06168A068884203D3A068401E91
:10C9D000A06054E0A068401EA06000BF2046103058
:10C9E000FFF7DBF90646002E00D148E0002D02D10A
:10C9F0003546374602E03E6077603746A068401C07
:10CA0000A0602046FFF7C2FE2146384600F03EF8FF
:10CA1000002809D133E000002222000075253034BF
:10CA200078000000EFBBBF002046FFF7AFFE002CF0
:10CA300008D06168A068884204D2A1682068405C80
:10CA40002C28CBD0002C08D06168A068884204D282
:10CA5000A1682068405C5D2800D010E000BFE0685D
:10CA6000401EE060002D00D06F6020210198C16061
:10CA700001988560A068401CA060012084E7002D1B
:10CA800002D02846FFF797F900207DE770B50546EC
:10CA90000C46002C02D02068002801D1002070BD77
:10CAA000002C14D0A068001D616888420FD8A268CD
:10CAB000216888180422F94907F061F8002806D196
:10CAC0000420E860A068001DA0600120E7E7002CBA
:10CAD00014D0A068401D616888420FD8A268216800
:10CAE00088180522EEA107F04AF8002806D1012097
:10CAF000E860A068401DA0600120D0E7002C16D09F
:10CB0000A068001D6168884211D8A2682168881851
:10CB10000422E5A107F033F8002808D10220E860DC
:10CB200001206861A068001DA0600120B7E7002C0B
:10CB30000DD06168A068884209D2A1682068405C75
:10CB4000222804D121462846FFF794FCA7E7002CB1
:10CB500017D06168A068884213D2A1682068405C41
:10CB60002D2809D0A1682068405C302809DBA16825
:10CB70002068405C392804DC21462846FFF750F93C
:10CB80008DE7002C0DD06168A068884209D2A168A9
:10CB90002068405C5B2804D121462846FFF7E9FE67
:10CBA0007DE7002C0DD06168A068884209D2A16899
:10CBB0002068405C7B2804D121462846FFF72FFEE1
:10CBC0006DE700206BE7FFB589B004460E461546B9
:10CBD0001C2102A806F09DFF00270020B449086030
:10CBE0004860002C01D0002E00D135E0029403965D
:10CBF00000200490AF4A07CA06AB07C3AD48FFF751
:10CC0000CCF80746002F00D126E002A8FFF7E6FD8A
:10CC10000090FFF7BBFD014601903846FFF736FF55
:10CC2000002800D118E00C9800280CD002A8FFF7CB
:10CC3000ADFD03990498884204D204990298405C9F
:10CC4000002800D008E0002D03D004990298401875
:10CC5000286038460DB0F0BD002F02D03846FFF7EF
:10CC6000AAF8002C1AD0009400200190039904988F
:10CC7000884202D20498019005E00398002802D06F
:10CC80000398401E0190002D03D001990098401890
:10CC900028608748019A009906C000BF0020D9E7A4
:10CCA000F8B504460D461646002C00D1F8BD2046C6
:10CCB00006F03AFF471C33462A4639462046FFF71E
:10CCC00082FFF3E710B50446002211462046FFF725
:10CCD000E7FF10BD70B504460D4600231A462946ED
:10CCE0002046FFF770FF70BDF3B581B00C460025FC
:10CCF000002601988768002C01D10020FEBD6069E4
:10CD0000002801D0022000E001200646711C2046C8
:10CD1000FFF775F90546002D00D1EFE77B2028705D
:10CD20006D1CE068401CE0606069002802D00A20A9
:10CD300028706D1CA0688019A06072E060690028EE
:10CD400019D02046E168FFF75AF90546002D00D1B9
:10CD5000D4E70020009005E0092028706D1C0098A1
:10CD6000401C0090E16800988142F5D8E168A06815
:10CD70004018A06000BF2146386AFFF746FC002833
:10CD800000D1BBE72046FFF7B6F96069002801D063
:10CD9000022000E00120064631462046FFF72FF929
:10CDA0000546002D00D1A9E73A2028706D1C606966
:10CDB000002802D0092028706D1CA0688019A0608E
:10CDC0002146384600F0C0F8002800D196E72046FA
:10CDD000FFF791F96069002801D0012000E00020F0
:10CDE0003968002901D0012100E000214618711C9A
:10CDF0002046FFF704F90546002D00D17EE738688C
:10CE0000002802D02C2028706D1C6069002802D0F8
:10CE10000A2028706D1C00202870A0688019A0606E
:10CE20003F68002F8AD16069002802D0E068401C6A
:10CE300000E0022001462046FFF7E1F80546002DFC
:10CE400000D15BE7606900280AD0002003E00921D7
:10CE500029706D1C401CE168491E8142F7D800BF53
:10CE60007D2028706D1C00202870E068401EE06066
:10CE7000012043E7F3B581B00C4600250027019857
:10CE80008668002C01D10020FEBD01212046FFF75D
:10CE9000B6F80546002D0FD1F6E700004CC400108F
:10CEA00066616C73650000007472756500000000B7
:10CEB000BC300020C43000205B202870A068401CDB
:10CEC000A060E068401CE0602AE02146304600F0A7
:10CED0003BF8002800D1D7E72046FFF70CF930686F
:10CEE00000281CD06069002801D0022000E0012049
:10CEF0000746791C2046FFF782F80546002D00D131
:10CF0000C2E72C2028706D1C6069002802D0202008
:10CF100028706D1C00202870A068C019A0603668B9
:10CF2000002ED2D102212046FFF769F80546002DD8
:10CF300000D1A9E75D2028706D1C00202870E068F2
:10CF4000401EE06001209FE7F8B504460E4600252C
:10CF5000002C01D0002E01D10020F8BD207B10282C
:10CF600058D008DC01281BD0022827D0042809D07B
:10CF700008285ED131E0202851D0402854D08028A4
:10CF800057D12FE005213046FFF739F80546002D2F
:10CF900000D1E2E7F849284606F0E8FD0120DCE789
:10CFA00006213046FFF72BF80546002D00D1D4E7C7
:10CFB000F249284606F0DAFD0120CEE70521304689
:10CFC000FFF71DF80546002D00D1C6E7EB490831F3
:10CFD000284606F0CBFD0120BFE731462046FFF78B
:10CFE000D8F8BAE700272069002800D1B5E7206902
:10CFF00006F09AFD471C39463046FFF700F8054613
:10D00000002D00D1A9E73A462846216906F068FDBF
:10D010000120A2E731462046FFF7B0FB9DE73146ED
:10D020002046FFF727FF98E731462046FFF75CFED2
:10D0300093E7002091E7F0B589B007460E46144605
:10D0400000252421684606F064FDFF200130216898
:10D0500088470090FF20013001900596204607C8C0
:10D0600006AB07C30098002800D137E06946384670
:10D07000FFF76AFF002800D130E06846FFF73BF871
:10D08000A06800280BD0029B591C0098A26890470A
:10D090000546002D00D121E0002000901BE0029AFF
:10D0A000501C216888470546002D00D116E00298E3
:10D0B000401C019B834201D2019801E00298401C70
:10D0C00002462846009906F00BFD0020029968549C
:10D0D000009861688847284609B0F0BD009800288C
:10D0E00002D0009861688847002D02D02846616808
:10D0F00088470020F0E710B50446A14A01212046E8
:10D10000FFF799FF10BD10B504469D4A0021204647
:10D11000FFF791FF10BD70B58AB006460C46154664
:10D12000242101A806F0F5FC002C02DA00200AB048
:10D1300070BD9348016820468847019001980028F7
:10D1400000D1F4E7029400200390059006958C4AE4
:10D1500007CA07AB07C301A93046FFF7F5FE002851
:10D1600005D1874A0198516888470020DFE7019878
:10D17000DDE7F0B589B007460C4615461E4624216A
:10D18000684606F0C6FC002D01DB002C02D1002011
:10D1900009B0F0BD00940195002002900120049098
:10D1A0000596774A07CA06AB07C369463846FFF7B4
:10D1B000CBFEEDE7014600220023002900D1704795
:10D1C0008A6801E05B1C1268002AFBD11846F6E76A
:10D1D00002460B460021002A00D17047916801E009
:10D1E0005B1E0968002901D0002BF9D10846F4E73D
:10D1F00070B505460C46002C01DA002070BD2146B2
:10D200002846FFF7E5FFF9E7F8B505460E4617464D
:10D210000024002D01D0002E01D10020F8BDAC6803
:10D22000002F0DD000E02468002C13D0206A0028C5
:10D2300010D03046216A06F07EFC0028F3D109E0C8
:10D2400000E02468002C05D03046216AFEF739FD45
:10D250000028F6D1002C02D0206A002801D100203D
:10D26000DCE72046DAE770B504460D460022294681
:10D270002046FFF7C9FF70BD70B504460D46012278
:10D2800029462046FFF7C0FF70BD70B504460D4625
:10D2900029462046FFF7E7FF002801D0012070BD96
:10D2A0000020FCE701604860704770B505460E46F7
:10D2B0000024002D00D170BD3046FEF76EFD0446FF
:10D2C000002C00D1F7E728222946204606F008FC6A
:10D2D00000202062FF210131E0680843E060002067
:10D2E000606020602046E6E770B505460C460026E3
:10D2F000002C03D0002D01D0A54201D1002070BD2B
:10D30000AE68002E04D1AC6064600020206008E0AC
:10D310007068002805D021467068FFF7C3FFA86831
:10D3200044600120EBE770B504460D4629462046CF
:10D33000FFF7DAFF70BD7047FEB505460E4614468E
:10D340001F46002001900090002D05D0002E03D034
:10D35000002C01D0A54201D10020FEBD0898002874
:10D3600010D03046FFF7E7FF019001214902E06845
:10D370000843009014E000004CC40010A0CE001040
:10D38000C430002039463046FEF7C1FC01900198B8
:10D39000002800D1E1E701214902E06888430090BC
:10D3A00001214902E0680840002805D1206A0028D0
:10D3B00002D0206A79688847019820620098E0606E
:10D3C00021462846FFF790FFC7E7F8B504460D460B
:10D3D00016460020FB4B3246294600902046FFF7B8
:10D3E000ABFFF8BDF8B504460D4616460120F54BD7
:10D3F0003246294600902046FFF79EFFF8BD70B5E3
:10D4000004460D46002C00D170BDEE492846FFF7BA
:10D410004CFF064631462046FFF766FFF4E7F8B5B5
:10D4200004460D461646002C01D0002D01D10020E7
:10D43000F8BDE4493046FFF738FF07460020E14BCE
:10D440003A46294600902046FFF776FFF0E710B5F0
:10D45000DC48FEF7A2FC0446002C01D00420E0606A
:10D46000204610BDF8B504460D46FFF7F0FF06460E
:10D470000020D44B3246294600902046FFF75CFF3F
:10D48000002801D03046F8BD3046FEF794FC00205D
:10D49000F9E710B5CB48FEF780FC0446002C01D01C
:10D4A0000220E060204610BDF8B504460D46FFF7A7
:10D4B000F0FF06460020C34B324629460090204626
:10D4C000FFF73AFF002801D03046F8BD3046FEF79E
:10D4D00072FC0020F9E710B5BA48FEF75EFC04467E
:10D4E000002C01D00120E060204610BDF8B50446B4
:10D4F0000D46FFF7F0FF06460020B24B32462946A4
:10D5000000902046FFF718FF002801D03046F8BDF4
:10D510003046FEF750FC0020F9E770B50546A948F3
:10D52000FEF73BFC0446002C05D0002D01D0022064
:10D5300000E00120E060204670BDF8B505460E46CB
:10D5400014462046FFF7E9FF074600209D4B3A4668
:10D55000314600902846FFF7EFFE002801D03846FC
:10D56000F8BD3846FEF727FC0020F9E770B5054600
:10D570000E469448FEF711FC0446002C1DD00820EE
:10D58000E060E661A561904A904B2846314607F07D
:10D590000FF802D88E4860610FE000228D4B2846BC
:10D5A000314606F0F1FF03D80120C007606104E0B6
:10D5B0002846314606F092FF6061204670BDFEB5F8
:10D5C00006460F4614461D4620462946FFF7CEFF65
:10D5D000019000207B4B009039463046019AFFF7BE
:10D5E000ABFE002801D00198FEBD0198FEF7E3FBD9
:10D5F0000020F9E770B505467248FEF7CEFB0446F9
:10D60000002C0ED01020E0606E492846FEF77FFB0C
:10D6100020612069002804D12046FEF7CCFB0020C1
:10D6200070BD2046FCE7F8B505460E461446204678
:10D63000FFF7E0FF07460020624B3A463146009074
:10D640002846FFF779FE002801D03846F8BD384655
:10D65000FEF7B1FB0020F9E770B505465948FEF723
:10D660009CFB0446002C0ED08020E06055492846E3
:10D67000FEF74DFB20612069002804D12046FEF70B
:10D680009AFB002070BD2046FCE7F8B505460E4623
:10D6900014462046FFF7E0FF07460020494B3A4674
:10D6A000314600902846FFF747FE002801D0384653
:10D6B000F8BD3846FEF77FFB0020F9E710B541487A
:10D6C000FEF76BFB0446002C01D04020E0602046B2
:10D6D00010BDF8B504460D46FFF7F0FF06460020E2
:10D6E000384B3246294600902046FFF725FE002899
:10D6F00001D03046F8BD3046FEF75DFB0020F9E76B
:10D7000010B53048FEF749FB0446002C01D020201C
:10D71000E060204610BDF8B504460D46FFF7F0FF67
:10D7200006460020274B3246294600902046FFF748
:10D7300003FE002801D03046F8BD3046FEF73BFB23
:10D740000020F9E70246002A01D0002901D100207B
:10D7500070479068884202D04B6808681860086873
:10D76000002802D00B68486858609068884202D14F
:10D770000868906005E00868002802D1486893684E
:10D7800058600020486008600846E1E770B505462B
:10D790000C46002C01DA002070BD21462846FFF718
:10D7A00017FD064631462846FFF7CCFFF4E770B573
:10D7B00004460D4629462046FFF7E8FF0646FEF7D9
:10D7C000FAFA70BDC43000200000C0FFFFFFDF4147
:10D7D000FFFFFF7F0000E0C170B504460D462946FB
:10D7E0002046FFF740FD064631462046FFF7AAFFD8
:10D7F00070BD70B504460D4629462046FFF73CFD36
:10D80000064631462046FFF79DFF70BD70B50446C1
:10D810000D4629462046FFF7DFFF0646FEF7CBFA06
:10D8200070BD70B504460D4629462046FFF7E1FF5E
:10D830000646FEF7C0FA70BDF8B506460F46144618
:10D840000025002F01DA0020F8BD39463046FFF7E9
:10D85000BFFC0546002D04D121463046FFF744FDAC
:10D86000F2E72560686860606C60B068A84201D12A
:10D87000B46001E0606804600120E5E770B5064629
:10D880000D461446002E03D0002C01D0002D01D1EE
:10D89000002070BDAC4201D10120FAE72868206069
:10D8A000686860602068002801D020684460B06823
:10D8B000A84207D1B0684068B168884200D164606E
:10D8C000B46009E06068002801D0606804602068E6
:10D8D000002801D1B06844600020286068602846B4
:10D8E000FEF769FA0120D4E7F8B505460C4616465E
:10D8F000002C01DA0020F8BD21462846FFF768FC1D
:10D900000746324639462846FFF7B8FFF3E7F8B531
:10D9100007460D4614461E46002C01D0002D01D1AD
:10D920000020F8BD01214902E0680840002805D127
:10D93000206A002802D0206AFEF72AFBF749284611
:10D94000FEF7E5F9206201214902E0688843E060C2
:10D95000324629463846FFF757FC224601460090DA
:10D960003846FFF78BFFDCE770B504460D461646D8
:10D970000023324629462046FFF7C9FF70BD70B527
:10D9800004460D4616460123324629462046FFF737
:10D99000BEFF70BD70B50546E048FEF7FEF90446CF
:10D9A000002C06D0FF201130E0602846FFF7C3FCB2
:10D9B0002061204670BD70B50546D848FEF7EDF9E8
:10D9C0000446002C06D0FF204130E0602846FFF7D7
:10D9D000B2FCA060204670BD70B50546CF48FEF78A
:10D9E000DCF90446002C06D0FF202130E0602846F8
:10D9F000FFF7A1FCA060204670BDF3B583B00746D9
:10DA0000002600250020029000240498002801DB55
:10DA1000002F02D1002005B0F0BDFFF771FE0446D3
:10DA2000002619E0B100785806F01CFD0191009025
:10DA3000FFF79CFD0546002D04D12046FEF7BBF9FB
:10DA40000020E8E7002E01D1A56003E029460298F6
:10DA5000FFF728FC0295761C002C02D00498864221
:10DA6000E0D3002C04D0A068002801D0A068456055
:10DA70002046D0E7F3B583B00746002600250020F6
:10DA8000029000240498002801DB002F02D100201E
:10DA900005B0F0BDFFF734FE0446002619E0B100E2
:10DAA000785806F05DFD01910090FFF75FFD054697
:10DAB000002D04D12046FEF77EF90020E8E7002E75
:10DAC00001D1A56003E029460298FFF7EBFB029520
:10DAD000761C002C02D004988642E0D3002C04D09F
:10DAE000A068002801D0A06845602046D0E7F3B5C3
:10DAF00081B00746002600250020009000240298EF
:10DB0000002801DB002F01D10020FEBDFFF7F8FD4A
:10DB10000446002618E0F00039180A6849681046E3
:10DB2000FFF724FD0546002D04D12046FEF743F9FA
:10DB30000020EAE7002E01D1A56003E02946009805
:10DB4000FFF7B0FB0095761C002C02D002988642AD
:10DB5000E1D3002C04D0A068002801D0A068456063
:10DB60002046D2E7F3B581B0074600260025002005
:10DB7000009000240298002801DB002F01D1002032
:10DB8000FEBDFFF7BDFD0446002615E0B100785844
:10DB9000FFF730FD0546002D04D12046FEF70BF9B6
:10DBA0000020EDE7002E01D1A56003E02946009892
:10DBB000FFF778FB0095761C002C02D00298864275
:10DBC000E4D3002C04D0A068002801D0A0684560F0
:10DBD0002046D5E7F3B581B0054600240027002094
:10DBE00000900026002D00D157E04C48FEF7D5F8F4
:10DBF0000446002C00D150E0FF210131E868884341
:10DC0000E06068696061E969A869E161A06128690B
:10DC1000002808D041492869FEF779F82061206979
:10DC2000002800D139E0286A002810D001214902DB
:10DC3000E8680840002801D0286A03E03749286ACC
:10DC4000FEF765F82062206A002800D125E00298DE
:10DC5000002801D12046FEBDAF6813E001213846FF
:10DC6000FFF7B8FF0646002E00D116E00098002806
:10DC700005D00098066000987060009601E0A660EC
:10DC800000963F68002FE9D1002C04D0A06800283E
:10DC900001D0A06846602046DDE7002C02D0204677
:10DCA000FEF789F80020D6E70168891C01600AE0C8
:10DCB000016809780A2903D10168491C016070478D
:10DCC0000168491C0160016809780029F0D100BF92
:10DCD000F5E70168891C01600EE0016809782A29CE
:10DCE00007D1016849782F2903D10168891C016097
:10DCF00070470168491C0160016809780029ECD16E
:10DD000000BFF5E7026812780B681A700268521CAF
:10DD100002600A68521C0A602BE00000C430002038
:10DD2000026812780B681A7002681278222A08D1E9
:10DD30000B681A700268521C02600A68521C0A6062
:10DD40007047026812785C2A0DD102685278222A44
:10DD500009D1026852780B685A700268521C02603E
:10DD60000A68521C0A600268521C02600A68521C4F
:10DD70000A6002681278002AD2D100BFE0E701B53C
:10DD800082B0029801900298002800D10EBD3CE0BC
:10DD90000298007820280CD006DC09280AD00A282E
:10DDA0000AD00D2825D106E022281DD02F2820D109
:10DDB00006E000BF00BF00BF0298401C029023E0B5
:10DDC000029840782F2803D102A8FFF76DFF0AE0E0
:10DDD000029840782A2803D102A8FFF77AFF02E0D0
:10DDE0000298401C02900FE001A902A8FFF78AFFE9
:10DDF0000AE002980078019908700298401C02908D
:10DE00000198401C019000BF00BF029800780028D4
:10DE1000BED10199087000BFB8E70146002900D1C2
:10DE20007047087B002801D10120F9E70020F7E7BF
:10DE30000146002900D17047087B012800D1FAE78C
:10DE40000020F8E70146002900D17047087B02282E
:10DE500001D10120F9E70020F7E70146002900D1B0
:10DE60007047087B8007800F002801D00120F7E76A
:10DE70000020F5E70146002900D17047087B0428FF
:10DE800001D10120F9E70020F7E70146002900D180
:10DE90007047087B202801D10120F9E70020F7E72F
:10DEA0000146002900D17047087B402801D101209C
:10DEB000F9E70020F7E70146002900D17047087B09
:10DEC000802801D10120F9E70020F7E7F7B582B0FB
:10DED00004460F46002C0AD0002F08D0207B397B47
:10DEE000884204D12046FFF798FF002802D0002086
:10DEF00005B0F0BD207B102814D008DC01280DD01F
:10DF000002280CD004280BD008280FD109E02028C3
:10DF10000AD0402809D0802808D104E000BF00BF03
:10DF200000BF00BF00BF00BF00BF01E00020DFE76F
:10DF300000BFBC4201D10120DAE7207B102823D0AA
:10DF400008DC01280DD002280CD004280BD00828AA
:10DF50007FD10AE020282AD040283FD0802878D1DD
:10DF600013E000BF00BF0120C2E7BD69FB69E169A2
:10DF7000A0692A4601910090FEF7D1F8002801D04F
:10DF80000120B5E70020B3E700BF2069002802D0D8
:10DF90003869002801D10020AAE73969206905F015
:10DFA000CAFD002801D10120A2E70020A0E7A56852
:10DFB000BE6809E031462846049AFFF787FF00282B
:10DFC00000D195E72D683668002D01D0002EF1D1E3
:10DFD000B54201D000208BE7012089E7002500260B
:10DFE000002C01D0A06800E00020054611E0296A5D
:10DFF0003846049AFFF708F90646002E00D177E765
:10E0000031462846049AFFF761FF002800D16FE7E8
:10E010002D68002DEBD1002F01D0B86800E0002062
:10E02000064612E0316A2046049AFFF7EDF80546ED
:10E03000002D01D15CE70CE029463046049AFFF739
:10E0400045FF002800D153E73668002EEAD10120B1
:10E050004EE700204CE710B5044602480168204610
:10E06000884710BDC430002070B503460C4600211F
:10E07000002A01D1234D00E015882846002110E038
:10E08000051206023543A8B25D5C684005062D0FF7
:10E09000684005034540A8B205062D0D6D00684097
:10E0A000491CA142ECD370BD30B502460B46154861
:10E0B000002110E0555C6840002409E0C507ED0F21
:10E0C000002D03D04010104D684000E04010641C4B
:10E0D000082CF3D3491C9942ECD330BD30B502462D
:10E0E000002000230BE01478521C05126C4024061B
:10E0F000E40D064D2C5B05026C40A0B25B1C8B420C
:10E10000F1DB30BDFFFF000001A00000D05801107E
:10E1100001460A4600E0521C10780028FBD1501A34
:10E12000704730B503460C46002107E0585C655C3B
:10E13000A84201D0002030BD481CC1B29142F5DB9D
:10E140000120F8E710B5002819DBFE4A03231B0263
:10E15000D21883089B00D2588307DC0EFF23A3400C
:10E160009A438B071B0E8407E40EA3401A43F54B1A
:10E17000032424021B198408A4001A5118E0F24A4F
:10E1800003071B0F083B9B089B00D2588307DC0E3C
:10E19000FF23A3409A438B071B0E8407E40EA34082
:10E1A0001A43E94B0407240F083CA408A4001A51A1
:10E1B00010BD0EB572B6F3F7EEFFFF200130F2F797
:10E1C0007DFB0121684601700021C1700171417021
:10E1D00001218170C11D202005F0EAFC684603F092
:10E1E000AEFE03F0F1FE0520F2F7D6F962B60EBDE1
:10E1F0003EB504460D46D5480078C007C00F00283C
:10E2000010D01F21C94368460180891C4180182114
:10E2100081800121018123462A466946012003F0BD
:10E2200065FD3EBD0020FCE710B5C9480088401CD4
:10E23000C7490880C7480068C6494968884208D16C
:10E24000C3480088032804DD0020C349087005F096
:10E2500074F810BDF0B585B0BE4806684468A642A3
:10E260000ED0BD48007800280CD10120BA490870B2
:10E270000020B7490880B949A32005F02EF801E035
:10E2800005B0F0BDA64201D3351B02E03046803018
:10E29000051B142D3AD31CE00020AD49088000274F
:10E2A0000AE02046641CAE49085C6946C855802CCB
:10E2B00000D30024781CC7B2142FF2DB1421684667
:10E2C000FFF796FF002802D0A248446000E002E079
:10E2D000143D142DE0D200BF002D38D000270AE0F5
:10E2E0002046641C9E49085C6946C855802C00D3B2
:10E2F0000024781CC7B2AF42F2D3E9B26846FFF7F8
:10E3000077FF002801D09348446020E0002D1ED004
:10E310008F48008803281ADB00270AE02046641C87
:10E320008F49085C6946C855802C00D30024781CAE
:10E33000C7B2AF42F2D3E9B26846FFF759FF0028EF
:10E3400001D08448446000208149088000BF00BF9C
:10E3500096E710B58348007801281CD1F3F710FD2B
:10E3600081484088002812D17F480089401C7E499E
:10E37000088108460089142835DB0846807A002881
:10E3800031D108810120887203F062FA2BE000206D
:10E390007549088127E0F3F7F9FC6E4840686D493C
:10E3A00008602020F2F7D5FA20210840002803D089
:10E3B00000206D49088104E06B480089401C6A49CF
:10E3C000088169480089142802DB012066498872A7
:10E3D0006548807A012806D164480078002802D177
:10E3E00001206149C87210BD3EB50446002C02D020
:10E3F000012C11D107E010216846C180C82141815C
:10E400000021018108E010216846C180FF2191317F
:10E4100041810121018100BF00BFC0216846017117
:10E420000421417101A803F0C3FF00BF6846408981
:10E43000009068460389C2884DA1002002F0F2F8DE
:10E4400000BF3EBD10B556480078401C54490870C6
:10E4500008460078032808DB00203F4908700120A7
:10E46000FFF7C2FF012004F0E8FD10BD10B54D48D4
:10E47000007800284BD04B480078012804D00228AF
:10E4800017D0032841D127E000BF47A1002002F0A8
:10E49000C9F800BFF3F797F800BF47A1002002F0CA
:10E4A000C1F800BF02203F490870002045490870AC
:10E4B0002CE044480078401C424908700846007827
:10E4C000202808DD00BF40A1002002F0ABF800BF0B
:10E4D000022004F0B2FD19E0002032490870022049
:10E4E00004F0ABFD00BF3BA1002002F09BF800BF91
:10E4F0007D20C000F2F750F800BF3AA1002002F0E2
:10E5000091F800BF03F0A6FD00E000BF00BF10BD02
:10E5100010B539480068002870D0374800680221DB
:10E520000840002804D0FFF7A1FF022004F0E1FD1D
:10E5300031480078C007C00F002862D0FFF782FF83
:10E5400001205CE000E100E01CED00E0FF30002075
:10E55000FC300020A4360020FA30002029E2001010
:10E56000A4320020F830002088320020F93000204A
:10E57000736D6172745F706172616D7320696E7426
:10E58000657276616C3A2578206C6174656E63798A
:10E590003A2578207376746F3A25780D0A000000CA
:10E5A000FE3000207830002073746172742046774A
:10E5B00045726173650D0A004F5441207374617296
:10E5C000740D0A00793000204F5441206661696C57
:10E5D000650D0A004F54412066696E6973680D0A23
:10E5E00000000000537461727420526573657420DA
:10E5F00031303030730D0A009431002015E004F002
:10E6000078FDFE48006804210840002804D0FFF788
:10E61000A0FE042004F06DFDF848006810210840B9
:10E62000002802D0102004F064FD10BDFEB50025C6
:10E6300000260027002001900090FC21F04800688F
:10E6400020300170FF21EE48006820304170EC4816
:10E65000006820308170C721E94800682030C1700F
:10E66000FF21E748006820300171002434E0052CC8
:10E6700015D004DC002C07D0012C23D105E0082C98
:10E6800004D0152C1ED116E000BF22E00120A040CE
:10E6900007430121A14001988843019019E001201E
:10E6A000A04005430120A04006430120A04000995E
:10E6B000084300900DE00120A04005430120A04048
:10E6C000064306E00120A04005430120A040064388
:10E6D00000BF00BF601CC4B2202CC8DB00217F201B
:10E6E00002F099FB40211A2002F095FB3846F2F720
:10E6F0001DF839460020F1F7CFFF3A4601998A43C9
:10E700001046F2F7DBF80198F2F7F1F82846009985
:10E71000F2F725F831460020F1F773FFFEBD10B582
:10E7200002210120FFF70EFD02210846FFF70AFD36
:10E7300002210320FFF706FD02210420FFF702FD5E
:10E7400002210520FFF7FEFC02210620FFF7FAFC5C
:10E7500002210720FFF7F6FC02210820FFF7F2FC58
:10E7600002210920FFF7EEFC02210A20FFF7EAFC54
:10E7700002210B20FFF7E6FC02210C20FFF7E2FC50
:10E7800002210D20FFF7DEFC02210E20FFF7DAFC4C
:10E7900000210F20FFF7D6FC02211020FFF7D2FC4A
:10E7A00002211120FFF7CEFC02211220FFF7CAFC44
:10E7B00002211320FFF7C6FC02211420FFF7C2FC40
:10E7C00002211520FFF7BEFC02211620FFF7BAFC3C
:10E7D00002211720FFF7B6FC10BD1FB500216846C7
:10E7E000017007214172502141810A21818103F08A
:10E7F0004CF8844803F037F882488079824948729F
:10E800008048407988727F480079C8727D48C07816
:10E8100008737C48807848737A48407888737948D0
:10E82000807800117949085C774948767548807886
:10E830000007000F7549085C734988767148407875
:10E8400000117249085C7049C8766E48407800072C
:10E85000000F6E49085C6C4908770846407E6C4999
:10E8600008726948807E48726748C07E8872664830
:10E87000007FC8720B23674A1D21634803F00BF821
:10E880000120654908751FBD10B502F0E7FA10BDFB
:10E8900013B584B06846408A15214902884205D1E3
:10E8A0000C245B49204603F012FA4FE06846408A88
:10E8B0005A49884204D15AA1052003F008FA45E0DC
:10E8C0006846408A5549491F884204D156A109200B
:10E8D00003F0FDF93AE06846408A5049091F884232
:10E8E00004D154A1112003F0F2F92FE06846408AC8
:10E8F0004A49891E884204D153A1072003F0E7F951
:10E9000024E06846408A4549491E884204D150A106
:10E91000072003F0DCF919E06846408A3F491039C6
:10E92000884213D06846408A4B4988420ED1002164
:10E93000039100200190029003A901A8F3F757F971
:10E9400001A96846007B03F0C2F900BF06B010BD04
:10E950000FB410B5684640893F49E03188422FD056
:10E9600068464089891C884246D100BF6846837B3F
:10E9700003AA033239A1002001F066FE00BF6846F9
:10E98000807B022839DB6846C07B402835D1684649
:10E99000807B401E03A90331085C23282DD16846E3
:10E9A000807B06280DD1062230A103A80330FFF793
:10E9B000B8FB002805D000BF2EA1002001F032FED8
:10E9C0007FE06846807B052807D105222BA103A89C
:10E9D0000330FFF7A6FB002873D16846807B05282B
:10E9E0006FD1052227A103A80330FFF79AFB002867
:10E9F00067D0012025494BE059E052E094310020D6
:10EA000008300020D030002008310020E330002002
:10EA1000D73000202531002000000240292A0000C4
:10EA20004C7662750000000042443153342D303280
:10EA3000000000005359443450314D4244313234C7
:10EA4000313233310000000056322E302E300000BB
:10EA500056312E302E30000001FF0000424C455F41
:10EA600043544C5F555549443A00000040544553C7
:10EA700054230000404F4B230D0A0000404F4646F0
:10EA8000230000004043414C230000008832002056
:10EA9000C87100BF0846C279F3A1002001F0C2FD91
:10EAA0000FE000BFF6A1002001F0BCFD09E06846C0
:10EAB0004089F749884204D16846817B0F30F2F7DC
:10EAC0008DFE10BC08BC04B0184730B58DB00446AC
:10EAD000601C05F063F80121490288420FD10E2223
:10EAE00021461531684604F0FBFF1E22611D05A872
:10EAF00004F0F6FF05A80FC8FFF72AFF6FE1601CBE
:10EB000005F04CF8FF210131884209D10822611D2E
:10EB10000BA804F0E5FF0C990B98FFF7B9FE5EE136
:10EB2000601C05F03BF8022817D10120D949087074
:10EB30000020D94908818872D8490870012004F062
:10EB4000DDFA00BF0623A21DD5A1002001F07CFD47
:10EB500000BF0120F2F72FFE41E1601C05F01EF816
:10EB6000042838D100BF6279D1A1002001F05AFDFC
:10EB700000BFD648007840084000D4490870002003
:10EB8000C4490870C4490881022004F047FB0028EA
:10EB900006D0CF480078032802D0022004F04DFAB6
:10EBA000BD48807A00280CD1FFF717FE02F090FFD5
:10EBB0000120C849087000BFC7A1002001F032FD44
:10EBC0000DE1FFF761FE0020C249087000BFC8A137
:10EBD00001F028FD03E1601C04F0E0FF012149037E
:10EBE000884277D100BFA17A627A08021043009070
:10EBF000217AE579080228430346A179657908025C
:10EC000028430246BFA1002001F00CFD00BFA179FE
:10EC10006279080210439E49DF3188429CD1A17A73
:10EC2000627A0802104301283ED1217AE279080273
:10EC30001043192804D01C2812D01F2832D120E0FC
:10EC4000A248007801210843A0490870B8484168EB
:10EC5000016000BFB7A1002001F0E4FC00BF22E08A
:10EC60009A4800780221084398490870B0484068E3
:10EC7000AF49086000BFB5A1002001F0D3FC00BF80
:10EC800011E0924800780321084390490870A84891
:10EC90004068A749086000BFB2A1002001F0C2FC93
:10ECA00000BF00E000BF9AE0217AE2790802104339
:10ECB000192804D01C2814D01F282CD11EE083480A
:10ECC00000784008400081490870002002F0CBF82D
:10ECD00000BF00E021E0A9A1002001F0A3FC00BFDB
:10ECE0001AE07A480078022188437849087000BF0A
:10ECF000A8A1002001F096FC00BF0DE07348007849
:10ED0000800880007149087000BFA8A1002001F0B0
:10ED100089FC00BF00E000BF61E0601C04F03EFF22
:10ED20000121C903884223D1A179627908021043E5
:10ED3000030006F086F806041718191A1B1C00BFFA
:10ED4000A0A1002001F06EFC00BF0BA802F089FF1B
:10ED500000BF6846C38D828DA0A1002001F062FC37
:10ED600000BF04E003E002E001E000E000BF36E0A5
:10ED7000601C04F013FF0121090488420FD10BA885
:10ED800002F06FFF00BF6846008E00906846C38D9A
:10ED9000828D99A1002001F045FC00BF1FE0601C9E
:10EDA00004F0FCFE01281AD100BF9BA1002001F055
:10EDB00039FC00BF3848807A002805D102F088FE6F
:10EDC00001204449087004E0FFF75EFD002041493E
:10EDD000087000BF95A1002001F024FC00BF0DB019
:10EDE00030BD00B587B002F085FC012002F03FFF86
:10EDF000924802F067FF03216846017300214173C6
:10EE0000807B81088900491C68468173807B0421CE
:10EE100088430146684681731021C1730021017443
:10EE20000321417403A802F010FFC020059084481C
:10EE3000069005A802F02BFF002003F01BF9FFF756
:10EE4000CCFC002168460170C17001710121417044
:10EE500000218170C11D202004F0AAFE684603F045
:10EE60006EF807B000BD00005041532E61646A7512
:10EE70007374466C6167203D2025640D0A00000014
:10EE8000404552524F5220636D64230D0A0000002A
:10EE900001FF0000F830002088320020FE30002002
:10EEA000436F6E6E656374656420616464723A00DA
:10EEB000446973636F6E6E65637465642C72657309
:10EEC0006F6E3A3078253032780D0A00FF3000201E
:10EED00078300020F93000207265737461727420FC
:10EEE00061647620402064697363210D0A0000008C
:10EEF00073746F70206164762040206469736321AD
:10EF00000D0A00004741505F4556545F4154545F1D
:10EF100048414E444C455F434F4E46494755524544
:10EF20003D202532782C2532782C2532780D0A00A8
:10EF3000A4360020525050206E6F746966792045C7
:10EF40006E61626C6564210D0A00000043544C2020
:10EF50006E6F7469667920456E61626C6564210D1F
:10EF60000A000000424154206E6F746966792045A2
:10EF70006E61626C6564210D0A00000052505020E1
:10EF80006E6F746966792044697361626C6564218F
:10EF90000D0A000043544C206E6F7469667920445A
:10EFA000697361626C6564210D0A0000424154205E
:10EFB0006E6F746966792044697361626C6564215F
:10EFC0000D0A0000757064617465207273702041D1
:10EFD000434345505445440D0A000000696E746572
:10EFE0007276616C3A2578206C6174656E63793A4B
:10EFF00025780D0A00000000434F4E4E5F555044E7
:10F000004154455F434F4D503A2025642C202564E0
:10F010002C2025640D0A00004741505F4556545F7F
:10F020004144565F454E440D0A00000072657374FA
:10F03000617274206164760D0A000000F4300020D3
:10F04000CBEA001072B6FFF7CCFEFFF768FB00209A
:10F0500002F065FF01F0E2FE012001F098FF00F0F0
:10F060009DFF002001F0FFFE00BFF3A3F5A2F8A171
:10F07000002001F0D7FA00BFFFF7D8FAFC490420BE
:10F0800004F0DDF8F2F75EFA042004F037F802200D
:10F0900004F034F800F086FAF2F78EFFF2F770FE13
:10F0A000F2F7EFFE02F014FD0120F249087062B69B
:10F0B00019E003F023F9FFF72BFAEF480078C007B7
:10F0C000C00F002801D0FFF7C5F8EC480078C00752
:10F0D000C00F002801D102F06DFFE948C07A012875
:10F0E00001D1FFF766F8E4E70EB51F21C943684672
:10F0F0000180E44941801E21818001210181E04B92
:10F100005B1C01226946104602F0F0FD0EBD00288E
:10F1100007D001220A43D94B1B781A43D74B1A70E8
:10F1200010E0D64A12788A43D44B1A701A461278E5
:10F13000D54B1A40002A05D1D04A12785208520005
:10F14000CE4B1A707047F0B587B0064600BF324606
:10F15000CEA1002001F066FA00BFCB48401C8642D9
:10F160007ED000200690304605F075F9074605F080
:10F17000F7F9CB4ACB4B0391029005F081F8044696
:10F180000022C94B05F0E4F80591049005F024FA3B
:10F1900006908121C905069804F045FFC3490390F4
:10F1A00004F07EFF074605F0DBF9C14AC14B05912B
:10F1B000049004F0B3FF044605F00EFA069000BF79
:10F1C000069805F0CDF9044622460B46BAA1002068
:10F1D00001F028FA00BFBC49069804F024FFBB499F
:10F1E000019004F018FF074605F0BAF90446002222
:10F1F000B74B05F0ADF80022B64B0391029004F036
:10F200008DFF0591049005F069F9B349086008463F
:10F210000068002801DA00200860AF480068642810
:10F2200002DD6420AC490860AC480078401CAB4962
:10F23000087008460078022801DB00200870A64804
:10F240000078A749A54A127888540846007849787A
:10F25000884203D08A484078002805D19E4800E0C3
:10F2600012E000788649487000BF069805F078F9EA
:10F2700004469948006822460B469AA10090002057
:10F2800001F0D0F900BF05E000BF9DA1002001F012
:10F29000C9F900BF02210020FFF739FF07B0F0BD18
:10F2A00010B50620F1F76EFE9A48F2F797F80221A2
:10F2B0000120FFF72CFF98480078002801D0FFF7C5
:10F2C00013FF012010BD10B59448006800280ED02F
:10F2D00092480078C007C00F002808D000BF90A156
:10F2E000002001F09FF900BF012004F0F7F910BDE4
:10F2F000FFB587B000270020059004900024FEF79A
:10F30000DDF90590079805F0ADF802460B4601912E
:10F31000009087A10598FEF752F9089805F0A2F829
:10F3200002460B460191009082A10598FEF747F92D
:10F33000099805F097F802460B46019100907EA1CE
:10F340000598FEF73CF9FEF7B9F904907BA1049A01
:10F350000598FEF73AF8109805F084F802460B4637
:10F36000019100900A990498FEF729F9129805F086
:10F3700079F802460B460191009011990498FEF726
:10F380001EF90598FDF7B7FE03900398FEF7F7FC0A
:10F390000398FEF7BDFE06B2701D05F091FD05460F
:10F3A0007F222146641C6A542146641C6E54FF204F
:10F3B0000002304002122146641C6A542819324669
:10F3C000039904F08DFBA01904B221462846FEF7EC
:10F3D00085FE00B202900298C2B22046611C0CB2B7
:10F3E0002A54FF2109020298084002122046611C9B
:10F3F0000CB22A5400BF11E0E85D51490968514A36
:10F4000050544F480068401C4D4908600846006849
:10F41000802802D300214A4801607F1CA742EBDB11
:10F42000284605F01BFD0398FCF7B2FD0598FCF794
:10F43000C2FC0BB0F0BD000031373A34323A3135FE
:10F44000000000004A616E20313420323032350035
:10F4500053594438383131204750494F207465732F
:10F46000742064656D6F2025733A25730D0A0000C2
:10F47000D4310020F9300020FF300020003100207E
:10F4800088320020192A0000FEFF000062617474B7
:10F49000657279206164633A253034782000000079
:10F4A000CDCCCCCCCCCC0C400000904000004040F7
:10F4B0007B14AE47E17AA43F70696E5F766F6C3A59
:10F4C00025342E336620000000007A4400803B453E
:10F4D000000027400000E03F0431002030310020D0
:10F4E000313100206261745F766F6C3A25342E33BF
:10F4F00066206C6576656C3A25640D0A0000000094
:10F50000626174746572792061646320457272204F
:10F510000D0A000047F10010F8300020AC31002047
:10F520005254434556545F313835530D0A0000009C
:10F530004D000000530000004600000044000000A1
:10F54000A4360020A43200200EB50B480078C00776
:10F55000C00F00280ED00948407809A2074B0221AD
:10F56000595E08A301920091029004220021032019
:10F57000FFF7BEFE0EBD0000FF30002088320020E5
:10F58000353000003431000010B5F2F7F5FB10BD46
:10F5900010B5F2F779FBF2F783FBF2F78EFBF2F787
:10F5A000C2FB10BD10B5FFF7F3FFFFF7EDFF10BD75
:10F5B00010B5F2F7F3FB10BD10B511480078012823
:10F5C00001D1F2F76CFDFFF7BFFF10BD10B50D487C
:10F5D0000068182141180A7810464A781202104330
:10F5E0008A7812041043C97809060843044620208B
:10F5F0002040002802D02020F1F7ABF910BD000018
:10F60000883200201830002010B5F94C012020610C
:10F610006061F8A0A061FA49E161012189022162DB
:10F620000021A1626162E162F2A02063F549616399
:10F630001021A16300212164E1636164F2A1E01D56
:10F6400004F094FAF1A1204604F090FA2020A07171
:10F6500010BDF7B582B00446174600200190E5685A
:10F6600000BF206900900098A84203D90098401B71
:10F67000461E04E0A1680098281A401C0E1AA068D3
:10F68000401BB04201D9304601E0A068401B06464D
:10F69000BE4201D2304600E038460646616848194D
:10F6A0003246039904F01CFA0198801901900398DE
:10F6B00080190390BF1BAD19A068A84200D1002596
:10F6C000E560002FCDD1019805B0F0BDF7B582B04F
:10F6D00004461546E668A068871BAF4208D96168F2
:10F6E00088192A46039904F0FBF97019E06010E0CC
:10F6F000019761688819019A039904F0F1F9E81BF0
:10F700000190039AD1196068019A04F0E9F901980F
:10F71000E06005B0F0BD38B505460C46FF216846EF
:10F720000170BC48015D6846417002226946284666
:10F73000FFF78FFF38BD10B501460A69CB689A42C2
:10F7400004D88C68641EE41AA01801E0D41A601E64
:10F7500010BDF7B584B0174600BFA5480078002853
:10F7600001D1FFF751FF00BF182104984843A04979
:10F7700030314618059801903569F06802900020F4
:10F7800003900298854219D9B068441BBC4201D24B
:10F79000204600E038460446706841192246019828
:10F7A00004F09EF903980019039001980019019044
:10F7B0003F1B2D19B068A84200D100250298441BB8
:10F7C000BC4201D2204600E038460446002C0DD051
:10F7D000706841192246019804F082F903980019D3
:10F7E00003900198001901903F1B2D1903980028E0
:10F7F00000D03561039807B0F0BDF8B504460D465A
:10F800001646EFF310800746012080F3108800BFF2
:10F8100000BF324629462046FFF79BFF0090F8B212
:10F8200080F3108800BF00BF0098F8BDF7B582B024
:10F830000746164603980190182078436C49183102
:10F8400044182169E068884202D1A068451E0EE094
:10F850002169E068884204D22069E168401A451EA7
:10F8600005E02069E168401A401EA1684518AE42D3
:10F870000CD92069711B4018206103E02069A16840
:10F88000401A20612069A1688842F7D2E168A06827
:10F89000451A00BFB5420AD9E26861688818324645
:10F8A000019904F01DF9E0688019E06010E0E26859
:10F8B000616888182A46019904F012F901984019E4
:10F8C00001900020E060761BA068451E002EE1D16B
:10F8D00000BF05B0F0BDF7B584B01646059803909B
:10F8E000182104984843424918314418206902906D
:10F8F000E5680298A84236D8A068401E471BB74268
:10F900000AD3616848193246039904F0E9F8A81946
:10F91000E060012007B0F0BD02983F18B74231D334
:10F92000A068401B01900198B04208D9616848194D
:10F930003246039904F0D4F8A819E06011E0616838
:10F940004819019A039904F0CBF80198321A019BE7
:10F950000398C1186068009004F0C2F80198301A4A
:10F96000E0600120D6E70298401B471EB74209D34A
:10F97000616848193246039904F0B2F8A819E060AA
:10F980000120C7E70020C5E7F7B582B00746164655
:10F9900003980190182078431549183140180090B9
:10F9A00000984069002804D0012811D002283AD1DB
:10F9B00032E00098FFF7BFFE0546B54201D20024B1
:10F9C00005E03446324601990098FFF77FFE2CE0AF
:10F9D0000098FFF7B0FE0546B54201D2284600E088
:10F9E00030460446224601990098FFF76FFE1CE05E
:10F9F000AC3600205465726D696E616C00000000C9
:10FA0000F4360020F43A002052545400534547473E
:10FA10004552000033310020324601990098FFF72B
:10FA200018FE044601E0002400BF00BF204605B0D8
:10FA3000F0BDF8B504460D46164600BFFE480078F6
:10FA4000002801D1FFF7E0FD00BFEFF3108007466B
:10FA5000012080F3108800BF00BF324629462046AF
:10FA6000FFF792FF0090F8B280F3108800BF00BF4C
:10FA70000098F8BD70B505460C46204604F054F8D1
:10FA80000646324621462846FFF7D3FF70BD70B5C3
:10FA900003460C4618255D43E74E1836A919CD6874
:10FAA0006A1C8D68954200D100220D69954205D0EF
:10FAB000CE684D68AC55CA60012000E0002070BDE2
:10FAC000F3B581B0074600BFDB480078002801D1BC
:10FAD000FFF79AFD00BFEFF31080012181F310883A
:10FAE00000BF00BF18217943D34A18328C18E1684F
:10FAF0004D1CA168A94200D100252169A94206D068
:10FB00000299E3686268D154E560012600E00026AE
:10FB1000C1B281F3108800BF00BF3046FEBDF3B50F
:10FB200081B0074600BFC4480078002801D1FFF724
:10FB30006BFD00BFEFF31080012181F3108800BF3F
:10FB400000BF18217943BC4A18328C18E1684D1C5B
:10FB5000A168A94200D100256169022903D100BF33
:10FB60002169A942FCD02169A94206D00299E36823
:10FB70006268D154E560012600E00026C1B281F33D
:10FB8000108800BF00BF3046FEBD38B5012269466F
:10FB90000020FFF732FE0446012C02D168460478AB
:10FBA00001E00024E443204638BD10B500BFFFF754
:10FBB000ECFF0028FBDB10BD70B500BF9E4800784D
:10FBC000002801D1FFF720FD00BF9B48056CC06BEA
:10FBD000A84201D0012400E00024204670BD10B5E9
:10FBE000014618204843944C30340219D3681069F8
:10FBF000181A10BDFFB581B005460E46174600BF66
:10FC00008D480078002801D1FFF7FEFC00BFEFF31C
:10FC100010810846012181F3108800BF00BF002435
:10FC200000BF18216143844A30328918496800298D
:10FC300000D104E0641C80494969A142F1DC00BFA5
:10FC40007D494969A1421DDD182161437A4A30325C
:10FC500055501821614389184E6018216143891855
:10FC60008F60002218216143734B3033C9180A6139
:10FC700018216143C918CA6018226243D218049936
:10FC8000516101E00024E443C1B281F3108800BF58
:10FC900000BF204605B0F0BDFFB581B005460E4659
:10FCA000174600BF64480078002801D1FFF7ACFC7C
:10FCB00000BFEFF310810846012181F3108800BFD7
:10FCC00000BF002400BF182161435B4A1832891825
:10FCD0004968002900D104E0641C57490969A14220
:10FCE000F1DC00BF54490969A1421DDD18216143BF
:10FCF000514A183255501821614389184E60182115
:10FD0000614389188F600022182161434A4B1833E0
:10FD1000C9180A6118216143C918CA6018226243D0
:10FD2000D2180499516101E00024E443C1B281F387
:10FD3000108800BF00BF204605B0F0BDFFB581B000
:10FD400004460E46174600BF3B480078002801D104
:10FD5000FFF75AFC00BF38480069A04230D9EFF3E2
:10FD600010810846012181F3108800BF00BF002CDC
:10FD700018D018216143304A183256501821614377
:10FD800089184F60182262432B4B1833D2180499FC
:10FD90009160002218216143C9180A61182161434A
:10FDA000C918CA6018226243234B1833D2180A9923
:10FDB0005161C1B281F3108800BF00BF002501E08E
:10FDC0000025ED43284605B0F0BDFFB581B00446DF
:10FDD0000E46174600BF18480078002801D1FFF7EB
:10FDE00013FC00BF14484069A04232D9EFF31081E0
:10FDF0000846012181F3108800BF00BF002C18D0F5
:10FE0000182161430C4A3032565018216143891839
:10FE10004F6018226243084B3033D2180499916026
:10FE2000002218216143C9180A6118216143C918C9
:10FE3000CA601822624301E0AC360020BA4BD218E7
:10FE40000A995161C1B281F3108800BF00BF00253B
:10FE500001E00025ED43284605B0F0BD70B504462D
:10FE60000E4600BFB04830380078002801D1FFF7B7
:10FE7000CBFB00BFAC4830380069A04212D9EFF389
:10FE80001080012181F3108800BF00BF1821614359
:10FE9000A54A183A5650C1B281F3108800BF00BF7E
:10FEA000002501E00025ED43284670BD70B50446ED
:10FEB0000E4600BF9C4830380078002801D1FFF77B
:10FEC000A3FB00BF984830384069A04211D9EFF336
:10FED0001080012181F3108800BF00BF1821614309
:10FEE000914A5650C1B281F3108800BF00BF00256F
:10FEF00001E00025ED43284670BD70B504460E466E
:10FF000000BF894830380078002801D1FFF77CFB1A
:10FF100000BF854830380069A04213D9EFF3108044
:10FF2000012181F3108800BF00BF182161437E4A80
:10FF3000183A89184E61C1B281F3108800BF00BF22
:10FF4000002501E00025ED43284670BD70B504464C
:10FF50000E4600BF744830380078002801D1FFF702
:10FF600053FB00BF704830384069A04212D9EFF30C
:10FF70001080012181F3108800BF00BF1821614368
:10FF8000694A89184E61C1B281F3108800BF00BF71
:10FF9000002501E00025ED43284670BD10B5FFF7B0
:10FFA00033FB10BDFEB5044600BF5F483038007813
:10FFB000002801D1FFF728FB00BF0027FF2069467A
:10FFC0000871102C30DA5948005D4871564D183DC3
:10FFD000EFF310800090012080F3108800BF00BF75
:10FFE000287D8007800F022807D151480470022223
:10FFF00001A92846FFF72DFB0FE02846FFF79BFBE2
:020000041001E9
:100000000646022E07D34A480470022201A9284658
:10001000FFF75CFB01E00027FF430098C0B280F3CC
:10002000108800BF00BF01E00027FF433846FEBD37
:10003000F3B583B0074600BF3B483038007800284E
:1000400001D1FFF7E1FA00BF102F68DA36481838FF
:100050000290049803F068FD0646EFF310800190CB
:10006000012080F3108800BF00BF0298FFF763FBF8
:1000700005460298007D8007800F002804D00128E3
:1000800017D0022840D12FE0301D854201D2002434
:100090000EE039460298FFF73EFB3246049902987B
:1000A000FFF7D7FA0446224801780298FFF733FB9E
:1000B0002DE0042D02D20024E44314E039460298D6
:1000C000FFF729FB281FB04201D9304600E0281F66
:1000D000024604990298FFF7BCFA044614480178D6
:1000E0000298FFF718FB12E039460298FFF713FB5E
:1000F000324604990298FFF7ACFA04460C4801789E
:100100000298FFF708FB02E00024E44300BF00BFB1
:100110000198C0B280F3108800BF00BF01E0002446
:10012000E443204605B0F0BDDC360020333100202A
:100130004331002070B504460E46A568681C61680E
:10014000814206D320684655681CA060E068401CC8
:10015000E0606168A06888420DD1A26821682069CA
:10016000FFF767FCA168884203D00020C043E0602D
:1001700001E00020A06070BDFFB585B006461746BF
:100180001D460E9C0698029001200390019007E006
:100190003946029803F074FC02900198401C0190CB
:1001A0000298B842F4D20198854200D901950F987F
:1001B000C007C00F00281DD1002C1BD002210F98B2
:1001C0000840022804D1002D02D13020009001E027
:1001D0002020009008E0641E30460099FFF7AAFF37
:1001E000F068002800DA04E0002C02D00198A04258
:1001F000F1D300BFF068002848DB0FE0012D01D9E2
:100200006D1E08E00399069803F03AFC04900498E8
:10021000B84200D203E0039878430390EEE700BFB2
:1002200000BF0399069803F02BFC049003990498EF
:1002300048430699081A0690F74A0498115C30461C
:10024000FFF778FFF068002800DA07E039460398E6
:1002500003F016FC039003980028E2D100BF0F982A
:10026000C007C00F002811D0002C0FD008E0641E7A
:1002700020213046FFF75EFFF068002800DA04E036
:10028000002C02D00198A042F1D300BF09B0F0BD0C
:10029000FFB585B006460F460F9D0E9C002F01DA74
:1002A000784200E0384603900120049007E0079967
:1002B000039803F0FBFB03900498401C04900799FB
:1002C00003988842F3DA04990898884201D908987B
:1002D0000490002C06D0002F03DB042028400428C3
:1002E00000D1641E02202840002802D0089800286F
:1002F00015D0E807C00F002811D1002C0FD008E05E
:10030000641E20213046FFF715FFF068002800DA50
:1003100004E0002C02D00498A042F1D300BFF068A2
:1003200000283ADB002F05DA7F422D213046FFF707
:1003300001FF07E004202840042803D12B21304688
:10034000FFF7F8FEF068002827DB0220284002288B
:1003500018D1E807C00F002814D10898002811D13F
:10036000002C0FD008E0641E30213046FFF7E2FE7B
:10037000F068002800DA04E0002C02D00498A042C3
:10038000F1D300BFF068002807DB019500943946DF
:100390003046089B079AFFF7EFFE09B0F0BDF7B5AE
:1003A0009EB00D46144606A8199040201A900020D1
:1003B0001B901E981D9000201C9000BF2E786D1C75
:1003C000002E00D115E1252E72D1002701201890B2
:1003D00000BF2E78232E12D02B2E0CD02D2E02D023
:1003E000302E10D103E0012007436D1C0EE00220E7
:1003F00007436D1C0AE0042007436D1C06E008203B
:1004000007436D1C02E00020189000BF00BF189841
:100410000028DED1169000BF2E78302E01DB392E59
:1004200000DD08E06D1C0A2116984843314630393A
:1004300040181690F0E700BF002017902E782E2E5F
:1004400011D16D1C00BF2E78302E01DB392E00DD5E
:1004500008E06D1C0A21179848433146303940188E
:100460001790F0E700BF2E7800BF6C2E01D0682EE9
:1004700002D16D1C2E7800E000E0F6E700BF662E8A
:1004800052D00CDC582E40D004DC252E75D0462EE0
:1004900074D14AE0632E0CD0642EF9D116E0702E90
:1004A0006DD0732E6DD0752E1FD0782EF0D12BE02D
:1004B00097E02168081D2060086818901898C0B25D
:1004C000059019A80599FFF735FE87E02168081DFA
:1004D0002060086818901698019700900A2219A8C1
:1004E000179B1899FFF7D4FE78E02168081D20605B
:1004F000086818901698019700900A2219A8179B6F
:100500001899FFF739FE69E000BF2168081D2060D7
:1005100008681890169801970090102219A8179B48
:100520001899FFF729FE59E000BF002003900490BE
:10053000059003A802902068C01DC008C0000146B5
:100540000830206003C90191009034A103A8019BE9
:10055000009A04F04BFC00BF029806780298401CF9
:100560000290002E00D106E0314619A8FFF7E2FD07
:100570001C980028F0DA00BF30E029E02DE017E0F9
:10058000FFE72168081D20600868059000BF0598F6
:1005900006780598401C0590002E00D106E03146F3
:1005A00019A8FFF7C7FD1C980028F0DA00BF15E076
:1005B0002168081D206008681890002008210B465B
:1005C00010220091019019A81899FFF7D5FD05E0B8
:1005D000252119A8FFF7AEFD00E000BF00BF6D1C8C
:1005E00003E0314619A8FFF7A5FD1C98002800DBA1
:1005F000E4E600BF1C9800280BDD1B98002804D0FF
:1006000006A91B9A1E98FFF714FA1B991C9840180C
:100610001C901C9821B0F0BDD05A011025342E3307
:10062000660000000FB438B5044606A800906A467C
:1006300020460599FFF7B3FE0546002000902846A6
:1006400038BC08BC04B01847FFB581B00D4616464B
:100650001F460024002D03D029460198FFF7E2FF32
:1006600000241EE02046E117490F0918C910C900EF
:10067000611A04D1A2B213A10198FFF7D3FF325D32
:1006800012A10198FFF7CEFF601CC117490F09188E
:10069000C910C900411A03D10EA10198FFF7C2FF8A
:1006A000641CBC42DEDB2046E117490F0918C91063
:1006B000C900611A03D007A10198FFF7B3FF05B085
:1006C000F0BD00005B253034785D200025303278A5
:1006D000200000000D0A000004488047044800473D
:1006E000FEE7FEE7FEE7FEE7FEE7FEE7FD06011098
:1006F000C1000010034804490860704701480249DE
:10070000086070470024F40044310020F1B5F84837
:1007100080470746F74880470646F54C0120183CBD
:10072000A047F44D00200C35A847F34900988847AE
:100730003046A8473846A047F8BDF0B5EF4DF04821
:10074000E96885B00818044603F028FA2146401CE1
:1007500003F02EFA0024E9480125C668E8480C3861
:1007600031180391487C097C00020843A5402842C7
:1007700002903BD00B2060438119E1480091093081
:100780000818019003F00AFA0746DD48301803F014
:1007900005FA87422AD10F21009889014018007D6F
:1007A00000280CD0D64A00990D3A8A18517D127D46
:1007B000090211437818019903F0FAF905E002984B
:1007C0000399A8430874000A4874CD4800990D3075
:1007D000081803F0E3F9002808D0022D19D0042DE1
:1007E00017D0082D15D0102D1AD08047641CE4B204
:1007F0000A2CB0D3C148C168C1480C380918487CDC
:10080000097C00020843800501D1BE48804705B03D
:10081000F0BDBD49012088470028E7D0222005E02F
:10082000B949012088470028E0D03B20FFF76EFF40
:10083000DCE710B5B14912200969887072B6012150
:10084000B04A0320B43A904762B610BDFEB500210D
:10085000684601710170AD4F0172AD4EA74CB847AB
:10086000A07102AB6A4601A9606902F00AFA002889
:100870004ED00820B047002803D00220B0470028FF
:100880000FD068460078012811D0E0686569407A89
:1008900001283ED00228E2D19E4AA17928469047FD
:1008A000DDE7012168460170007A00282DD025215E
:1008B000E06849014118497B6569002908D09049E1
:1008C000D4314118487B097B00020843924988478C
:1008D000284602F029FA0028C1D068468D4A0179DD
:1008E0009632606990472878C0438007B7D1A878CE
:1008F0001228B4D121691320887072B60121814A6F
:100900000320B43A904762B6A9E73D20FFF7FEFE08
:10091000FEBD28780007000F0528A0D1687E297E3B
:1009200000020843062805D3687F297F0002084398
:100930000A2803D270491220884790E77349EE31A4
:10094000A81C8847287887224006C10FE068115408
:100950000622A91C883003F0C3F83721206903F070
:10096000D8F87CE7F0B5684999B00420884700289A
:100970000ED0654904201A31884762491F20AC31E6
:100980008847664880471620FFF7C0FE19B0F0BDC3
:1009900063488047002810D0584DEC68A1790807BB
:1009A000F4D5E079C2071CD05E49204698308847CC
:1009B000E868C179490849001FE0594E574F574D23
:1009C000B2361C376C46103507E06846B047012840
:1009D000DCD168460178601CB847A8470028F4D0ED
:1009E000D4E782070BD54F4A20461C328E30811C3B
:1009F0009047E868FD22C17923E0C171C6E742074C
:100A000008D5484920466031A8308847E868FB226D
:100A1000C17916E00207F726002A09DA414A214681
:100A20004232A07A0B319047E868C1793140E4E75F
:100A3000C00608D53B4968467C318847E868EF2204
:100A4000C1791140D9E720463140FF30A1712130F2
:100A5000017D0026002910D0067521460722873126
:100A60000CA803F03DF821460DA82A228E31033050
:100A700003F036F82C490CA8884701206946087015
:100A800048708E70E96800A82A2203308E3103F086
:100A900027F82D220821254C6B460020A04775E73A
:100AA00016490128896A0FD0022811D0042812D0D3
:100AB000082813D0102814D0202815D0402837D06B
:100AC000802839D0012070478878C007C00F704750
:100AD000887880072EE0887840072BE08878000728
:100AE00028E08878C00625E08878800622E00000AB
:100AF000BF650000776A0000CF1600004831002073
:100B0000CE03000001120000F50A00004957000062
:100B1000791900008B1E00002B620000BD600000F0
:100B2000054E000027260000DF470000A13E000020
:100B300088784006C00F70478878C009704710B5A4
:100B4000017801291FD1401C03F028F8FE4A102823
:100B50003AD00DDC012817D002281DD0042823D05C
:100B6000082810D1FFF79CFF00280CD1F74809E0B6
:100B7000202839D0402806D1FFF792FF002802D163
:100B8000F2485430804710BD0120FFF789FF00284C
:100B9000F9D1FFF7E7FE10BD0220FFF781FF002823
:100BA000F9D1FFF753FE10BD0420FFF779FF0028AD
:100BB000F9D1D068407A012803D00228F3D1E44863
:100BC000E0E7E348AE38DDE71020FFF769FF0028D3
:100BD000E9D1906A2030407D400701D53E2000E0F9
:100BE0000820FFF793FD10BD2020FFF759FF0028D4
:100BF000F9D1D6484830C5E770B510250826D24C43
:100C0000002821D0A06A817E31438176014660317F
:100C10000A7E637852095201DB06DB0E1A430A761C
:100C20002030427B067B1302E26833432332547C3C
:100C3000167C22023243934214D00273120A42738A
:100C4000C87D2843C8750DE002F008F8A06A0022AC
:100C5000014620310A734A736030C17D2943C17552
:100C6000BC480677012070BDB748C0682330417C7E
:100C7000027C080210430BD0B74948780A7800027A
:100C80001043032210430870000A48700120B3E7A4
:100C9000704730B4B14CA44630BC6047F8B5AE489C
:100CA000407A000663D5A848C66830462330417CA8
:100CB000007C0F02A84907434878097804020C43D6
:100CC000002F01D1600752D5A34DA87B697B00029C
:100CD0006D1C08434BD0002F49D068792979000258
:100CE00008432ED12136707C317C0002084303F08A
:100CF000CDFB00229A4B03F0C3FA03F013FC80B241
:100D00007843642102F0D2FE4004010C2971080AE4
:100D100068710A204143707D327D00021043814298
:100D200006D30A21401E02F0C1FE2871000A687134
:100D3000687929790002084303D101202871002035
:100D400068718548A10709D502218C4301210C4314
:100D50000470210A41700020FFF74EFF68792A795C
:100D6000010211437F4B00224020FFF792FFF8BDA4
:100D70001CB579494A7A002A40D04A780B78120289
:100D80001A43D3063AD44378047818022043012842
:100D900034D1C878401E0006000EC8702FD08B7862
:100DA0000846017BC47A0A022243017AC479090207
:100DB0002143C01C012B2AD0521A0272120A42721D
:100DC0001206037A120C1A43521A69460A80427AB2
:100DD000017A120612140A4369464A805E498A7BE8
:100DE000497B12020A4369468A80417B027B0802E2
:100DF00010436946C8805C49684688471CBD887AAC
:100E0000C870402002430A70100A48701CBD521876
:100E1000D3E7564A1047554A2032104738B50024C8
:100E200069460C7021467F20FFF7F5FF00213B202B
:100E3000FFF7F1FF29213B20FFF7EDFF69463B203B
:100E4000FFF7E7FF68460078800701D5012038BD2D
:100E5000641CA4B2FF2CF1D9002038BD10B5444861
:100E60008047012010BD10B53749424A88700028DC
:100E700007D1C8688078022803D00020904701205D
:100E800010BD0120FAE710B52F4C0128E1688870E9
:100E900004D0002831D0022846D073E0206B0146F0
:100EA000203002785208520002700278FD231A4066
:100EB00002700878800980011C3008704878800929
:100EC00080011C30487000217F20FFF7A4FF032120
:100ED0002120FFF7A0FF1F210320FFF79CFF022125
:100EE0007F20FFF798FF01210020FFF794FF0021EA
:100EF0007F20FFF790FF0F2141E000217F20FFF7C7
:100F00008AFF00210420FFF786FF02217F20FFF7E0
:100F100082FF00210846FFF77EFF00217F20FFF7B8
:100F20007AFF002103202BE002217F20FFF773FFCF
:100F300003210020FFF76FFF00217F20FFF76BFFE9
:100F40000021032018E0000048310020791600003D
:100F500027150000200002405B3B0020AB4400004E
:100F60000000F43F690C011033420000C56100002D
:100F700007470000A7650000FFF74DFF0021042090
:100F8000FFF749FFA078FFF76EFF012010BD10B5F5
:100F9000FFF779FF012010BD10B5F6488047F648ED
:100FA000C06A017ADF2211400172012010BDFEB536
:100FB000F2488047F04C0190E06A817A007ACF07CE
:100FC000FF0F0026C506EE49ED0E487809780002AD
:100FD0000843800608D5A06A2030417B027B0802C6
:100FE000104301D0FFF75AFEA80702D00126FFF7F1
:100FF000D3FFE148C06A817A490849008172DF491C
:101000000120183988470220FFF73DFFDD496420A1
:101010008847002469460C70254601217F20FFF790
:10102000FAFE00210A20FFF7F6FE22210A20FFF730
:10103000F2FE69460A20FFF7ECFE6846007840079A
:10104000EFD469460A20FFF7E4FE684600784007BF
:1010500005D568460078000706D4012504E0641C25
:10106000C948A4B28442ECD3C64964208847002012
:10107000FFF709FFC149019818398847BE48C06A7F
:10108000817A4908490039438172002E02D0B9485B
:101090000C388047002D01D00120FEBD0020FEBD90
:1010A00010B51121B64802F034FD10BD70B50446EC
:1010B000401C02F073FD022818D0042819D0012129
:1010C0004904884247D125462035687B092301071A
:1010D0000209090F0020072A1CD0032A20D0022A67
:1010E00025D0012A29D0002A2DD032E0FFF7D8FFE1
:1010F0003AE0A14D0121E868FF302130017501F08F
:101100005EFEE8688078002801D1FFF750FFFFF706
:1011100085FE29E0581A062148434121C94304E0CD
:10112000581A062148433521C943081A10E0581AB5
:10113000062148432321C943F7E7581A06214843AB
:101140001721C943F1E7581A06214843801D404240
:1011500040B2687308E040281DD00121C9038842CD
:1011600002D1601DFFF704FE854948780978000226
:101170000843800607D5601C02F010FD0005000F33
:1011800001D0FFF78BFD7C483C3002F007FD0146A3
:101190002046884770BD7848383002F0FFFC400692
:1011A000E2D570BDF0B5744C0646E0688DB0FF30F6
:1011B0002130407C0D46002829D0002D26D072B663
:1011C000A068183002F0EAFCE1683222FF312131D8
:1011D000897C6E4B514340186A463221984762B66B
:1011E000002E04D0E068FF302130807C3070E7684A
:1011F0000A21FF372137B87C401C02F041FCB9744A
:10120000E078401CC0B2E0700A2802D900200DB07E
:10121000F0BD684600780128D1D100A907222846F0
:10122000013102F05DFC2A22E81D02A902F058FCFF
:101230000120ECE7F0B5054655498DB020208847E0
:101240004D4C0426E16820690F4686700822C01CB8
:10125000C931BD3702F044FC2069042239460B3005
:1012600002F03EFC0D214B4A03209047E0682946DE
:1012700008220A31C13002F033FCE068294604221A
:101280001231B93002F02CFC287A434F002802D1E9
:10129000687A00281FD00020E070E0682A7A0146B2
:1012A0008030837B9A420AD16A7AC07B824206D11F
:1012B00008222846903102F04CFC002817D06946DD
:1012C0000020FFF76FFF012826D006220021334BB4
:1012D000012098479BE7E06802228179114302468A
:1012E0008171C132FF3011461030B84710E0E0681C
:1012F0008179024631438171C13211469830B84735
:10130000E06880308079012802D121490220884795
:101310002248A03080477AE7E06801A92A228E306F
:10132000033102F0DDFBB8E77CB5451C80782978F5
:1013300000020843104C022810D00F2810D00121C1
:101340001D2810D0FF3810280DD0154A69460120FD
:101350009047687829780002084302E0032000E003
:10136000022060717CBD61717CBD0348407970478B
:101370000C4908471347000048310020BF650000B2
:101380005B3B00202B620000FFFF00005953000070
:10139000050B00004D11000019220000D9190000B2
:1013A0001F1D0000B34400001CB5FF480821017058
:1013B00000214170017BC27A0902C01C114341D057
:1013C0004279037912021A43891A0BB26A461380D2
:1013D000417A027A0906091411436A46518019229A
:1013E0000624D201062B02DA6B461C8003E09342EE
:1013F00001DD6B461A80062902DA69464C8003E05B
:10140000914201DD69464A80417B027B080210431C
:101410006946C880E448817B427B080210436946E4
:101420008880E248C0682330417C027C0802104377
:1014300002D00020FFF7E0FBDD4968468847DD4920
:10144000402088471CBDD84948780A7800021043DC
:10145000C2050CD5FF22013290430870000A487083
:101460000879401E0006000E087109D09CE7202272
:10147000104310229043042210430870000A487061
:101480007047FEB5C84D04466878297800020843C5
:1014900000077DD5C848804769782A78090211433A
:1014A0000822914329700A0A6A706B7A0646284618
:1014B0001A066ED5A27967791202651C3A43BB4FB2
:1014C000E41C002A77D01022114301700A0A4270EE
:1014D00088065ED4687929790002084332D002F088
:1014E000D5FF01910090607821780002084302F056
:1014F000CDFFB24C0022234602F0C2FE019B009AAF
:1015000002F0BEFE01910090F8682130417C027C1F
:101510000802104302F0BAFF0022234602F0B0FE98
:1015200007460C46687A297A00020843801B02F0BD
:1015300099FF3A46234602F0A3FE019B009A02F06F
:10154000EDFD24E0607821780002084302F083FF7B
:101550000446F8682130417C027C0802104302F006
:101560007AFF214602F006FD02F0FAFF0022934BBB
:1015700002F086FE07460C46687A297A0002084384
:10158000801B02F06FFF3A46234602F079FE02E02C
:101590006EE064E00FE00022894B02F0D9FE02F019
:1015A000C1FF0104090C00D10121864B00228020DB
:1015B000FFF76FFB53E09A0651D58278012A4ED18E
:1015C0008A064CD4FF227848013211430170090A7F
:1015D0004170607821780002084373490A7BCB7A16
:1015E0001102194388423AD902F035FF0446F868DF
:1015F0002130417C027C0802104302F02CFF21467E
:1016000002F0B8FC02F0ACFF00226C4B02F038FE96
:1016100007460C46687A297A00020843801B02F0CC
:1016200021FF3A46234602F02BFE0022644B02F0D3
:101630008FFE02F077FF0104090C00D10121614BFC
:1016400000228020FFF725FB5748417802780902E5
:101650001143FF22013211430170090A4170032036
:101660006946088102229103574C02AB0020A04733
:10167000FEBD10B50446007800280DD1A17862782F
:101680000802104309D001281ED0032827D00C28B7
:1016900002D1201DFFF748FE10BD01F0DFFA4B49D3
:1016A000201D8847002802D12820FFF72FF8201D91
:1016B000FFF7E7FE3D480121C36806220904002028
:1016C000414C3133A04710BD01F0C8FA4049201DFC
:1016D00088470028F7D12820FFF718F810BD201DF3
:1016E000FFF7A8FD10BD10B50078012801D1FFF764
:1016F00024F810BDF0B5374885B0804701217F2020
:10170000FFF789FB69465020FFF783FB68460078A6
:10171000042801D030488047FFF780FB234CE06865
:10172000807801286DD002287ED0FFF740FC01258B
:1017300068464580058029481E49019068468439DD
:10174000884768460570457000254580244801900B
:10175000244BE06808226946C01802F0C1F9164E11
:10176000012140205E3EB04701218020B047012189
:101770002020B047FF210C31684601800B214180B9
:101780008580C580058145818581C5811648049085
:10179000164968468847A0680A3002F0FFF9024AF5
:1017A000134B573A572126E05B3B0020483100207D
:1017B00033420000B3440000BF5500000000F43F76
:1017C0000000594047140110A13E00005D5B00007D
:1017D000475F0000793D0000F7460000E716011062
:1017E0003F0B0110CE020000731601108D43000064
:1017F0005953000005E0984701F0E1FA012005B0D7
:10180000F0BDFE4880470746E06A817ACD07817ABD
:10181000ED0F490849008172F84E0120183EB0478B
:101820000220FFF730FB00E00EE0F5496420884716
:101830000120FFF728FB3846B047E06A817A490863
:1018400049002943817272E70220FFF71CFB6EE713
:1018500010B5EC488047012010BDEA4910B51E3193
:101860008847012010BDE74910B554318847012051
:1018700010BDE44910B560318847012010BDE14931
:1018800010B56E318847012010BDDE4910B57E319C
:101890008847012010BD10B5DA4CE634A04701207E
:1018A00010BDF8B5D84CD949E06837308847206971
:1018B0003B230178BF250A09E16812015B5C1B0725
:1018C0001B0F1A4302701207120F012A79D00B4620
:1018D00040335A781B7812021A430B4642331A706F
:1018E000120A5A7002788B7A2A409B011A435206D8
:1018F000520E027066235B5C42789B1D92099B0628
:1019000092019B0E1A4342700622801C0B3102F09A
:10191000E7F8E1686620425C002A04D0206967315C
:10192000083002F0DDF8E0680021203041772069BE
:10193000B74A41788906890E891C90472069017849
:101940000A091201121D0270E1682A408B7ADB0736
:101950005B0E1A43027046235B5C42789B1D920922
:101960009B0692019B0E1A4342700622801C0B318B
:1019700002F0B6F8E1684620425C002A04D02069F3
:101980004731083002F0ACF82069A14A41782C3286
:101990008906890E891C9047E06801270546203595
:1019A000E97E01293BD000294CD002294AD00629E2
:1019B00048D00023974C1A4601211846A047F8BD8D
:1019C000FFE70A464032137953718B7A0278DB07BE
:1019D0002A405B0E1A43027087235B5C5206520E4C
:1019E000DB011A43027042780B31920992010C32EA
:1019F00042700622801C02F073F82069E16806221A
:101A00000830883102F06CF8E16803223D2042542E
:101A10007E4A8720405C323A8831904787E74030E1
:101A2000417900290AD028200621A26A937EFD244C
:101A30002340937617756B7F2A7F43E0477101201F
:101A40000146F2E706464236717832780B021343BC
:101A500017D0192189014B432230417F047F0802AE
:101A6000204301228004800C009006D001461846D5
:101A700002F006F8421C7F2A10D8D4B23770380A18
:101A800014E03770390A71702230417F027F0802FA
:101A9000104301248004800C009008E07F2410464D
:101AA00021467E3001F0ECFF3070000A707056481D
:101AB000806A817E02221143817607756B7F2A7FBF
:101AC00000992046544CA04753483E30804776E763
:101AD00010B5FFF7E6FE012010BD10B54F490320F9
:101AE0000870474964201A3188474D4880470120D3
:101AF00010BD72B60021444A906A4175037C0121F1
:101B00000B430374D0684522115442300170002108
:101B1000417062B60120704710B5424988470120E4
:101B200010BDF0B5384CA56A2C4660342678FD27E8
:101B3000C0073E40800F06432670A1706270623578
:101B40002B71180A687105982071000A6071F0BD48
:101B5000F8B52D4D2D49E868373088471120EF68DA
:101B6000002480013D186E79A8790321401C01F002
:101B700087FF01208840A971064203D1641CE4B2AA
:101B8000032CF1D31125AD017C19607B217B000270
:101B90000843A91C7F18010A1B4E3873797300286B
:101BA0000BD0607A227A010219201143800101F0E2
:101BB00067FF0206120E04D004E0012038730020F3
:101BC00078730122787A397A000208430090607AAB
:101BD000217A03020B43A0791349095CE079FFF7EE
:101BE000A0FFF068002140190171C17001744174B7
:101BF0008178002901D008291AD917E0BF650000B3
